:10200000008000203DD5000025D5000025D500002A
:1020100000000000000000000000000000000000C0
:1020200000000000000000000000000025D50000B6
:10203000000000000000000025D5000091D5000040
:1020400025D5000025D5000025D5000025D50000A8
:1020500025D5000025D5000025D5000029D5000094
:1020600025D5000025D5000025D5000041AC000095
:1020700031AC000025D5000021AC000025D50000C2
:1020800025D5000025D50000A127000061800000B3
:102090000000000025D5000025D5000025D5000052
:1020A00025D5000025D5000025D5000025D5000048
:1020B0000000000010B5064C2378002B07D1054B1B
:1020C000002B02D0044800E000BF0123237010BDA4
:1020D0004802002000000000804A0100044B10B5B7
:1020E000002B03D00349044800E000BF10BDC046E8
:1020F000000000004C020020804A010000207047D0
:102100007047704770B5054C25000C3C6C352800B5
:102110000C3D0AF06EFEA542F9D170BD3C060020D0
:1021200070B5054C25000C3C6C3528000C3D0AF0C0
:1021300060FEA542F9D170BDC405002070B5054C04
:1021400025000C3C6C3528000C3D0AF052FEA542DF
:10215000F9D170BD240A002070B5054C25000C3C57
:102160006C3528000C3D0AF044FEA542F9D170BD43
:10217000AC09002070B5054C25000C3C6C352800DE
:102180000C3D0AF036FEA542F9D170BD140B0020BB
:1021900070B5054C25000C3C6C3528000C3D0AF050
:1021A00028FEA542F9D170BD9C0A002010B5080098
:1021B0000EF000FB10BD10B5080011000FF05AF82A
:1021C00010BD10B508000EF0FFFA10BD70B5114C2F
:1021D0002378002B0FD004200BF046FD00280AD0F6
:1021E00001240D4D1120297861400BF011FD2B7851
:1021F0005C402C7006E02378002B04D001211120D4
:102200000BF006FD70BD04200BF02EFD0028F5D06C
:10221000E6E7C046880200202000002010B500211B
:102220000C200BF0F5FC012114200BF0F1FC012136
:1022300015200BF0EDFC10BD074A03000020914271
:1022400008D0CA091B68D2007F309B18014058682B
:10225000C90040187047C046FFFF000070B5074B2B
:102260000D0041880400994206D02C321000FFF77F
:10227000E3FFC580658070BD0580FBE7FFFF0000C0
:1022800070B5040008000D000FF050F8024B6560B7
:10229000A0602360200070BDCC06002010B50AF0BD
:1022A00083FF030001205840C0B210BD10B50400E8
:1022B0008B680BF013F8200010BD10B50A004369BD
:1022C000016908F07DF810BD10B54269016908F098
:1022D000C7F810BD0A4A10B50B0004000020944254
:1022E0000CD8210009318C4208D81A6818001268ED
:1022F0009047002802D00123C480838010BDC046CF
:10230000FFFF000070B505000C002968002906D009
:102310000B6820002B6023685B689847F5E770BD69
:1023200070B504000D001600081E01D00EF0FEFF6F
:10233000256060602672200070BD70B5C5882C31A4
:10234000040008002900FFF777FFA580206000281F
:1023500001D0C388E38070BD70B50025436A0400D6
:10236000C3181D71011D00680AF09EFEA84200D02E
:102370006562606A70BD70B5436A040001330D0088
:102380001F2B06D80120636A5A1C6262E41825716B
:1023900070BDFFF7E1FF0028F4D00020F8E770B52A
:1023A000037904000D00DB0714D500220168AB6837
:1023B000002B0FD0994226D18B882868013B9BB215
:1023C0008B80002B06D10B68002A1AD0136003689B
:1023D0005B6898472379DB0608D5280026882C30CF
:1023E0003100FFF729FFAB8E0380AE866023227990
:1023F0001A4203D02900200000F008F800232371BE
:1024000070BDAB60E3E71A001B68D1E7F7B50700C2
:102410000D0004880B4B9C420FD0280021002C306B
:10242000FFF70AFF0600C38829000193FFF7B7FFF3
:10243000AB8E3380AC86019CECE701235B423B8092
:102440007B80F7BDFFFF0000F0B505000F0044687A
:10245000634A238885B013402380E37BDB09FCD1EA
:102460003E686049301C0BF0B1FE002839D0E023F3
:102470002288DB00134323808023DB006B61E67B33
:10248000F609FCD168690EF05BF802900391386898
:102490000EF0C2F80022544B0CF03CFE02000B0080
:1024A000029803990CF036FE02000B0000204F4901
:1024B0000CF030FE0EF00EF8431EAB61208A228B2A
:1024C00080B2009392B2330031000AF0DFF980B29B
:1024D0002082AB699BB22383E37BDB09FCD105B08F
:1024E000F0BD4349301C0BF071FE00280DD03D4972
:1024F000301C0BF061FE002807D0C0232288DB00CF
:102500001343238080235B00B8E73A49301C0BF06B
:102510005DFE00280CD03649301C0BF04DFE002823
:1025200006D0A0232288DB00134323804023A5E7A5
:102530003149301C0BF04AFE00280CD02D49301CCC
:102540000BF03AFE002806D080232288DB001343DC
:102550002380102392E72949301C0BF037FE002816
:102560000CD02549301C0BF027FE002806D0C023D4
:1025700022889B001343238008237FE72049301CD7
:102580000BF024FE00280CD01C49301C0BF014FE6C
:10259000002806D0802322889B0013432380042335
:1025A0006CE71849301C0BF011FE00280CD01449C0
:1025B000301C0BF001FE002806D0802322885B002F
:1025C00013432380022359E70E49301C0BF0F4FD1E
:1025D000002800D153E723889BB2238001234DE7D5
:1025E000FDF8FFFF007C924880842E4160E3864125
:1025F00000409C4700409C4600401C4600409C45D3
:1026000000401C4500007A44F8B506000F004468FD
:10261000584A236813402360A3689B07FCD43D6895
:102620005549281C0BF0D2FD002825D0E023226854
:10263000DB00134323608023DB00736170690CF0BF
:1026400003FA4E49051C38680BF0D4FE011C281C07
:102650000BF0D0FE011C4A480BF0CCFE0CF0D4F974
:102660000138B0612064A3681B06FCD4454B636449
:10267000A368DB05FCD4F8BD4349281C0BF0A6FD7C
:1026800000280DD03C49281C0BF096FD002807D0EF
:10269000C0232268DB001343236080235B00CCE768
:1026A0003A49281C0BF092FD00280CD03649281C12
:1026B0000BF082FD002806D0A0232268DB00134324
:1026C00023604023B9E73249281C0BF07FFD002826
:1026D0000CD02E49281C0BF06FFD002806D080235B
:1026E0002268DB00134323601023A6E72949281C36
:1026F0000BF06CFD00280CD02549281C0BF05CFD6C
:10270000002806D0C02322689B00134323600823BF
:1027100093E72149281C0BF059FD00280CD01D49D6
:10272000281C0BF049FD002806D0802322689B005E
:1027300013432360042380E71849281C0BF046FD4F
:1027400000280CD01449281C0BF036FD002806D0B8
:10275000802322685B001343236002236DE70F4947
:10276000281C0BF029FD002800D167E723682360AF
:10277000012362E7FDF8FFFF007C924800247449C2
:10278000001B374CFF0F000000409C4700409C4658
:1027900000401C4600409C4500401C4500007A4417
:1027A00010B5064B9A7BD20606D51022997B0A43B8
:1027B0009A73034B1B68984710BDC046002C00421B
:1027C0000C05002070B504000968594815000BF08D
:1027D00011FE26782061022E58D856490BF0F6FCDF
:1027E00003000020834249D13F22534B7600F35A25
:1027F0001A408023DB011343504A1380504A537818
:10280000DB09FCD10221626813888B431380626864
:1028100013889BB213806368DA7BD209FCD11988D4
:1028200020320A431A806368DE7BF609FCD121005E
:1028300020001031FFF708FE63685E7310236268A2
:10284000517B0B43537323783E4AD25C1F231A40BB
:102850001E3B93403C4A13600223626811880B437D
:1028600013806268D37BDB09FCD12078A560374BED
:10287000002809D0012802D1354B1D6070BD022807
:1028800001D00120FAE7334B1D60FAE7F31E022B5B
:10289000F7D83F22284B7600F35A1A408023DB01F9
:1028A0001343264A1380264A5378DB09FCD10221C0
:1028B000626813688B431360626893689B07FCD45B
:1028C000210020001031FFF79FFE6368DA6BDA63A6
:1028D000626893685B06DB0FFBD19362616801332A
:1028E0008A6A1A438A62802261685202886A0243B5
:1028F0008A62227813498A5C1F210A409340124A57
:1029000013600223626811680B4313606268936866
:102910009B07FCD42378A560032B01D10E4BB3E7B2
:10292000042B01D10D4BAFE7052BAAD10C4BABE724
:1029300000247449ABAAAA49C2340100020C004029
:10294000000C00400038010000E100E00C05002010
:102950001005002014050020200500201805002087
:102960001C050020F7B505000AF020FE00242427EE
:1029700001903E0066432422A81900210DF06BFF50
:10298000019B01347351102CF3D1902300229B0042
:10299000EA50F7BD90239B00C35802000F2B0CDCBC
:1029A000002024210B004343D3185B68002B03D085
:1029B00001301028F6D11138704701204042FBE762
:1029C000F7B5009308AB1B780500019390239B009B
:1029D000C3580C001700002B01DAFFF7C3FF2800D3
:1029E000FFF7D8FF061E1BDB002F19D02368242415
:1029F00044432C192361009B6760A3606B461B79DD
:102A00002373099B1B686361012323770AF0CEFDC2
:102A1000902220609200AB580133AB503000FEBDD5
:102A200001267642FAE71FB5002303AC0194009318
:102A30000393FFF7C5FF04B010BDF8B504000868A4
:102A40000F000F2816D89026B600A359002B11D0DE
:102A50002425684320184368002B0BD02A0000214E
:102A60000DF0F9FE3F680AF0A1FD7D432851A359FE
:102A7000013BA351F8BDF0B585B006000AF096FD04
:102A800000250700242400236C4334192362636863
:102A9000002B1AD023682269FB1A934215D32068B1
:102AA00021692369381A0093236801930BF0B4F964
:102AB000009B5843019BC0182060237F002B04D04B
:102AC0006369002B22D1013323620135102DD9D146
:102AD000002414352B006343F3181A6A002A10D01F
:102AE0001A7B002A21D05A68986890472B006343CC
:102AF000F3181B6A022B04D103A930000394FFF7DB
:102B00009CFF0134102CE5D105B0F0BDA2696369CA
:102B10009A42DAD201232362A3690133A361A26935
:102B200063699A42D1D30223CEE75B689847DDE719
:102B300010B50248FFF79FFF10BDC0469402002069
:102B400010B50400012809D100210C200BF060F819
:102B5000210015200BF05CF800210AE002280CD1BE
:102B600000210C200BF054F8002115200BF050F838
:102B7000012114200BF04CF803E0032802D1FFF7E9
:102B80004DFB10BD0428FCD101210C200BF040F8B6
:102B90000021DEE710B501292CD1032816D1284BDE
:102BA0001A78002A11D119700100264C200005F076
:102BB00027FB254B1978200005F072FB234B186882
:102BC0000AF02AFD200005F023FB10BD012807D1E3
:102BD0001F4B1A78002AF8D118701E4C0521E5E722
:102BE0000228F2D11C4B1A78002AEED119701B4C26
:102BF0000A21DBE703280CD1114B1A78002AE4D014
:102C0000002201000F4C1A70200005F0F9FA144B55
:102C1000D0E7012808D10E4B1A78002AD5D000221F
:102C20000C4C1A700521EFE70228CED10A4B1A7816
:102C3000002ACAD00022094C1A700A21E4E7C046D3
:102C40007A0700203A070020140000201C00002012
:102C5000780700203407002079070020370700207C
:102C6000C005002070B5040086B0302832D17C4BFE
:102C70001B78002B02D031227A4B1A6030227A4B1B
:102C8000002110201A700AF0C3FF00210F200AF063
:102C9000BFFF00210E200AF0BBFF002107200AF031
:102CA000B7FF01210C200AF0B3FF704B1B78013BEA
:102CB000022B49D80420FFF743FF00210120FFF732
:102CC00069FF00210220FFF765FF00210320FFF7C5
:102CD00061FF39E0312839D1634B01211870102090
:102CE0000AF096FF00210F200AF092FF00210E202B
:102CF0000AF08EFF002107200AF08AFF5B4C25783E
:102D0000012D06D103202900FFF744FF2800FFF71B
:102D100017FF2578022D0AD101210800FFF73AFF9D
:102D200028000021FFF736FF0120FFF709FF237875
:102D3000032B09D101210800FFF72CFF01210220FC
:102D4000FFF728FFFFF76AFA06B070BD322821D1DD
:102D5000464B1D78022DF7D1434B002118701020EF
:102D60000AF056FF01210F200AF052FF01210E2028
:102D70000AF04EFF002107200AF04AFF002101203F
:102D8000FFF708FF28000121FFF704FF2800FFF7E5
:102D9000D7FED9E733282DD1002110200AF038FFC3
:102DA00001210F200AF034FF00210E200AF030FF2D
:102DB000012107200AF02CFF2C4E3578012D08D177
:102DC000294B032029001C70FFF7E4FE2800FFF7C1
:102DD000B7FE3378023B012BB6D83322224B0420B6
:102DE0001A70FFF7ADFE01210800FFF7D3FE0121A5
:102DF00002206CE73428A7D11C4B1B4D1E78012EF6
:102E000013D1002110200AF003FF00210F200AF047
:102E1000FFFE31000E200AF0FBFE002107200AF021
:102E2000F7FE0420FFF78CFE2C70114903A80AF06E
:102E30002FF8297868460AF04AF8694603A80AF08C
:102E400062F90C490AF06CF901000B4809F03CFFEB
:102E5000684609F0CEFF03A809F0CBFF74E7C0462F
:102E60002400002084020020900200202C0000207A
:102E7000272C0100732E0100401A0020F0B5D94C18
:102E80000123A5440400FFA80092983000220F00FF
:102E90000AF024FAFFA8D4499830FFF7FFF906009A
:102EA000FFA8983009F0A5FF002E2FD0CF4EFFA825
:102EB0003100983009F0ECFFFFA8390098300AF093
:102EC00022F9CB4D29000AF02BF90100C94809F07D
:102ED000FBFEFFA8983009F08CFFFFA83100983066
:102EE00009F0D6FFFFA8390098300AF00CF9290044
:102EF0000AF016F9010020000AF051F8FFA89830F6
:102F000009F077FF2000BC4B9D44F0BDFFA8BB49F2
:102F1000983009F0BDFFFFA90222983138000AF06D
:102F2000A1F901220300390005A80AF0D7F9FFA88A
:102F3000983009F05EFFB24D0BA8290009F0A8FFF8
:102F400029000EA809F0A4FF290011A809F0A0FF8C
:102F5000290014A809F09CFF290017A809F098FF80
:102F600029001AA809F094FF29001DA809F090FF74
:102F7000290020A809F08CFF06250295BB68019561
:102F80009D4229D20135FFA82B00019A39009830C3
:102F90000AF0A4F9FFA8994998300AF005F90390BE
:102FA000FFA8983009F025FF039B002BE6D0FFA86F
:102FB000029A019B390098300AF090F90C20704376
:102FC0000BABFFA91818983109F0F3FFFFA8983050
:102FD00009F00FFF0136D0E78A4905A80AF0E4F8A6
:102FE0008949061E00D0C5E2884905A80AF0DCF828
:102FF00000283DD0009B7E4D8549864F002B11D186
:103000007C4E300009F031FE3900300009F038FE06
:103010002900300009F062FE7F49200009F038FFE6
:10302000002616E0FFA8983009F032FFFFA839000B
:1030300098300AF039F8FFA8290098300AF034F8DF
:10304000FFA99831200009F0C9FEFFA8983009F0C7
:10305000D0FE20AD08AF28000C3D09F0CAFEBD42ED
:10306000F9D105A8012E00D0BBE309F0C2FE49E763
:103070006A4905A80AF098F8061E28D0009B5C4F04
:103080006749684E002B0AD15A4D280009F0F8FD17
:103090003100280009F0F4FD39002800BAE7FFA844
:1030A000983009F0F5FEFFA83100983009F0FCFFD8
:1030B000FFA83900983009F0F7FFFFA998312000E8
:1030C00009F08CFEFFA8983009F093FEA8E7564956
:1030D00005A80AF069F8002841D0009B444D5349E7
:1030E000002B1FD1434E300009F0BFFD504B022290
:1030F0001968A4A809F06EFFFFA8A4A9983009F0E8
:103100004EFFFFA8290098300AF00AF801003000AD
:1031100009F0DAFDFFA8983009F06BFEA4A809F0C9
:1031200068FE79E7A4A809F0B3FE414BFFA819682F
:103130000222983009F04EFFFFA99831A4A809F0A7
:10314000A1FFFFA8983009F054FE2900A4A809F0B7
:10315000ABFFA4A9200009F041FEA4A877E73549F8
:1031600005A80AF021F8002800D055E7324905A843
:103170000AF01AF8051E00D04EE7304905A80AF0FB
:1031800013F8061E11D00BA80AF0AEF92C4B1B78D1
:10319000002B00D140E73020FFF764FD294B1D6074
:1031A000294B1D60294B1D7036E7294905A809F0F8
:1031B000FBFF002871D001250BA80AF095F93122F8
:1031C000204B07001D60204B1D601D4B1A701F4BCC
:1031D000C2B21E701F4B002A3ED131201A70FFF779
:1031E00041FD19E764F9FFFF7C3A0100492D010018
:1031F000732E0100401A00209C060000533201008B
:1032000023380100682D01006D2D0100752D01008E
:103210007A2D0100812D01001D380100852D01004E
:103220008A2D0100912D0100C02D0100C52D010046
:103230009C090020CC2D0100D12D0100D62D0100CC
:103240009002002084020020800200202400002040
:10325000DB2D01000C0700200EA81D700AF044F9B8
:10326000060011A80AF040F9FF22FA2317409B003C
:103270005F43D5490F60F7B21900D44B002F09D135
:103280001D60C0B24843D24B18600AF08FF9D14B91
:103290001860C1E616401E60F3E7CF4905A809F0A3
:1032A00083FF00281DD0CD4B1B78322B01D1012686
:1032B000CFE6CB4B1D78022D0AD13220FFF7D2FC8E
:1032C0000022C84B1D60C84B1D60C84B1A70EEE74A
:1032D000009BC749002B00D09FE6C64809F0EAFCD6
:1032E0009AE6C54905A809F05FFF071E16D0BB4B3B
:1032F0001B78332B00D18FE63320FFF7B3FCB84B9C
:10330000B8491A78B84B022A06D101321A600A600D
:103310000022B64B1A707FE60222F7E7B74905A8EC
:1033200009F042FF061E12D0AC4B1B78342BBED0E6
:10333000AB4B1E78012ECBD13420FFF793FC032337
:10334000A84A1360A84A1360A84B1F7081E6AC49D5
:1033500005A809F029FF00283BD0009BFFA8A94D34
:103360009E4FA9499830002B19D109F091FD397869
:10337000A4A809F0ACFDFFA8A4A9983009F0C3FEE9
:10338000290009F0CDFE01009A4809F09DFCA4A88F
:1033900009F02FFDFFA8983009F02BFD3CE609F05D
:1033A00077FD3978A4A809F092FDFFA8A4A9983068
:1033B00009F0A9FE290009F0B3FE0100200009F080
:1033C000EEFDA4A809F015FDFFA8983009F011FD45
:1033D0003FE68E4905A809F0E7FE061E20D08C497D
:1033E000A4A809F055FD7E4BFFA819780A22983051
:1033F00009F07BFDFFA99831A4A809F043FEFFA8BE
:10340000983009F0F6FC7F49A4A809F04DFE009B16
:10341000A4A9002B00D0E0E1764809F055FC80E03B
:103420007C4905A809F0C0FE0190002825D00BA812
:103430000AF05AF8C5B26B1E022B14D87649774AA7
:103440000D7023A80DF0EBF9754F3800FEF73CFF27
:1034500023A93800FEF731FF614B72491D70009BB4
:10346000002B06D139E7009B6F49002B00D134E7D0
:103470006E49200009F0DDFDEBE56D4905A809F076
:1034800093FE061E55D00BA80AF02EF8C3B2050015
:10349000B42B4CD8674EEDB20521300004F0B0FEDD
:1034A0002900300004F0FCFE634F38680AF0B4F8DD
:1034B000300004F0ADFE614E0A21300004F0A0FEA1
:1034C0002900300004F0ECFE38680AF0A5F830005E
:1034D00004F09EFE5A4E0321300004F091FE2900B4
:1034E000300004F0DDFE38680AF096F8300004F091
:1034F0008FFE5449A4A809F0CBFC394BFFA81978DA
:103500000A22983009F0F1FCFFA99831A4A809F02B
:10351000B9FDFFA8983009F06CFC4B49354809F01B
:10352000C9FB4A49200009F0B3FCA4A8CCE54849EE
:10353000D3E6484905A809F037FE002822D00BA899
:1035400009F0D2FFC5B26B1EDBB2B22B11D83249E3
:10355000324A4D70A4A80DF062F9314F3800FEF7E1
:10356000B3FEA4A93800FEF7A8FE3B4B3B491D70F3
:1035700075E73B49009B002B00D1AEE6200009F027
:1035800058FD4DE5374905A809F00EFE00286FD01B
:103590000BA809F0A9FFC5B26B1EDBB2B22BE8D8AD
:1035A0001D49FFA88D701D4A98300DF038F91C4E4A
:1035B0003000FEF789FEFFA998313000FEF77DFE4E
:1035C000294B2A491D70D5E7100700201407002059
:1035D000180700201C070020E02D010090020020A9
:1035E0002C00002084020020800200202400002003
:1035F000E52D0100401A0020FD2D0100022E0100E2
:10360000072E0100732E0100272C01000C2E010053
:10361000112E0100182E0100800700200202000078
:10362000840900201D2E0100452E0100762E010088
:10363000A82E0100340700201C00002037070020BE
:103640003A070020AD2E0100B52E01001D38010003
:10365000C02E0100CB2E0100C0050020D02E01009D
:10366000FB2E0100292F0100140000202E2F010045
:103670005E4905A809F098FD002805D05C49A4A87A
:1036800009F006FC5B4BAFE65B4905A809F08CFD31
:10369000002805D05949A4A809F0FAFB584BA3E625
:1036A000584905A809F080FD002865D00BA908A895
:1036B00009F075FC0EA923A809F071FC524E0023F5
:1036C000FF22310008A809F09FFD504D0023FF2282
:1036D000290023A809F098FD4D4908A809F064FDC8
:1036E0004C4C00283FD000234B4908A8237009F018
:1036F00066FC3100FF2249480DF01FFE2900FF2221
:1037000047480DF01AFE23784649FFA8CB70464A79
:1037100098300DF084F8454C2000FEF7D5FDFFA948
:1037200020009831FEF7C9FD4149A4A809F0B0FB7B
:1037300008A9A4A809F0E7FC3E4909F0F1FC010042
:103740003D4809F0C1FAA4A809F053FBFA20800013
:1037500009F062FFBFF34F8F384B394ADA60BFF38D
:103760004F8FC046FDE7374908A809F01DFD002826
:10377000B9D101232370BCE7334905A809F014FD32
:10378000002800D193E53149A4A809F081FBFFA8E6
:103790001D49983009F07CFBFFA99831A4A809F0D5
:1037A00071FCFFA8983009F024FB2949A4A809F06E
:1037B0007BFCFFA81549983009F06AFBFFA99831F6
:1037C000A4A809F05FFCFFA8983009F012FB20497B
:1037D000A4A809F069FC0F4B06E6200009F0FEFAE8
:1037E000A3E609F006FBFFF78DFBC0465A2F010048
:1037F0005F2F0100C0050020662F01006B2F010024
:1038000014000020722F01009C0C00209D0B002052
:103810001D3801009C0B0020772F01008407002039
:103820008308002080070020020200008409002095
:10383000832F0100942F0100401A002000ED00E0CA
:103840000400FA0523380100A12F0100A62F010072
:103850005332010073B509F0A9FE164D04002B7810
:10386000002B0ED1144E154A3368C31A934208D95F
:103870001349684604F0D8FE124B34601C600123E3
:103880002B702B78002B13D00E4B1B68E41A0E4BB9
:103890009C420DD900210A4804F068FF0B49041C22
:1038A0000AF07AFC002801D1094B1C6000232B7020
:1038B00073BDC046A009002020070020CF070000EC
:1038C00058070020A4090020ED0200000000FEC2FD
:1038D0009C090020F8B53E4B1B78002B52D009F014
:1038E00065FE3C4B3C4D1C683C4F2A68041B3C4E1B
:1038F0003B68012A47D19C424BD2FEF78FFC012145
:103900000800FFF747F901210220FFF743F93B6860
:103910009C421BD32F68012F18D100222C4B04206E
:103920001A70FFF70DF900213800FFF733F9002175
:103930000220FFF72FF939000C200AF069F9302234
:10394000284B294929481A7009F0B4F933689C4278
:1039500018D32B68023B012B14D800241C4B0420E5
:103960001C70FFF7EDF821000120FFF713F921008B
:103970000220FFF70FF930221A4B1B491B481A701F
:1039800009F098F9F8BD022A0CD13268D31A9C428A
:10399000B3D80420FFF7D4F800210120FFF7FAF88C
:1039A0000021B1E7032AB2D15B089C42A5D332685B
:1039B000D31A9C42EDD39442EBD201210800FFF7C9
:1039C000E9F801210220FFF7E5F8FEF727FC9EE762
:1039D0000C0700201C0700201407002010070020FF
:1039E0001807002090020020F32C0100401A00204C
:1039F000F0B5002406002700250089B0019102924D
:103A00000393B3689C4223D8039A954220DA9C42E0
:103A100016D16B1C00930C235D43029B3A005D1989
:103A20003100230005A809F059FC05A9280009F078
:103A3000C0FA05A809F0DDF9009D671C0134E0E734
:103A40002100300009F0DCFB019B9842F6D1E0E751
:103A500009B0F0BD4B6843608B688360CB68C3607E
:103A6000044B03600B7C03744B8A43820B7D03750C
:103A70007047C046003C01007FB51A4E1A4930001D
:103A800009F018F9194C01A8210009F088FA184D1D
:103A900001A8290009F044FB21000C3109F033FB97
:103AA000290009F03DFB2100183109F02CFB290009
:103AB00009F036FB2100243109F025FB290009F02B
:103AC0002FFB2100303109F01EFB0100300009F00E
:103AD000FBF801A809F08DF9CA22064B52001A80A2
:103AE0007FBDC046401A0020883401009C0A002097
:103AF0009234010022000020F0B500275A4B040048
:103B000089B05A495A481F7009F059FA594E05A808
:103B1000310009F0BDF905A9200009F0B3FB05004B
:103B200005A809F066F96B1C00D19AE00C257D43CD
:103B3000514B31005B1902A8009309F0A9F902A9C1
:103B4000200009F09FFB00220300210005A809F0D6
:103B5000C5FB05A9009809F02CFA05A809F049F958
:103B600002A809F046F9310002A809F091F902A96A
:103B7000200009F087FB2100421C05A8FEF796FBF8
:103B800005A9200009F015FA05A809F032F902A8E4
:103B900009F02FF9394E05A8310009F079F905A986
:103BA000200009F06FFB019005A809F022F9344BC1
:103BB0005D19019B01334FD0310002A809F068F96B
:103BC00002A9200009F05EFB00220300210005A8E5
:103BD00009F084FB05A9280009F0EBF905A809F014
:103BE00008F902A809F005F9310002A809F050F916
:103BF00002A9200009F046FB2100421C05A8FEF79F
:103C000055FB05A9200009F0D4F905A809F0F1F841
:103C100002A809F0EEF81B4905A809F00AFA05A95F
:103C2000009809F0B3FA060005A809F0E2F8002EA2
:103C30000ED00F4E2900300009F0A1F912493000D2
:103C400009F0B2FA002803D00849300009F0B7F9AA
:103C5000054B01371F7059E72100280009F08FF943
:103C6000D9E7012009B0F0BDC105002023380100CB
:103C70007402002094340100C40500209634010031
:103C80003C060020983401001D380100F8B50500FD
:103C90000F0000240D4B1B78A34211DD0C26664358
:103CA0000B483900801909F071FA002806D009493B
:103CB0002800891909F073F92800F8BD0134E9E7F3
:103CC0000549280009F0E4F8F6E7C046A8090020F5
:103CD000AC090020140B00201D380100F8B50500C8
:103CE0000F0000240D4B1B78A34211DD0C26664308
:103CF0000B483900801909F049FA002806D0094913
:103D00002800891909F04BF92800F8BD0134E9E7CA
:103D10000549280009F0BCF8F6E7C046C1050020B7
:103D2000C40500203C0600201D380100836870B5E2
:103D30000500002B22D00024AB68A34220D921002B
:103D4000280009F045FA03782B2B01D10134F3E761
:103D50002100280009F03CFA03782D2BF6D0210031
:103D6000280009F035FA03782E2BEFD02100280027
:103D700009F02EFA0378303B092BE7D9002070BDFB
:103D80000120FCE7F8B504000F000026A38C216A8F
:103D9000B3420ED9F5004D196968002903D03B687C
:103DA00038005B689847002301362B606B60B6B221
:103DB000ECE70023A384013B23858C4206D03B68BB
:103DC00038005B68984704232462E384F8BD10B58B
:103DD00004000C302168FFF7D5FF00232000237179
:103DE00008302168FEF78EFA10BD10B504000830C7
:103DF0002168FEF787FA200021680C30FFF7C2FF28
:103E0000200010BDF0B585B0050001AC0191029213
:103E100003930A9E00280BD03100FEF7C0FA019FE1
:103E2000002F05D0237A002B04D004232F602B71A0
:103E300005B0F0BD029C032C1BD81A00E1B2009122
:103E40000098D1B2884205D9B95C01324842484154
:103E50000343F5E7002B0CD102222A710099DAB254
:103E6000914203D9FA5CEA540133F7E700232B555A
:103E7000DEE7B068002815D0C3889C4209D1002332
:103E80009C4208D0C218F95C127A914201D10133E8
:103E9000F6E70068EEE78388013383800523286016
:103EA0002B71C5E731682000FEF714FA00230200E9
:103EB0000832984202D101333371B9E79C4203D0F2
:103EC000F95CD1540133F9E7002304192372B36874
:103ED0000360B060E2E77FB510C902AB60C960C3A0
:103EE0000300446002A9083330C930C3026104B042
:103EF00070BD30B58B8C096A013B9BB2DA00891822
:103F00004C68002C09D04A880D88954205D9551C6B
:103F10004D80D1006118002904D100230360013BCA
:103F2000838030BDDB01D21801608280F9E7000098
:103F3000F0B585B000908D8E384B0C009D420ED0B0
:103F4000080029002C30FEF777F90388A3860023A8
:103F50000371013BC380009B18609D805BE00B00F8
:103F60000C3301930B8E0F68002B09D002A8019926
:103F7000FFF7BFFF0298002802D002AB9D88E6E75A
:103F8000238E668E9E4217D180239B009E423BD09B
:103F90007600E16A0198B6B23B68F20088422ED101
:103FA0001B68110038009847051E2DD0202201996A
:103FB0000CF035FCE5626686268EE36A751CF60019
:103FC0009E19174BADB22586ED186B1E9D413B68BF
:103FD0007F35E9001B68380098477060431E9841A0
:103FE0000023404205403580738002A80199FFF705
:103FF00080FF029802AB9D880028A8D104E09B684E
:1040000038009847051ED5D1012323710023009A5B
:104010001360013B9380009805B0F0BDFFFF0000E6
:1040200000FEFFFF73B5060068460D00FFF780FF36
:10403000009C002C05D06B462A0099883000FEF7C2
:104040000DF9200076BD0023F0B5066885B00F009D
:1040500001939E4219D0456802A82900FFF768FF26
:10406000029C002C11D002AB9B88290020000193F8
:104070003F68FEF794F90C23276023712A00019909
:104080003000FEF7EBF801230193019805B0F0BD75
:10409000F0B5002503688BB003910293AB4221D0A9
:1040A000446805AF21003800FFF742FF059EAE428D
:1040B00018D0BD88039A01270792072207AB1F7209
:1040C00003990094099B30000892FFF79BFE002C97
:1040D0000BD02379002B08D1290022000298FEF78B
:1040E000BDF83D0028000BB0F0BD21003000FEF708
:1040F00056F9A38E3380A5860025F3E707B5CB00DC
:1041000001680822C91868460CF089FB00980199DB
:1041100003B000BD4B680A004360030030B50833AC
:10412000083230CA30C30B69036130BDF8B50500F1
:1041300016000C008F18BC4205D021782800FEF72D
:104140001AF90134F7E7AB6A9E19AE62F8BD70B593
:10415000050008000C000DF0E9F82100020028001D
:10416000FFF7E4FF70BDF0B51624070016001D0030
:1041700087B06C44300029000A2200230AF03AF884
:10418000013C30322270300029000A2200230AF05C
:1041900031F80D0006000143ECD116236B441A1BC5
:1041A00021003800FFF7C2FF07B0F0BDF0B585B0C1
:1041B00001900E00029103921F00081E4ED01500C0
:1041C000032A1DD800221300E8B2D1B2884205D9D3
:1041D000B15C01324C4261410B43F6E7002B0FD139
:1041E000022201990A71DAB2904204D9F25C019973
:1041F000CA540133F7E70023019A535501202DE0FB
:10420000BC68002C21D0E3889D4207D120002A0001
:10421000310008300CF0F4FA002812D02468F0E7DE
:1042200020002A00310008300CF0F9FA002365194B
:104230002B72BB682360BC600523019A1371146064
:10424000DCE7A3880133A380F6E739682800FEF78E
:1042500041F8041EE4D1012320003B7105B0F0BDFC
:10426000F0B58DB002AF00900D0002917A601C0095
:10427000002905D10991012209AB52429A8037E009
:104280002000039B2C300193009B1E883100FDF71A
:10429000D3FF07AB07909E80002815D0C288012667
:1042A000DA80079900294DD0002E44D00B7909A857
:1042B000042B0BD0052B36D00022022B08D0002374
:1042C00003604360013334E0314AE8E701220968C2
:1042D000FEF726F80A9B019A93422CD129000998EF
:1042E0000CF08EFA002826D109AA07AB03CB03C233
:1042F000099B002B06D0210009A8FEF71EF8099D96
:10430000002D0DD105AE330006CF06C307AF210047
:104310003800FFF70DFE079B0193002B14D10025F9
:1043200028000DB0F0BD0B68DA8808330360002365
:1043300042600372CEE70123210007A85E40FDF72B
:10434000FCFFAEE7099196E7210009A8FFF7F0FD11
:10435000099D002DE3D006CE23000198FFF726FF2C
:104360000028DCD002AB1E8C019BBF88DE80009B46
:104370005988074B994207D020002C30FDF75CFF8D
:10438000009BC7805E80CBE7009B1F80FAE7C0469A
:10439000FFFF000013B5019200910A1E10D00179B1
:1043A00000290AD120220271213A02804280019A1A
:1043B0000099FFF755FF020002E000222029F6D005
:1043C000100016BD036802001800383010B5002830
:1043D00003D051689268FFF7DDFF10BD70B50D0086
:1043E00004000800FFF7EEFF2B68206063602000E8
:1043F00070BD37B50D0001006846FFF7EFFF0020E4
:10440000009C844207D020000199FDF7C8FF0623D5
:104410000120237125703EBD30B589B00D00040028
:10442000010003A8FFF7DAFF002005AB187204981B
:104430002968AA680090079B039805910692FFF7E8
:10444000E1FC2368181E02D001201B79584009B0F6
:1044500030BD37B50D0001006846FFF7BFFF0020F3
:10446000009C844207D020000199FDF798FF0C239F
:104470000120237125603EBD37B50D00010068465F
:10448000FFF7ACFF0020009C844207D02000019978
:10449000FDF785FF0A230120237125603EBD000042
:1044A00070B500258AB02B4C2B482100401908F02C
:1044B00086FD2A482100401908F081FD2848210086
:1044C000401908F07CFD27482100401908F077FDCD
:1044D00025482100401908F072FD244821004019A8
:1044E0000C3508F06CFD782DDDD10025204B210026
:1044F0001D70204B20481D7008F061FD1F492048A9
:1045000008F05DFDC8221F4E1F4B30003C361A805C
:10451000FFF75DFC357007AE30001C49FDF7B0FEBB
:1045200029003000FFF795FF04A81949FDF7A8FE00
:1045300004A902A8FFF752FF01233372039B7560A1
:10454000009321002A00B36802980794FFF75AFCF1
:104550000AB070BD1D3801009C0A0020240A00200A
:10456000AC090020140B0020C40500203C060020EC
:10457000A8090020C10500202807002023380100D9
:1045800074020020CC06002022000020302D010003
:104590003C2D0100F0B504008DB0FFF781FF03232F
:1045A0000022210009A808F099FEC84D09A8290099
:1045B00008F0ECFD060009A808F01BFC002E03D053
:1045C0002900C34808F0DBFC03230022210009A8CE
:1045D00008F084FEBF4D09A8290008F0D7FD0600A9
:1045E00009A808F006FC002E03D02900B84808F0FE
:1045F000C6FCB94909A808F04BFC042209A920000F
:1046000008F030FE04220300210003A808F066FE33
:1046100009A808F0EEFB002503270C26AF4C09A8DB
:10462000210008F035FC012209A903A808F01AFEB0
:1046300000220092431C04D0EB0FAF425341DBB287
:10464000009309A808F0D5FB009B002B35D0210072
:1046500006A808F01DFC012206A903A808F002FE26
:104660000122030003A909A808F038FE33006B43B8
:104670009B4809A9C01808F09CFC09A808F0B9FBE0
:1046800006A808F0B6FB210006A808F001FC0122EC
:1046900006A903A808F0E6FD03A9020009A8FDF792
:1046A00005FE09A903A808F084FC09A808F0A1FBED
:1046B00006A808F09EFB0135B0E78A4D09A829003D
:1046C00008F0E6FB09A903A808F0DCFD060009A82C
:1046D00008F08FFB731C2ED0290006A808F0D8FB29
:1046E00006A903A808F0CEFD0122030003A909A82A
:1046F00008F0F4FD7A4809A9303008F05AFC09A8FE
:1047000008F077FB06A808F074FB290006A808F05B
:10471000BFFB06A903A808F0B5FD03A9020009A87C
:10472000FDF7C4FD09A903A808F043FC09A808F097
:1047300060FB06A81BE0210009A808F0A9FB0122E4
:1047400009A903A808F08EFD060009A808F051FB8E
:10475000634D731C00D09CE0012203A909A8FDF75A
:10476000A5FD280009A9303008F023FC09A808F0AD
:1047700040FB5B480027303008F080FE5A4D09A806
:10478000290008F085FB09A903A808F07BFD0400B7
:1047900009A808F02EFB631C00D1AFE00C2629000D
:1047A00006A8524C08F074FB06A903A808F06AFD9D
:1047B0007E4303000122A41903A909A808F08EFD75
:1047C00009A9200008F0F5FB09A808F012FB06A8CB
:1047D00008F00FFB200008F051FE290006A808F0A1
:1047E00057FB06A903A808F04DFD03A9421C09A820
:1047F000FDF75CFD09A903A808F0DBFB09A808F098
:10480000F8FA06A808F0F5FA394D09A8290008F0C9
:104810003FFB09A903A808F035FD019009A808F09D
:10482000E8FA344C019BA419013344D0290006A8AE
:1048300008F02EFB06A903A808F024FD00220300BF
:1048400003A909A808F04AFD09A9200008F0B1FB56
:1048500009A808F0CEFA06A808F0CBFA290006A8A5
:1048600008F016FB06A903A808F00CFD03A9020036
:1048700009A8FDF71BFD09A903A808F09AFB09A8E0
:1048800008F0B7FA06A808F0B4FA1B4B01371F70FE
:1048900074E7210006A808F0FBFA06A903A808F0AF
:1048A000F1FC03A90300012209A808F017FD280064
:1048B00009A9303038E7002203A909A8FDF7F6FC62
:1048C00009A9200008F075FB09A8DCE7F404002022
:1048D0002807002000050020612C0100923401000F
:1048E0009C0A0020AC34010094340100AC09002083
:1048F00096340100140B0020A80900203F4909A8A4
:1049000008F04DFB0A233E4A3B2109A8FFF770F847
:1049100009A808F06EFA3B4906A808F0B9FA06A9FA
:1049200009A8FFF7B3F9384C09A9200008F041FBAA
:1049300009A808F05EFA06A808F05BFA334E2000DA
:10494000310008F031FC002803D03149200008F084
:1049500036FB304C3049200008F018FC002825D0E8
:1049600020002E490C3008F011FC00281BD020003C
:104970002B49183008F00AFC002814D024342449AC
:10498000200008F011FC002807D00123009303A8A1
:1049900008F02FFA00980DB0F0BD2249200008F071
:1049A00003FC0028F1D1FFF767F8F0E71E4920006B
:1049B00008F0ECFB00280BD00C343100200008F08C
:1049C000F3FB0028E1D12000144908F0DFFBE8E701
:1049D000164D2000290008F0D9FB002803D0200044
:1049E0000E490C30F1E73100200008F0DDFB002813
:1049F000D9D0200029003030E7E7C046140B002052
:104A0000240A0020AE340100740200201D38010089
:104A1000233801009C0A0020540500206C0500206A
:104A200048050020832D0100780500206005002046
:104A30007FB50E002D490400150008F016F92C4B27
:104A40001B88C82B2FD12B49200008F033F92A49A5
:104A500001A808F01DFA290001A808F054FB010084
:104A6000200008F031F901A808F0C3F9200008F08F
:104A700019F9012008F0D0FD2049280008F086FB34
:104A8000002803D01E49200008F0FAF83100200069
:104A900008F01AF9200008F005F9200004F0C8FA1F
:104AA000FFF7FEFC7FBD1749C92B1BD01649CC2B45
:104AB00018D0C82215495200934213D0CA22144973
:104AC000520093420ED0CF2212495200934209D095
:104AD000A022FF321049934204D0FA22520093429E
:104AE000C4D10E49200008F0E5F8BFE7422C0100D0
:104AF000220000204C2C0100532C01003C0500201A
:104B0000EC2C0100632C01006F2C01007E2C0100B5
:104B10008E2C01009C2C0100B52C0100D22C010030
:104B2000C82270B5124C134B8CB052000600200006
:104B30001A800D00FFF74BF900233C34237031003D
:104B400006A8FEF787FF2900684608F028FA0A49F8
:104B500003A808F024FA03AA694606A8FFF768FF2D
:104B600003A808F046F9684608F043F90CB070BD98
:104B7000CC060020220000209005002070B5050022
:104B800008000E00FFF71EFC3168041E06D0FDF77A
:104B900006FC40232371413B238063803368280057
:104BA0006B602C6070BD7FB506000C0015000028FE
:104BB00001D00CF0BBFB02960390002C09D0290019
:104BC0002000FDF7ECFB2B000299039A2000FFF771
:104BD000EDFA7FBD30B50D00040085B0010002A8DC
:104BE000FFF7FCFB2D68082202A968460BF017FEB0
:104BF00028000099019AFFF7D6FF2368181E02D0FB
:104C000001201B79584005B030BD0200406810B546
:104C1000002804D09368D1681269FFF7BBFB10BD70
:104C200037B504000D00FFF7F0FF0100A268286807
:104C300000910192FFF7B7FFA368181E02D0012070
:104C40001B7958403EBD0000F0B5060085B0083025
:104C5000FFF7B8FB051E02D1002005B0F0BD0379B7
:104C60007469B768002B20D140330371413B038046
:104C7000438038002B882C3019000193FDF7DCFAB3
:104C80006A46928802AB02909A80002810D0C388AE
:104C900002AAD380029800281DD0002C15D039001C
:104CA00002A8FDF74AFB013CF4E7402BE1D0D3E733
:104CB0000A4BEDE739002800FFF7B4F90028CCD003
:104CC000013C002CF6D10028C6D0B368B169F26966
:104CD000FFF760FBC1E70134F3E7C046FFFF0000C8
:104CE00037B504000D00FFF7AFFF0100A268286888
:104CF00000910192FFF757FFA368181E02D0012010
:104D00001B7958403EBD70B505000E00FFF79CFFB3
:104D100004000020A968844206D02000FDF73FFB74
:104D20000C2301202371266070BD10B50400FDF72F
:104D300022FBA36A1818A06210BD0000F8B50C0091
:104D4000160022210500FFF7F0FFA619A64209D0A0
:104D500021780F4B1F78002F12D05A788A4206D044
:104D60000233F7E728002221FFF7DFFFF8BD5C21BF
:104D70002800FFF7DAFF39002800FFF7D6FF05E02B
:104D80000029F9D103492800FFF7E1F90134DDE7F3
:104D90000F3801001E38010070B5060014001D1EFA
:104DA00007DA2D21FFF7C1FF22002B000025544216
:104DB0009D412B0030002200FFF7D5F970BD0000A7
:104DC000F0B51C008DB012AB1B7804905BB202935F
:104DD000100023002100170009F0A4F9002805D1D4
:104DE000BA490498FFF7B3F90DB0F0BD00220023D3
:104DF0003800210009F096F900280DD13A0023006F
:104E00003800210009F06AFE02000B003800210082
:104E100009F088F90028E3D100220023380021009E
:104E200009F086F9002806D02D210498FFF77DFFB0
:104E300080231B06E4180123029E05930933002EEC
:104E400004D0059A013E5A430592F8E70022A04B90
:104E50003800210009F08AF9002866D0802308254F
:104E60005B00019603939B4B290006A80693FFF76E
:104E700045F93A00230009F065F9002813D0964B54
:104E8000290006A80693FFF739F902000B00380045
:104E900021000AF049FD039A070094460C00019B8B
:104EA00063441BB20193039B5B100393013DDAD271
:104EB000002200233800210009F04EF900283AD0E2
:104EC000864A874B3800210009F03CF92E00002863
:104ED00031D06B1C2FD0804B310006A80693FFF712
:104EE0000DF900227F4B0AF01FFD3A00230009F064
:104EF00033F9002812D0774B310006A80693FFF74C
:104F0000FDF802000B00380021000AF00DFD07003B
:104F10000C00019B039A9B1A1BB20193039B013D5A
:104F20005B1003936DB2013ED3E780235B000393D4
:104F300008250196BCE73800210009F07BF905003F
:104F40000600092E0ED90A21059808F065FF029B7C
:104F50000590013B5BB230000A21029308F05CFF30
:104F60000600EEE728000BF025FB02000B003800DE
:104F700021000AF04BFF060005980F000BF01AFB0A
:104F800002000B00300039000AF0CEFC0F000600D2
:104F900009F050F904000BF00DFB02000B0030008B
:104FA00039000AF033FF0B00020009F097FD09F009
:104FB00041F9059B2418A3420BD80024019B01351D
:104FC000A34206D0092D04D91E000125013633B2B3
:104FD00001930A263100200008F0A4FF00290CD11B
:104FE000029B002B09DD2000310008F015FF029B19
:104FF0000400013B5BB20293ECE716260A2706ABDE
:10500000F6182800390008F08DFF013E303131706C
:105010002800390008F000FF051EF2D1162306AA69
:105020009B189A1B31000498FFF780F8029B002B15
:105030001DD00AAF1D003E00013D6DB2013F6B1C4B
:105040000BD020000A2108F06DFF303139702000AC
:105050000A2108F0E1FE0400EEE76B461B7A2E22DF
:10506000D94304988A554A427118FFF75FF8019BAB
:10507000002B00D1B8E665210498FFF756FE6B4679
:105080009C88019B002B05DA2D210498FFF74DFE2B
:105090006442A4B2162306AA9B181D000A2620000B
:1050A000310008F03FFF013D303129702000310010
:1050B00008F0B2FE84B2002CF1D1162306AA9B1888
:1050C0005A1B29000498FFF731F88DE606380100D5
:1050D000D0126341882B0100402B0100F168E38866
:1050E000B5F8E43E000024401023F0B50579060031
:1050F0002B400C0087B00188181E03D02C32100002
:10510000FDF79AF80C2D00D198E018D8042D00D1A5
:1051100086E007D8022D00D177E0032D00D186E08C
:105120004F4999E0062D00D191E000D27BE00A2D95
:10513000F6D1002332682000FFF715F81EE01C2D81
:1051400000D181E006D80E2D0ED01A2DE8D10268CC
:105150004368F0E7202D34D0402D12D01E2DDFD132
:1051600002684368092105E030680BF055FA0B002E
:105170000200062100912000FFF722FEA06A07B07E
:10518000F0BD5B212000FFF7D0FD3588354EB542DC
:1051900012D0E76A290038002C30FDF74DF80500E1
:1051A0003A002100FFF7A0FFED88B542EED02C2198
:1051B0002000FFF7BAFDE9E75D212000FFF7B5FD0C
:1051C000DCE77B212000FFF7B0FD35880126254B69
:1051D0009D4218D0E76A290038002C30FDF72CF8E2
:1051E00005003A002100FFF77FFFED881D4B9D422F
:1051F00006D02C21002E00D00E312000FFF795FDA7
:1052000001235E40E3E77D21D7E70022310003A8B8
:10521000FDF786F8049A03992000FFF78FFDADE7AC
:1052200001223168F3E73168CA880831F4E7316850
:105230002000CA880831FEF779FF9FE73268D3174C
:105240002000FFF7A9FD99E702684368F8E7337883
:105250000549002B00D105492000FEF778FF8DE7B6
:1052600006380100FFFF0000253801002A38010040
:10527000F0B54749B9B0060007F00AFE454808F006
:1052800033F9454905002CA8FCF7FAFF2CA968461C
:10529000FFF7A4F8009C002C09D001992000FDF72D
:1052A0007EF80C232371EB43DB171D4025603B493F
:1052B0002CA8FCF7E5FF3A4B2CA902A81D68FFF7C4
:1052C0008DF8029C002C06D003992000FDF767F8AA
:1052D0000A2325602371334C258E2768002D10D0BA
:1052E000314B3800ED18E36AED005D196A883B68C0
:1052F000D2009B6869689847002802D06B88686074
:105300002B802300E16A0C3399420BD0228E638EEE
:10531000934207D03B68D2009B6838009847238EA1
:10532000E06263860024300021000D94049607F0AB
:1053300046FE04A928220EA80BF071FA0EA9282215
:1053400018A80BF06CFA18A9282222A80BF067FA0B
:1053500022A928222CA80BF062FA22A83694FCF786
:10536000FBFF104C18A83794FCF7F6FF2000220032
:105370002CA93830FFF7B8FE2CA8FCF7EDFF0EA8DB
:10538000FCF7EAFF04A8FCF7E7FF300039B0F0BDF6
:105390001D38010074020020983401002E2C0100F9
:1053A00070020020CC060020FFFFFF1FF0B5C24AAC
:1053B000A5B01368C14901330500136007F0F4FE7E
:1053C00017ACBF4E00281FD0BE49BF4807F0DEFE15
:1053D00000281FD0BD490FA807F02BFE31001CA8E4
:1053E000FEF738FB0FA912A807F0D9FDB849200035
:1053F00007F01FFE1CA8220012A9FFF719FB2000CE
:1054000007F0F7FC00F077FCB249280007F0CCFE6B
:105410000028D9D1B04FB149380007F0B7FE0028B5
:1054200000D187E1AE49280007F0BEFE00282DD14B
:10543000AC49280007F0B8FE00284DD1AA49280041
:1054400007F0B2FE002800D0B0E031001CA8FEF743
:1054500001FBA6490FA807F0ECFD0FA912A807F061
:105460009EFD290012A807F04EFE0100200007F063
:1054700096FD1CA82100FFF753FB200007F0B9FCA4
:1054800012A807F0B6FC0FA800F0F3FC8D498E4877
:1054900007F07CFE0028CBD095491CA8FCF7F0FE55
:1054A0001CA90FA8FFF76AFB01231CA90FA81C93D6
:1054B000FEF7C9FD31001CA8FEF7CCFA12A8FFF7D1
:1054C000D7FE8C49200007F06AFD1CA8220012A913
:1054D000FFF7AEFA200064E07A497B4807F056FEF9
:1054E0000028ABD082491CA8FCF7CAFE0FA81CA953
:1054F000FFF744FB0F98109D041E0CD02900FEF707
:1055000091FD041E07D02900FCF749FF20232371D9
:10551000213B238063800A27774B17A91F93774B82
:105520001CA8209717931D941E95FFF779FB744BC9
:1055300017A91F93734B1CA8209717931D941E95B2
:10554000FFF76EFB704B1CA81F930C231D941E9538
:105550002093FFF75AFB1E99071E05D0FCF71FFF8B
:105560000C233B7100233B60684B17A91F93082352
:105570002093624B1CA81D941E951793FFF750FBB8
:1055800031001CA8FEF766FA12A8FFF771FE594910
:1055900017A807F004FD1CA817AA12A9FFF748FADC
:1055A00017A807F026FC12A800F063FC45494648FE
:1055B00007F0ECFD002800D147E74D491CA8FCF797
:1055C0005FFE1CA8FEF7FEFE1C99041E06D0FCF729
:1055D000E6FE20232371213B238063804C4B1C9EDD
:1055E0001F930A232093454B17A91CA817931D94BA
:1055F0001E96FFF715FB474B17A91F930C2320930B
:10560000454B1CA817931D941E96FFF709FB434BAF
:1056100043491F93132312A820931D941E9607F04D
:1056200037FC404F0FAD3900280007F002FD29007C
:1056300012A807F068FD3C4907F072FD390003909D
:1056400017A807F0F6FC17A9039807F05CFD374987
:1056500007F066FD07001CA8FFF7D7FA3968BA689B
:10566000002784460CAB1E981F720E9B009060466C
:105670000C910D92FEF7C6FB17A807F0BAFB2800A5
:1056800007F0B7FB12A807F0B4FB294B1CA81F9327
:1056900008231D9420931E96FFF7B7FA01232B725F
:1056A0001E9B0C496F6000933A00AB680F91FEF7A8
:1056B000A9FB034965E7C04670020020AD2F010039
:1056C0009C050020F404002028070020B32F0100CF
:1056D000313001001D3801009C0A002078050020AF
:1056E0003B30010047300100B73201005F3001005C
:1056F00059300100840500206F3001007A3001002C
:10570000853001009030010097300100A430010085
:10571000AD300100B8300100C5300100D1300100CA
:10572000812D0100612C0100E5300100F130010004
:10573000FA300100CA49280007F036FD002800D0E1
:1057400018E1C849280007F02FFD002800D02CE1FF
:10575000C549280007F028FD002800D03BE1C349D7
:10576000280007F021FD002800D04AE1C0492800A8
:1057700007F01AFD002800D04FE1BD49280007F0CE
:1057800013FD002800D0CBE1BA49280007F00CFD3A
:10579000002800D014E2B849280007F005FD0028D1
:1057A00000D01AE2B549280007F0FEFC002800D01E
:1057B00060E2B349280007F0F7FC002800D062E25D
:1057C000B049280007F0F0FC002800D068E2AE499C
:1057D000280007F0E9FC002800D08EE2AB49280041
:1057E00007F0E2FC002800D094E23800A849183005
:1057F00007F0CCFC002800D127E63800A54924306A
:1058000007F0D2FC002800D11FE6A349280007F0CA
:10581000CBFC002800D098E2A049280007F0C4FC87
:10582000002800D0A2E29E49280007F0BDFC002815
:1058300000D063E39B49280007F0B6FC002800D0A5
:105840006AE39949280007F0AFFC002800D095E3EF
:105850009649280007F0A8FC002800D0BDE3944931
:10586000280007F0A1FC002801D000F00BFC9149B2
:10587000280007F099FC002801D000F037FD8E4980
:10588000280007F091FC002801D000F06AFD8B4948
:10589000280007F089FC002801D000F0E9FD8849C4
:1058A000280007F081FC874F002801D000F06CFE33
:1058B0008549280007F078FC002801D000F0EDFEB3
:1058C0008249280007F070FC002801D000F02FFF6B
:1058D0007F49280007F068FC002801D000F07EFF17
:1058E0007C49280007F060FC002801D001F09CF8FA
:1058F0007949280007F058FC002801D001F0BDF9D3
:105900007649280007F050FC002801D001F0E2F9A8
:105910007349280007F048FC002801D001F0F8F98D
:105920007049280007F040FC002801D001F02FFA50
:105930006D49280007F038FC002801D001F061FA19
:1059400039001CA8FEF786F868490FA807F071FB1C
:105950000FA912A807F023FB290012A807F0D3FB18
:10596000010017A807F01BFB1CA817A9FFF7D8F820
:1059700017A883E55E495F4807F008FC002800D1BE
:10598000DFE65D491CA8FCF77BFC5C4B1CA8198872
:10599000FEF772FD5A491CA8FCF772FC594B210016
:1059A0001CA81793FFF716F984E55149514807F0F1
:1059B000EDFB002800D1CBE64F491CA8FCF760FCAA
:1059C0004E4B1CA81988FEF757FD4D491CA8FCF743
:1059D00057FC4D4BE3E74649464807F0D7FB002804
:1059E00000D1BCE644491CA8FCF74AFC434B1CA868
:1059F0001988FEF741FD42491CA8FCF741FC434BC6
:105A0000CDE73B493B4807F0C1FB002800D1ADE69C
:105A10003F49404807F0FCFA4CE53F49354807F05C
:105A2000B5FB002800D1A8E639491CA807F001FB06
:105A30001CA9384807F0AAFB05001CA807F0D9F9F3
:105A400036491CA8002D06D0FCF71AFC01211CA821
:105A5000FEF7CFFC2EE5FCF713FC2900F7E7C04664
:105A600003310100103101001C310100A631010099
:105A70005D31010082310100B7320100A331010024
:105A8000AE310100C53101002E340100F4310100B6
:105A900048050020233801000D3201001E320100AC
:105AA000253201002F320100723201007B320100E9
:105AB000A2320100AE320100C632010024330100DF
:105AC000593301009C050020683301007733010041
:105AD00086330100903301009F330100E43301005D
:105AE000053401000E340100333401005F30010041
:105AF0000005002028070020302D01000C000020A8
:105B00003C2D01002A3101004431010067310100C0
:105B10002538010064020020F404002059300100FF
:105B2000DD49DE4807F032FB002800D12CE6DC49D5
:105B30001CA807F07EFA1CA90FA8FEF7CFF81CA836
:105B400007F057F90FA807F099FCD649200007F095
:105B500070FA21000FA807F019FB051E0BD1D249DE
:105B60001CA807F066FA1CA90FA807F00FFB050098
:105B70001CA807F03EF9200007F03BF9002D0FD0DC
:105B80000FA9CA4807F0FBF931001CA8FDF762FF16
:105B900012A8FFF76DFBC649200007F000FA29E4C0
:105BA00031001CA8FDF756FFC249200007F041FA5A
:105BB0001CA82100FEF7B4FF200007F01AF962E4E8
:105BC000BD49B64807F0E2FA002800D1E3E5BB4939
:105BD0001CA8FCF755FB002139E7B749AF4807F08F
:105BE000D5FA002800D1DDE5B4490CA8FCF748FB44
:105BF000B3490FA807F04CF90FA917A807F0CFF980
:105C0000B04917A807F09AFA0400AF491CA807F09A
:105C10003FF91CA9200007F076FA0CA9040004A89B
:105C2000FEF7DCFB002012ABA26821681872059811
:105C3000149B0090049813921291FEF7E3F81CA8AD
:105C400007F0D7F817A807F0D4F80FA807F0D1F895
:105C50009E491CA8FDF7FEFE0FA8FFF709FB94491B
:105C600017A807F09CF917AA0FA91CA8FEF7E0FED9
:105C700017A8A2E78849894807F088FA002800D1C8
:105C800097E58949C5E68C49844807F07FFA0028E2
:105C900000D195E589491CA8FCF7F2FA8C4B7EE609
:105CA00085497E4807F072FA002800D18FE58349C4
:105CB0001CA8FCF7E5FA1CA906A8FEF78FFB012338
:105CC00003222372079B62607F490093A3680698B2
:105CD0001791FEF797F831001CA8FDF7BBFE0FA83F
:105CE000FFF7C6FA724912A807F059F912AA0FA9CC
:105CF0001CA8FEF79DFE12A85FE76F49674807F0F2
:105D000045FA002800D169E56C491CA8FCF7B8FAEF
:105D1000704B44E66849614807F038FA002800D122
:105D200063E566491CA8FCF7ABFA0FA81CA9FEF7AF
:105D300025FF0F98002802D01099FCF767FB6649F1
:105D40000FA8FEF7A5F9FFF7B5FB5B49534807F02D
:105D50001DFA002800D15FE558491CA8FCF790FA0D
:105D600003211CA8FEF775FBFFF7A4FB4A494B482B
:105D700007F00CFA002800D155E558491CA807F097
:105D800058F91CA909A8FDF7A9FF1CA807F031F8CC
:105D900053491CA807F04DF91CA90CA8FDF79EFF5C
:105DA0001CA807F026F84F4917A807F071F84E49CC
:105DB0001CA807F06DF81CAA17A90CA807F0ACFAEC
:105DC0001CA807F016F817A807F013F847490FA802
:105DD00007F05EF809A807F051FB3F4909A807F052
:105DE000E3F9002849D0424912A807F051F80CA95C
:105DF00012A807F088F93F4907F092F9010017A8A7
:105E000007F0CDF8012217A91CA8FDF737F81CA947
:105E10000FA807F0CEF81CA806F0EBFF17A806F0B5
:105E2000E8FF12A806F0E5FF24491CA8FCF728FAB1
:105E30000FA91CA8FEF7F0FA31001CA8FDF70AFE16
:105E400012A8FFF715FA1A4917A807F0A8F817AA19
:105E500012A91CA8FEF7ECFD17A806F0CAFF12A8AD
:105E600006F0C7FF0FA806F0C4FF0CA806F0C1FF9C
:105E700009A806F0BEFF25B0F0BD31001CA8FDF753
:105E8000E9FD1D4917A807F0D4F81CA817A9FEF7CB
:105E900047FE17A8E4E7C0460005002028070020B9
:105EA0008D310100253801002A38010064020020EC
:105EB0008405002097310100F404002059300100CE
:105EC000912D0100B9310100812D01009C050020B8
:105ED000D33101007A30010005320100383201006F
:105EE0003F3201004A320100533201001D380100E7
:105EF0004E320100732E01005532010056495748B9
:105F000007F044F9002800D194E455491CA8FCF797
:105F1000B7F9544B196824E74F49504807F036F950
:105F2000002800D18DE450491CA807F082F81CA974
:105F30000FA8FDF7ABFE1CA806F05BFF0FA91CA87D
:105F400007F02DF81CA8FDF7F1FE05001CA806F0CF
:105F500050FF002D00D154E20FA807F0C5FA002829
:105F600065DB404B1B68834261DD3D491CA8FCF7A3
:105F700087F900211CA8FEF73CFA05E636493748A8
:105F800007F004F9002800D162E437491CA807F0A3
:105F900050F81CA90FA8FDF779FE1CA806F029FFF0
:105FA0000FA91CA806F0FBFF1CA8FDF7BFFE05000B
:105FB0001CA806F01EFF002D00D122E20FA807F05A
:105FC00093FA002833DB274B1B6883422FDD2449DB
:105FD0001CA8FCF755F90121CCE724491F4807F01C
:105FE000D5F8002800D13AE421491CA807F021F88F
:105FF0001CA90FA8FDF772FE1CA806F0FAFE0FA957
:106000001CA806F0CCFF1CA8FDF790FE05001CA8FC
:1060100006F0EFFE002D00D1F3E10FA807F064FABF
:10602000002804DB0F4B1B68834200DDACE51149FF
:106030001CA8FCF725F9104B1CA81988FEF71CFAC0
:106040000E491CA8FCF71CF90D4B210017931CA846
:10605000FEF7C0FD98E5C046F404002028070020A4
:106060005930010010000020BF340100000500205D
:10607000C3320100302D01000A0000203C2D010038
:1060800087320100E249E34807F080F8002801D197
:10609000FFF7EDFBE04B0CA8197806F018FF0CA8F1
:1060A00007F022FADD4C050021000FA8FCF7E8F804
:1060B00000220FA912A8FDF70EFF12A917A8FEF7DC
:1060C00029F817A91DA8FEF725F8D54B17A9229383
:1060D00004232393D34B1CA81793FEF701FE210042
:1060E0000FA8FCF7CDF800220FA912A8FDF7F3FEC8
:1060F00012A917A8FEF70EF817A91DA8FEF70AF8AF
:1061000005232393C84B1CA822941F78FEF79CFDFF
:106110001E99061E04D0FCF742F90A23376033713A
:10612000042621000FA8FCF7ABF801220FA912A842
:10613000FDF7D1FE12A917A8FDF7ECFF17A91DA8BE
:10614000FDF7E8FFB94BB64F17A91CA81793229784
:106150002396FEF7C5FD21000FA8FCF791F8012258
:106160000FA912A8FDF7B7FE12A917A8FDF7D2FFD5
:1061700017A91DA8FDF7CEFF0523691E23931CA8B0
:106180004B4259412294FEF7BEFD21000FA8FCF7B7
:1061900077F802220FA912A8FDF79DFE12A917A8F1
:1061A000FDF7B8FF17A91DA8FDF7B4FFA04B17A96D
:1061B0001CA8179322972396FEF792FD21000FA8A3
:1061C000FCF75EF802220FA912A8FDF784FE12A9BF
:1061D00017A8FDF79FFF17A91DA8FDF79BFF052333
:1061E000A91E23931CA84B4259412294FEF78BFD14
:1061F00021000FA8FCF744F803220FA912A8FDF70D
:106200006AFE12A917A8FDF785FF17A91DA8FDF7BB
:1062100081FF884B17A91CA8179322972396FEF796
:106220005FFD21000FA8FCF72BF803220FA912A88D
:10623000FDF751FE12A917A8FDF76CFF17A91DA8BD
:10624000FDF768FF0523E91E23931CA84B42594123
:106250002294FEF758FD21000FA8FCF711F8320038
:106260000FA912A8FDF737FE12A917A8FDF752FFD4
:1062700017A91DA8FDF74EFF6F4B17A91CA8179370
:1062800022972396FEF72CFD21000FA8FBF7F8FFBD
:1062900032000FA912A8FDF71EFE12A917A8FDF7DC
:1062A00039FF17A91DA8FDF735FF0523043D6942F5
:1062B00069411CA823932294FEF725FD5F491CA881
:1062C000FDF7C8FB12A8FEF7D3FF5D4917A806F03B
:1062D00066FE17AA12A91CA8FEF7AAFB17A806F0CB
:1062E00088FD12A806F085FD0CA8C2E5484949487A
:1062F00006F04CFF002801D1FFF7C1FA51491CA854
:1063000006F097FE1CA90FA8FDF7C0FC1CA806F01C
:1063100070FD0FA91CA806F042FE1CA8FDF706FDA3
:1063200005001CA806F065FD002D6AD00FA807F037
:10633000DBF8002805D139491CA8FBF7A1FF424B27
:1063400083E6012805D135491CA8FBF799FF3F4B8F
:106350007BE6022836D131491CA8FBF791FF3C4B64
:1063600073E62B492B4806F011FF002801D1FFF7F7
:106370008EFA34491CA806F05CFE1CA90FA8FDF794
:1063800085FC1CA806F035FD0FA91CA806F007FE29
:106390001CA8FDF7CBFC05001CA806F02AFD002D6B
:1063A0002FD00FA807F0A0F80028C4D00128CAD029
:1063B000022807D119491CA8FBF762FF244B179349
:1063C00017A944E6032805D114491CA8FBF758FF78
:1063D000204BF4E7042805D110491CA8FBF750FF17
:1063E0001D4BECE71D491CA8FBF74AFF1C4B1CA8E2
:1063F0001988FEF741F81B491CA8FBF741FF1A4B0F
:10640000DDE731001CA8FDF725FB1849FFF7CDFBA0
:10641000F4040020280700209002002059300100D9
:1064200075300100D43201002C000020E43201005C
:10643000F432010004330100143301009C050020F4
:1064400084050020BF3401002E33010045330100D4
:106450004A3301004F33010054330100302D010055
:106460000A0000203C2D0100873201005532010056
:10647000CE49CF4806F08AFE002801D1FFF70FFA77
:10648000CC491CA806F0D5FD1CA90CA8FDF7FEFB05
:106490001CA806F0AEFC0CA91CA806F080FD1CA8E8
:1064A000FDF744FC05001CA806F0A3FC002D00D15C
:1064B000E5E00CA807F018F8BF4B070019780FA803
:1064C00006F005FD0FA807F00FF80500002F24D1F6
:1064D000BA491CA8FBF7D4FE0121B94B1B7899429D
:1064E000894149421CA8FDF784FF31001CA8FDF733
:1064F000B1FA12A8FEF7BCFEB249200006F04FFD2B
:106500001CA8220012A9FEF793FA200006F071FCE5
:1065100012A806F06EFC0FA8E4E6012F08D1A749E7
:106520001CA8FBF7ADFE013D69426941C9B2D9E73C
:10653000022F05D1A1491CA8FBF7A2FE023DF3E7FB
:10654000032F05D19D491CA8FBF79AFE033DEBE7FD
:10655000042F05D199491CA8FBF792FE043DE3E7FF
:106560001CA89949FBF78CFE984B1CA81988FDF7CD
:1065700083FF1CA89649FBF783FE964B17A91CA81E
:106580001793FEF727FBB0E78849894806F0FEFD20
:10659000002801D1FFF78CF986491CA806F049FDB7
:1065A0001CA90CA8FDF772FB1CA806F022FC0CA984
:1065B0001CA806F0F4FC1CA8FDF7B8FB05001CA8FD
:1065C00006F017FC002D5AD00CA806F08DFF7A4B70
:1065D000040019780FA806F07AFC0FA806F084FFD3
:1065E000002C25D175491CA8FBF74AFE744B1CA949
:1065F00009A81D78FDF7F2FE099C0A99002C05D028
:106600002000FBF7CCFE0A232560237139001CA86B
:10661000FDF720FA12A8FEF72BFE6A4917A806F02C
:10662000BEFC1CA817AA12A9FEF702FA17A86DE76C
:10663000631E032B0FD86149844207D11CA8FBF7C6
:106640001FFE01211CA8FDF704FFDFE71CA8FBF7D4
:1066500017FE0021F6E71CA85B49FBF711FE5B4B18
:106660001CA81988FDF708FF1CA85949FBF708FE6C
:10667000584B17A91CA81793FEF7ACFAC6E73100D0
:106680001CA8FDF7E7F95449200006F0D2FC1CA82D
:106690002100FEF745FA200024E64449444806F06C
:1066A00075FD002801D1FFF70BF942491CA806F03F
:1066B000C0FC1CA90FA8FDF7E9FA1CA806F099FB7D
:1066C0000FA91CA806F06BFC1CA8FDF72FFB04000B
:1066D0001CA806F08EFB002C00D1A3E30FA806F047
:1066E00003FF002805D135491CA8FBF7C9FD01218E
:1066F00007E00138032849D830491CA8FBF7C0FD42
:1067000000211CA8FDF7A5FE39001CA8FDF7A2F981
:1067100012A8FEF7ADFD2B4917A806F040FC1CA8F7
:1067200017AA12A9FEF784F917A8FEF769FE1F49F8
:106730001F4806F02BFD002801D1FFF7C9F81D49BD
:106740001CA806F076FC1CA90FA8FDF79FFA1CA850
:1067500006F04FFB0FA91CA806F021FC1CA8FDF7B2
:10676000E5FA04001CA806F044FB002C00D159E314
:106770000FA806F0B9FE002805D110491CA8FBF7A8
:106780007FFD0421BDE701380328ACD90E491CA8C0
:10679000FBF776FD0D4B1CA81988FDF76DFE0C4923
:1067A0001CA8FBF76DFD0B4BEBE2C046F404002088
:1067B00028070020BF34010090020020593001005A
:1067C0002C00002084050020302D01000A0000204C
:1067D0003C2D01008732010055320100D949DA48C9
:1067E00006F0D4FC002801D1FFF77AF8D7491CA89D
:1067F00006F01FFC1CA906A8FDF770FA1CA806F0FD
:10680000F8FAD3491CA806F014FC1CA909A8FDF746
:1068100065FA1CA806F0EDFACE4D0CA8290006F08A
:1068200037FB06A91CA806F0BAFB1CA8FDF77EFAE8
:1068300004001CA806F0DDFA002C00D10FE206A827
:1068400006F052FE041E31D1C34909A806F0ACFC83
:106850000400601E84410134C04912A806F018FBF0
:106860000A2221000FA806F051FB0FA912A806F07A
:106870004AFCBB4906F054FC010017A806F08FFB48
:10688000012217A91CA8FCF7F9FA1CA90CA806F00C
:1068900090FB1CA806F0ADFA17A806F0AAFA0FA8FC
:1068A00006F0A7FA12A806F0A4FA1BE0012838D1D6
:1068B000AC4917A806F0ECFA220017A91CA8FCF7AF
:1068C000DDFA1CA90CA806F074FB1CA806F091FACE
:1068D00017A806F08EFAA04909A806F065FCA2499F
:1068E00000283AD139001CA8FDF7B4F812A8FEF729
:1068F000BFFC9E4917A806F052FB17AA12A91CA8B4
:10690000FEF796F817A806F074FA12A806F071FAC6
:106910000CA806F06EFA09A806F06BFA06A8FFF7B5
:10692000A8FA022843D18F4917A806F0B1FA01222C
:1069300017A91CA8FCF7A2FA1CA90CA806F039FBA1
:106940001CA806F056FA17A806F053FA824909A8BF
:1069500006F02AFC86490028C4D017A806F098FA49
:10696000012217A91CA8FCF789FA1CA90CA806F09B
:1069700020FB1CA806F03DFA17A806F03AFA2900F9
:106980000CA8FBF78BFC0028ACD01CA87949FBF7BE
:1069900077FC794B1CA81988FDF76EFD1CA8774978
:1069A000FBF76EFC0CA91CA8FDF736FD9AE703283F
:1069B0001BD16C4917A806F06BFA012217A91CA875
:1069C000FCF75CFA1CA90CA806F0F3FA1CA806F068
:1069D00010FA17A806F00DFA5F4909A806F0E4FBC3
:1069E0006749002800D17DE7B7E7042800D027E1F8
:1069F0005C4917A806F04CFA012217A91CA8FCF75D
:106A00003DFA1CA90CA806F0D4FA1CA806F0F1F96E
:106A100017A806F0EEF9504909A806F0C5FB0028B2
:106A200000D15FE7574998E74649474806F0AEFB73
:106A3000002801D1FEF75CFF44491CA806F0F9FAD2
:106A40001CA906A8FDF74AF91CA806F0D2F94E4980
:106A50001CA806F0EEFA1CA909A8FDF73FF91CA82E
:106A600006F0C7F93B490CA806F012FA06A917A8C8
:106A700006F095FA17A8FDF759F9041E0AD009A9DE
:106A80001CA806F08CFA1CA8FDF750F904001CA8FD
:106A900006F0AFF917A806F0ACF9002C00D1DEE043
:106AA00006A806F021FD050009A806F01DFD04005A
:106AB000002D17D1431E032B00D8CDE62D491CA86D
:106AC000FBF7DEFB314B1CA81988FDF7D5FC2B49E1
:106AD0001CA8FBF7D5FB2E4B17A91CA81793FEF794
:106AE00079F8FFE6012D55D10128E7D81D4917A8EF
:106AF00006F0CEF92A0017A91CA8FCF7BFF91CA9BB
:106B00000CA806F056FA1CA806F073F917A806F0B0
:106B100070F91549012C00D0E4E617A806F0B8F981
:106B2000220017A91CA8FCF7A9F91CA90CA806F0BB
:106B300040FA1CA806F05DF917A806F05AF90549B5
:106B40001EE7C0460005002028070020C3320100D0
:106B5000AA3301001D380100B0330100B533010034
:106B6000732E0100BC330100C433010084050020F2
:106B7000CC330100302D0100080000203C2D010025
:106B8000D4330100DC330100593001000A00002039
:106B9000F2330100022D19D101288FD8A84917A876
:106BA00006F076F9012217A91CA8FCF767F91CA9C1
:106BB0000CA806F0FEF91CA806F01BF917A806F0B1
:106BC00018F9A049012C00D08CE6A6E7032D1AD1B4
:106BD000012800D972E79A4917A806F059F901224D
:106BE00017A91CA8FCF74AF91CA90CA806F0E1F9A2
:106BF0001CA806F0FEF817A806F0FBF89249012C35
:106C000000D06FE689E7042D1AD1012800D955E795
:106C10008B4917A806F03CF9012217A91CA8FCF71C
:106C20002DF91CA90CA806F0C4F91CA806F0E1F87F
:106C300017A806F0DEF8012C00D053E683496CE774
:106C400083491CA8FBF71CFB824B1CA81988FDF785
:106C500013FC81491CA8FBF713FB804B3CE7390070
:106C60001CA8FCF7F7FE7E4917A806F0E2F91CA85D
:106C700017A9FDF755FF17A848E67A497A4806F0A4
:106C800085FA002801D1FEF73BFE78491CA806F0E2
:106C9000D0F91CA90FA8FCF7F9FF1CA806F0A9F869
:106CA0000FA91CA806F07BF91CA8FDF73FF804000B
:106CB0001CA806F09EF8002C00D1B3E00FA806F047
:106CC00013FC002800DA61E5694B1B68834200DC95
:106CD0005CE508E56749644806F058FA002801D1E8
:106CE000FEF716FE5A491CA8FBF7CAFA624B1CA80D
:106CF0001988FDF7C1FB58491CA8FBF7C1FA5F4B87
:106D000017A91CA81793FDF765FF3900FEF739FC9A
:106D10005849554806F03AFA002801D1FEF700FE1E
:106D200057491CA806F085F91CA90FA8FCF7D6FF47
:106D30001CA806F05EF80FA91CA806F030F91CA8E4
:106D4000FCF7F4FF04001CA806F053F8002C69D0EF
:106D50000FA806F0C9FB3E49002800DA17E5444BAE
:106D60001B68834200DC12E51CA8FBF789FA424B42
:106D70001CA81988FDF780FB37491CA8FBF780FA8F
:106D8000404B17A91CA81793FDF724FFBCE4394911
:106D9000354806F0FBF9002801D1FEF7C9FD384956
:106DA0001CA806F046F91CA90FA8FCF797FF1CA821
:106DB00006F01FF80FA91CA806F0F1F81CA8FCF7B4
:106DC000B5FF04001CA806F014F8002C2AD00FA868
:106DD00006F08AFB1E49002800DAD8E4244B1B6821
:106DE000834200DCD3E41CA8FBF74AFA224B1CA820
:106DF0001988FDF741FB18491CA8FBF741FA224B03
:106E0000BFE71849184806F0C1F9002801D1FEF77C
:106E100097FD16491CA806F00CF91CA90FA8FCF751
:106E200035FFC4E739001CA8FCF714FE0C4917A86D
:106E300006F0FFF817A91CA8FDF772FEFEF718FF71
:106E4000BC330100CC330100D4330100DC3301003A
:106E5000302D01000A0000203C2D01008732010086
:106E600055320100F404002028070020BF3401003F
:106E700010000020000500200C0000201C34010040
:106E8000C3320100473401006A340100F8B500251F
:106E9000944A9549954803F07BFA954C9548964B52
:106EA0002200964943600570856006F0A3FF902399
:106EB0000121934A9B0049429248D15001F0DAF8EF
:106EC000914801F0D7F8914801F0D4F8502190484A
:106ED00002F00EF98F4802F081F88F4802F094FA20
:106EE0008E4E8F48310040190C3505F0D1FF782DBA
:106EF000F6D122008B49002006F07CFF00258A484D
:106F0000310040190C3505F0C3FF782DF7D1220070
:106F10008649002006F06EFF0025854831004019A3
:106F20000C3505F0B5FF782DF7D1220081490020FE
:106F300006F060FF00258048310040190C3505F04F
:106F4000A7FF782DF7D122007C49002006F052FFE0
:106F500000257B48310040190C3505F099FF782D4C
:106F6000F7D122007749002006F044FF002576483B
:106F7000310040190C3505F08BFF782DF7D1220038
:106F80007249002006F036FF714F3100380005F0DD
:106F90007FFF704D22002900380006F02BFF6E4F56
:106FA0003100380005F074FF29002200380006F097
:106FB00021FF6A486A4B02000C32C2628022D20270
:106FC0000263010001220360002352423C310B7036
:106FD000037183608286C2876249220006F00AFF3D
:106FE000614F6249380005F053FF22002900380044
:106FF00006F000FF5E4F5F49380005F049FF2200B0
:107000002900380006F0F6FE5B4F5C49380005F0B9
:107010003FFF22002900380006F0ECFE584F3100F7
:10702000380005F035FF22002900380006F0E2FEA6
:10703000544E5549300005F02BFF22002900300046
:1070400006F0D8FE514E5249300005F021FF2200D3
:107050002900300006F0CEFE4E4E4F49300005F0BC
:1070600017FF22002900300006F0C4FE4B4E4C49A9
:10707000300005F00DFF22002900300006F0BAFEB6
:10708000484E4949300005F003FF22002900300036
:1070900006F0B0FE454E4649300005F0F9FE2200EC
:1070A0002900300006F0A6FE424E4349300005F0AC
:1070B000EFFE22002900300006F09CFE3F4E4049C2
:1070C000300005F0E5FE22002900300006F092FEB7
:1070D0003C4C0821200001F003FC21003A4801F05B
:1070E0001DF9F8BD020200000035010084090020EE
:1070F00000000020D8040020002C004203210000E2
:107100009402002034070020370700203A070020AF
:107110008C0B00209C050020B40600201D380100C7
:107120009C0A002091210000140B00207521000012
:10713000AC09002059210000240A00203D21000054
:10714000C4050020212100003C060020052100008C
:1071500028070020F3CD000074020020CC06002098
:1071600004000020EB3D0000F4040020D02B0100BF
:1071700000050020D42B0100640200202A38010001
:10718000B405002048050020813401006C05002072
:10719000D82B010054050020DB2B010060050020E6
:1071A000AD2F010078050020DF2B010084050020B1
:1071B000EA2B01003C050020FB2B0100900500207C
:1071C0000D2C01004007002058070020F0B5C84CE6
:1071D000A544C84C200004F073F8E12120004902C6
:1071E00003F05CFFFA20C00006F016FAC249200046
:1071F00005F074FDC14D280001F081F9002128003F
:1072000001F0DEF9BE4BBF4A0BA9BF480B93FBF759
:10721000D9FA002800D1EFE0BC49200005F025FD97
:1072200006F0C4F90A220100200005F09FFD642346
:10723000B74A0BA9B7480B93FBF7F5FB01211020C8
:1072400006F09AFC01210F2006F096FC01210E2089
:1072500006F092FC0121152006F08EFC012114207D
:1072600006F08AFC0021152006F0D2FC0021142033
:1072700006F0CEFC0121112006F07EFC0121072042
:1072800006F07AFC0021122006F076FC0021042092
:1072900006F072FC0021082006F06EFC01210C2093
:1072A00006F06AFC01210C2006F0B2FC30229A4B59
:1072B0001A7006F07BF9994B0BAA1860984843693D
:1072C000016903F0DFF8974E974A0BA9300009F0E7
:1072D000A6FA3378013B022B00D992E0934905A826
:1072E00005F0D6FD0A22317802A805F0FEFD02A9BC
:1072F00005A805F008FF0100200005F0E5FC02A844
:1073000005F077FD05A805F074FD3278884B1A70FA
:107310007378884DB42B79D88749200005F0A5FCF7
:107320000A22717805A805F0E0FD05A9200005F006
:10733000CBFC05A805F05DFD73782B70B378B42BFA
:1073400069D87E49200005F090FC0A22B17805A892
:1073500005F0CBFD05A9200005F0B6FC05A805F059
:1073600048FDB278764B1A70F678012E58D1FF227C
:107370007449754809F0E1FFFF227449744809F027
:10738000DCFF744B1E70744E0521300000F038FF96
:107390002978300000F084FF704F386806F03CF91F
:1073A000300000F035FF6E4E0A21300000F028FF5B
:1073B0002978300000F074FF386806F02DF93000AD
:1073C00000F026FF674E0321300000F019FF2978F6
:1073D000300000F065FF386806F01EF9300000F05C
:1073E00017FF614D280001F0DDFBFF281CD15F492C
:1073F000200005F073FCFEE75D49200005F05AFC13
:1074000015E75C49200005F055FC81E75A4920004A
:1074100005F050FC92E75949200005F04BFCA3E72A
:1074200000234C4A1370AEE74A4B1B78012B23D143
:107430005349200005F052FC5249280001F099FB05
:107440000627514E3368032B00D1AFE0013F002FD8
:1074500048D04E49200005F013FC3B49200005F0C0
:107460003DFC3B4A3849280001F0ACFB3060FA2073
:10747000800006F0D1F8E4E74549200005F02EFC35
:107480000F23A8220093C0210B3B05A805F0D2FAD8
:1074900005A9280001F051FB3E4A3F49280001F0B0
:1074A000FBFA002809D120003C49FA2405F016FC1B
:1074B000A400200006F0B0F8FBE7FA20800006F0F8
:1074C000ABF8290005A801F064FB3549200005F060
:1074D000D7FB05A9200005F0DCFB3249200005F0B0
:1074E000FDFB83E03049200005F0CAFBF5E7C0460C
:1074F000CCFDFFFF401A0020423801005807002051
:107500000000C842312B0000D80400205B38010085
:10751000CD210000940200209002002028000020CD
:10752000840900208007002002020000AB3801001F
:107530002C000020C0050020DA38010023390100AA
:1075400014000020840700209C0C002083080020E9
:107550009D0B00209C0B0020340700201C00002005
:10756000370700203A070020480E00206E3901003E
:107570007B380100BC380100F738010041390100B7
:10758000963901007A3001009C0D0020B1390100CC
:10759000253A01003D3A0100483A0100513A010004
:1075A000623A0100732E0100A93A0100290005A8E2
:1075B00001F0EFFA2949200005F062FB05A920003F
:1075C00005F067FB264E2000310005F087FB2549BA
:1075D000254801F00FFE2549002800D1244920004C
:1075E00005F043FB3100200005F064FB05A92800ED
:1075F00001F0C4FA1F49200005F042FB00256B464C
:1076000014229B185B5D0F2B03D81B49200005F04B
:1076100037FB14226B469B18595D043A200005F095
:10762000A1FB6E1C052D06D01449200005F028FB97
:107630003500062EE3D10A49200005F04FFB104823
:1076400001F06DFD0F49200005F048FB0E492000B8
:1076500005F044FB8D239B009D44F0BDC83A01001A
:10766000732E0100E37D0000B4060020DA3901002A
:10767000FD390100733A0100233801007C3A010012
:107680008C0B00207E3A0100963A0100102228233C
:10769000F0B595B000AFBA18D4189B49002220006D
:1076A00001F04CFD9948FB6B4360A3688360E3687D
:1076B000C360237C0374638A4382237D037501F0D6
:1076C000C4FAB860002800D1DAE014239049F81811
:1076D00005F0DEFBBC688D4801F0C8FC002800D135
:1076E000CAE08A4801F01AFB0028F4D0874801F06C
:1076F00021FBC3B2FB6019001423F81805F0DDFC70
:10770000FB680A2B00D0F9E0002CE3D01424190008
:10771000381905F0A2FD102528260300781939191B
:107720000022801905F0DAFD7A199019FCF732FF72
:107730007A190400901905F05CFB002C78D0102019
:1077400000233A18734D901973492B6005F0A0FB84
:1077500010201423391801228919F81805F082FD28
:107760000600102028233A18D01805F042FB002EFE
:1077700048DD6A4614230F367A60F9683200F8183B
:1077800005F05CFD3200102614210300B8197918A9
:10779000801905F0A3FDBA19901905F0A5FE6946F8
:1077A000C31DDB08DB00C91A8D460200286057485C
:1077B00001F0D6FA10230C36FA186946901905F034
:1077C00067FB296810257B19981905F051FE7A1975
:1077D00018359119501905F0E2FB1023FA185019C9
:1077E000FCF78AF91023FA185019183D05F001FB2F
:1077F0007B19981905F0FDFA7B19581905F0F9FA6B
:107800007B689D46142310262825F818404905F06A
:10781000D6FB4249BB193031581905F0C0FBBB19E2
:107820005819FDF7C3FDBB19581905F0E2FA52E7E4
:10783000102528262C007B1998193449FCF70AF9E1
:107840007A195019324905F023FB0C353A195019B1
:10785000334905F0A4FB3A19391938195219091995
:107860008019FDF7E5F83B19581905F0C2FA3B19E4
:10787000181905F0BEFA2DE71423F81805F0B9FA27
:10788000284C200001F064FD002834D0264D182239
:1078900029001026200001F0A1FD29001C25BB199C
:1078A000581905F0F5FABB19581905F0F4FDBB1984
:1078B0001E49581905F078FC002816D0BB190C3564
:1078C0005819210001F079FD200001F065FDBB1978
:1078D00002005919200001F0FDFC1122144920007A
:1078E00001F015FD200001F00DFD10221C23BA1837
:1078F000D01805F07EFABD4615B0F0BDFB680D2B23
:1079000000D1E8E60024E6E68C0B00209C05002070
:107910001D3801008C020020FD2C01009C0A002073
:1079200084050020B4060020240500200D2D010050
:107930001E2D0100F0B593B0FBF78CFF7B4B1B783D
:10794000002B01D0FBF7C6FF042006F08DF9784D1F
:10795000071E7BD105F02AFE764E774C3368C01A9D
:10796000764B1B68984223D9122006F097F8C8235B
:1079700001229B00984200DC3A0071490A6071497B
:10798000984211DD0B68002B0ED101276E48236849
:10799000076028780133471E2360012F00D9BBE020
:1079A000042B01D1002323600A6005F0FFFD306045
:1079B0002768002F07D1654E3368002B03D0302095
:1079C000FBF750F937602768012F07D15F4E336806
:1079D000012B03D03120FBF745F937602368022BD8
:1079E0000AD15A4E3368022B06D02F78022F03D1CA
:1079F0003220FBF737F937602768022F0AD1534E40
:107A00003368022B06D02B78022B03D03320FBF7F0
:107A100029F937602768032F0AD14C4E3368032BAE
:107A200006D02B78022B03D13320FBF71BF93760EC
:107A30002668032E0AD1454C2368032B06D02B78E9
:107A4000012B03D13420FBF70DF92660404C2000B8
:107A500003F026FC00281CD00A22210003A805F010
:107A6000A5F903A805F017FD059B052B0ED903A961
:107A700006A805F094FA002206A90CA8FBF7FEF967
:107A80000CA805F0B6F906A805F0B3F903A805F0AF
:107A9000B0F92B78042B46D106A800222D4901F01D
:107AA0004DFB06A801F0D1F8002833D02A49200068
:107AB00005F0E6F806A90CA801F077F90CA920005A
:107AC00005F016F90A2206A9684605F06FF968461E
:107AD00005F0E1FC6946200005F0F6F869460CA8BF
:107AE00005F05DFA01220CA903A8FBF7C7F90CA861
:107AF00005F07FF903A906A805F0E6F806A801F04D
:107B0000A3F806A801F094FA03A805F072F96846F4
:107B100005F06FF913B0F0BD032800D044E7032B44
:107B200000D041E73EE7FFF7B1FDF3E70C07002087
:107B30002C000020280000208002002018000020D7
:107B400054070020240700207C0700208402002026
:107B5000401A00208C0B002030380100F8B50700D7
:107B60000C0000258E18B4420BD021780D2906D0C8
:107B70003B6838001B689847002802D00135013463
:107B8000F1E72800F8BD00000023012170B5436033
:107B90000B4B0C4A08330360136804000B400A4D7A
:107BA00005D12B60094B11606B602F232B8100F0F6
:107BB000B5F9290000F06EF9054B2000236170BD76
:107BC0000C3B0100B40D0020B80D0020DB3A010091
:107BD000243B010010B50C0000F0A0F9082322009E
:107BE000022100F067F910BD10B587291FD978313F
:107BF000C9B2837A8B4214D0C37A8B4211D0037BF3
:107C00008B420ED0437B8B420BD0837B8B4208D0C0
:107C1000C37B8B4205D00023C218947A002C31D14B
:107C2000917201000831FFF7D5FF012011E04BB23E
:107C3000002B07DA012380398B40027A002113439D
:107C40000372D6E70369595C002903D1012343601D
:107C5000002010BD3F220B009343C02B08D1047AB3
:107C6000803B2343037211403229C2D13231C0E735
:107C70004BB2002BF8DA0223027A134303727F23FC
:107C80001940F1E70133062BC6D1DFE770B587292C
:107C900016D97831C9B20300020000240A33103229
:107CA000002903D01D788D4200D11C70013393420E
:107CB000F6D101000831FFF78DFF0123180070BDD8
:107CC0004BB2002B07DA012280398A40037A002167
:107CD00093430372DFE70369595C00239942EDD0B7
:107CE0003F220B009343C02B08D14024037A11405C
:107CF000A34303723229CED13231CCE74BB2002BF1
:107D0000F8DA0222037A934303727F231940F1E7E2
:107D100070B505000E00FFF767FF04003100280072
:107D2000FFF7B4FFE0B270BD10B50248FFF72CFFBB
:107D300010BDC046A00D0020482310B50F240B70C5
:107D400001334B70053B8B70028B22404132CA706D
:107D5000038B05201B11234041330B7110BD000024
:107D600030B50B7889B001330B706B4605000D22DE
:107D70000021981D08F06FFD134B01AC2380134BBD
:107D8000134AA380092363721833A372203BE37262
:107D9000237323762B79E2810E4AA3702B8B6282A8
:107DA000032223741B126374802362753D32E282C6
:107DB0006A795B421343210019220748237503F0B7
:107DC000FDFE09B030BDC0460904000001030000FB
:107DD0000122000007050000A41A0020F8B50B7866
:107DE00004000025812B22D1CB78222B1FD14B7987
:107DF000087922791B0203439A4218D12F000D4EB5
:107E00000121300003F0E2FF6469002C0AD02289CE
:107E10006168300003F0D2FE0500431C07D03F1814
:107E20002468F2E72100300003F0D0FF3D00280075
:107E3000F8BDC046A41A00200B0010B55A79097984
:107E4000047912020A430021944211D11C785A7815
:107E5000A12C0FD1022314009C43012C16D0022A1E
:107E600006D1020001231B32094803F083FE0121E1
:107E7000080010BD212CFBD10B2A02D19B78837600
:107E8000F5E70A2AF4D19B78C376F0E72100EFE703
:107E9000A41A00204369002B06D14161038B0A8993
:107EA0009B180383704713001A68002AFBD11960DE
:107EB000F4E7000030B591B01C0005006B460800E7
:107EC000110018702200581C08F0A9FC631C697985
:107ED0006A46024803F0C8FD11B030BDA41A002064
:107EE0000223FF3310B5C380030010338360094BB6
:107EF00083220833036000230400C3604361064B00
:107F00000261836104F076FE210004F044FE20004B
:107F100010BDC046A43B01000000010170B5012660
:107F2000054D064C2B68334203D12000FFF7D8FFE4
:107F30002E60200070BDC046C40D0020C80D00207A
:107F4000F7B50C27404E0193335C04005BB20D0083
:107F500000924743002B2EDA00230B82EB7BDB09D8
:107F6000FCD1335D394A01335BB23355335D12784E
:107F70005BB2DB19934203DA335D5BB20B2B34DD6A
:107F80002F8ABFB2EB7BDB09FCD1314B314918683A
:107F900005F042FF304B04375843009B00090C3377
:107FA00087424DD280B25B005853EB7BDB09FCD19A
:107FB000FF33335540E0335C244A5BB21278DB195F
:107FC0009342CEDA335C254A5BB2DB19DB009B5C63
:107FD0005B06C6D5335C00215BB2DB19DB00985C25
:107FE0008006800E05F014FEBBE7335D1B4A5BB2D2
:107FF000DB19DB009B5C5B0609D5335D01215BB2BD
:10800000DB19DB00985C8006800E05F001FE2A8AF1
:1080100092B2EB7BDB09FCD1335D5BB2DF190F4B16
:10802000FF00DF197B68D318009A9BB20C32520014
:108030005353EB7BDB09FCD16B461B79AB73F7BD6C
:10804000BFB25B005F53B0E7E50D0020E40D0020F8
:108050003800002040420F00204E0000E80D0020B4
:10806000002210B5102302491000FFF769FF10BD70
:108070000030004270B50C4B05001C780B2C10D85A
:10808000621C1A70094B04701868094905F0C4FE97
:10809000084BE4005843084B00091C196060280095
:1080A00070BDFF230370FAE7E40D002038000020C4
:1080B00040420F00DC050000E80D0020F7B50193F9
:1080C000037804000E0017000B2B00D986E0C8B21D
:1080D000012105F051FD3F2132002078404DC300C1
:1080E0005E5D0A408E4316435E5588230322962127
:1080F0009B00DB1BDF171740FF18019B0901C91A02
:10810000CB1713405B189B10BF10A37067700C2136
:1081100005F082FE0C23C0B243431A000C32D90092
:10812000695C490654D401339342F8D100284FD1F9
:108130002C4B2D4A5A805A78D209FCD12B4E023250
:10814000338893433380F37BDB09FCD101333380E5
:10815000F37BDB09FCD13388DB07FCD433889BB28B
:108160003380402332881343338080233288DB00FE
:10817000134333800123327913433371F37BDB09DB
:10818000FCD11B4B1B49186805F046FE0300FA2082
:1081900080005843000980B23083F37BDB09FCD1B7
:1081A0008021154B0903D967C023C420134A5B0003
:1081B000D150800013581B021B0A1350102311606A
:1081C000737332880E3B13433380F37BDB09FCD19E
:1081D00040222378DB00E95C0A43EA542078FEBDA4
:1081E000E80D0020000C00401C4000000030004260
:1081F0003800002040420F0004E100E000E100E010
:108200009623882210B51B019200FFF757FF10BD7F
:108210004021007810B50C4CC200135D8B43135500
:10822000343905F0F9FDC3B20C20584303000C3378
:10823000C200A25C520605D401309842F8D1102247
:10824000024B1A7310BDC046E80D002000300042FA
:1082500070B505780B2D1BD801238824C356E41A6A
:10826000A4008C4208DC96248078A40040B2241A32
:10827000A4008C4200DD0C00064B0749186805F08D
:10828000CBFD053C6043054BED0000095D196860BE
:1082900070BDC0463800002040420F00E80D0020AD
:1082A0000F4B13B50400994216DCB420B42902DC4C
:1082B000C843C017084001228823A25602219B1AF6
:1082C000962261569200521A9200009200219B0061
:1082D000B42204F0DBFA01002000FFF7B9FF13BD60
:1082E0001F02000000230922C360C37103720370E0
:1082F000C2704370083AC361FF33027142718271E8
:10830000038370470023C371037203700933C37082
:10831000083BC160037143718371704770B50400FD
:108320000D00FFF7DFFF29002000FFF7EBFF200023
:1083300070BD10B54378002B03D08078002105F084
:1083400067FC10BD10B54378002B03D08078012165
:1083500005F05EFC10BD0B78282B04D005D8102B3F
:1083600001D0222B05D1012004E03B2BFBD0422B76
:10837000F9D00020704710B50C000721200000F054
:1083800041FBE379181A43425841C0B210BDF7B51A
:10839000C37905000F001600934214D90024C06869
:1083A00000F098FA731CDBB2019301223900E868EF
:1083B00000F0B2FA002806D0A64206D00134019B94
:1083C000E4B29C42F1D1002005E039002800FFF71B
:1083D000D2FF0028F2D0FEBD70B50400C0680D00C9
:1083E00000F0D6F9002D12D1E06800F06DFA0022FD
:1083F000B421E06800F026FAE06800F00DFA05000C
:10840000E06800F0C5F968426841C0B270BD29005B
:10841000E06800F047FAEAE78A18914206D0013195
:108420004B1E1B78002BF8D0002070470120FCE782
:10843000F8B50600C0680F001500002400F0A8F988
:10844000A04218D03900F06800F02CFA2200BE21BA
:10845000F06800F0F7F92C000935F06800F010FA28
:1084600020700134AC42F8D1F06800F091F9013885
:1084700044424441E4B22000F8BD70B50500140048
:10848000FFF7D6FF002811D0092221002800FFF7AE
:10849000C3FF03000020834208D10821200000F020
:1084A000B1FA237A181A43425841C0B270BD30B5B0
:1084B0000A7885B00C000C23102A1DD001AD2A00CB
:1084C000FFF7DBFF0023984216D023782A793B2B55
:1084D00003D151B22F3B00290EDB0A233F2A0BD0D8
:1084E00004D8013B1F2A07D0002305E00B235F2A95
:1084F00002D001337F2AF7D1180005B030BD37B55F
:1085000004000325E06800F0E5F900233220E37160
:10851000237205F081F801226946E06800F0FCF959
:10852000002825D069462000FFF725FF0028F2D05B
:10853000E37969460133E3712000FFF70CFF00285F
:10854000E9D0237A013323722378002B07D16946BF
:108550002000FFF741FF002801D001232370694666
:108560002000FFF7A4FFE3788342D4D2E070D2E783
:10857000E379002B03D1013DEDB2002DC2D137BD0F
:10858000064B10B5984206DB06F05EFAF02189052D
:1085900006F008F910BD0248FCE7C04681E4FFFF81
:1085A0000000FEC20938C0B2022803D8024B4000C6
:1085B000C05A70470148FCE7BC3B0100EE020000D6
:1085C0000171704710B5C06800F026F901384342C8
:1085D0005841C0B210BD000070B5437904001500C9
:1085E000002B10D00378002B0DD12000FFF7EAFFFD
:1085F000002815D104F0DAFF0A4B401B98420FD82F
:1086000005F037F8F1E70800FFF7CCFF0500200080
:10861000FFF78FFE280004F0FFFF2000FFF792FE17
:1086200070BDC046ED020000002370B50C00036071
:10863000013303700500C86800F0AAF8E06800F094
:1086400043F922784421E06800F0FCF804F0AEFF22
:10865000686023790200002B03D0E1782000FFF747
:10866000BBFF280070BD0000F8B556780F7875B2D2
:10867000ED17EC04250013783B2F1ED111797F29CB
:108680001BD901210B4210D094780C423CD1A30796
:108690003CD40420044063425C41C5206442C001D4
:1086A0001B4B0440E4182000F8BDFC20DB00C00098
:1086B0000340F60233431C43F5E7F1020C00D800F7
:1086C00004432C43282F0ED1502B06D1052EEAD17E
:1086D00093790C2BE7D10F4CE5E7FF2BE3D1072E65
:1086E000E1D10D4CDFE7102FDDD1D1790029DAD0AF
:1086F0009079E400081AC00105F018FC074B1C40F3
:10870000203C04192C43CEE7054CCCE7054CCAE7C6
:108710000082FFFF8082FFFF0083FFFF80FF0700D2
:108720000081FFFF8081FFFFF0B505000E001700FC
:10873000002485B0E3B29F420ED301AA3100280085
:10874000FFF79BFE01340028F4D001AA3100280075
:10875000FFF78AFF05B0F0BD0048FBE780E4FFFFAC
:1087600010B5FFF7E1FFFFF70BFF10BD13B50A00CF
:1087700069460400FFF70BFE002805D00022694679
:108780002000FFF7EDFF16BD0048FCE70000FEC229
:1087900070B550C872B6746062B67D25013DEDB209
:1087A000002D1CD0022004F059FF336A1C42F5D082
:1087B00072B67461B46062B6F020400004F04EFFFF
:1087C00072B64620746004F049FF336A1C4063426D
:1087D0005C41E5B262B6CD20400004F03FFF2800C6
:1087E00070BD70B505684468CB070BD572B60A201A
:1087F0006561A56004F032FFA56162B6372004F020
:108800002DFF70BD72B641206561A56004F026FFA2
:10881000A56162B60520F2E770B530C872B60320D4
:10882000AC606C6104F01AFF6C600A2004F016FF63
:108830002D6A62B635202C4004F010FF601E844182
:10884000E0B270BDF7B504000F00082601250192C3
:10885000290039404B1E99412000C9B26D00013EEC
:10886000FFF7BFFFEDB2002EF2D1019B002B06D126
:1088700072B6636822685A600CCC5A6162B6F7BD62
:10888000F8B507000826002501243800FFF7C4FFCB
:10889000002800D025436400013EE4B2002EF4D14C
:1088A0002800F8BD70B50C000022552126000500F7
:1088B000FFF7C8FF08362178002228000134FFF7AF
:1088C000C1FFB442F7D170BD10B50022CC21FFF733
:1088D000B9FF10BD002383748360C36003827047B7
:1088E00070B50D0004000021280005F045F918219D
:1088F0006943074A531858680123834023608B5605
:10890000044ADB019B1863602000FFF7E3FF70BDA2
:108910006042010000440041F0B585B00391867CBF
:1089200005001400002E03D1FFF732FF002804D108
:108930000020A874288205B0F0BD002C2BD0320096
:10894000F02101272800FFF77DFF00233E0001935F
:1089500002932800FFF760FF04002800FFF75CFF88
:10896000012C1BD1012833D1402EE1D96B461B7A53
:108970002B74029B002B01D10133AB742B7A002B9B
:10898000D6D00023EA18127A0399CA540133082B6F
:10899000F8D10120CFE72200EC21D2E7019BEB18B0
:1089A00084420DD12C7CB4420ED91C7A3C40621E0C
:1089B0009441E4B2002C0BD10296082E00D86E74BC
:1089C0001A7ABA431A7209E0A41B62425441F0E7D2
:1089D0000124019BEA18137A3B4313727F002100A4
:1089E00028000136FFB2FFF7FCFEF6B2002F04D1DB
:1089F000019B01370133DBB20193019B072BA8D9FF
:108A0000B2E7000030B5030041180F240020074AE8
:108A10008B420AD01D7801336840050000092540CB
:108A20001018555D007C6840F2E730BDC23B010084
:108A300070B5060004F0BAFD0024050004F0B6FD90
:108A40003368401B984207D2642004F0E5FD01F032
:108A50003DFB04000228F1D9200070BDF0B50700ED
:108A600085B0080016000D00039308F05FFC0400B9
:108A7000300008F05BFC039AC3B20092E1B232000E
:108A8000280001F025FC03000920013302D0380042
:108A9000FFF7CEFF05B0F0BD10B50123FFF7DEFFF5
:108AA00010BD0000030070B5044A04C30A1D70CA5B
:108AB00070C312681A600B7D037570BD78460100A3
:108AC00010B5080014000A7D00218A4200D1016916
:108AD0000022187D904200D11A690023022001F083
:108AE00025FA0021237D8B4200D12169002201203B
:108AF00001F06AFA10BD70B598B00500684616001E
:108B00000C00FFF7CFFF0321684603F0E7FF0123C6
:108B10002100037006A8FFF7C5FF31000CA8FFF77E
:108B2000C1FF694612A8FFF7BDFF12AB0CAA06A948
:108B30002800FFF7C5FF18B070BD30B593B0050031
:108B400068460C00FFF7AEFF0321684603F0C6FF3E
:108B500001232100037006A8FFF7A4FF69460CA8B3
:108B6000FFF7A0FF0CAA06A92800FFF7C4FF13B067
:108B700030BD10B5080001F069FA10BD10B50C0049
:108B800001F0CEFA06220100200007F048FE200086
:108B900010BD10B5040003F045FF200001F0F6FA07
:108BA000200010BD10B501F091FA10BD10B50800FD
:108BB000110001F081FB10BD436810B5002B00D0FF
:108BC000984710BDF8B5050008000E00170008F022
:108BD000ADFB0400380008F0A9FBE1B2C3B23A00D3
:108BE000300001F05FF90424431C14D004F0DEFCD3
:108BF0000024060004F0DAFC2B68801B98420AD29D
:108C00002800FFF7D9FF642004F006FD01F05EFAAA
:108C100004000228EED92000F8BD00000022024B1B
:108C2000024906C37047C046480E002050C30000EA
:108C300013B56B460268D9710733546819000122D5
:108C4000A04716BD017570477047007CFF38431E72
:108C50009841C0B270470000F0B50E008FB004001C
:108C600002A8019203F0DEFE02AA31000B48FFF7D2
:108C70009DFF002810D0236803AADE69084B08A9CD
:108C8000089309ABA1CAA1C3126820001A6002AB05
:108C90001B7D019A0B75B0470FB0F0BD480E002048
:108CA0007846010013B5069C080011001A0004ABB9
:108CB0001B880194059C009400F0EEFF16BD10B5D2
:108CC00001F036F810BDF8B50500007C0E00140068
:108CD000FF2804D1012300246B602000F8BD002A86
:108CE000F8D092B200F020FF002815D12B7D002B88
:108CF00003D1287C00F06EFDECE72B682200DF6CCE
:108D0000310001232800B847041EF2D0287C00F06F
:108D10004DFF0028DED0E0E70400F7E710B5017C46
:108D20000020FF2902D0024800F09EFB10BDC04683
:108D3000500E0020036837B51B69040098470028CF
:108D400009D06B46DD1D217C01232A00034800F079
:108D5000C7FB28783EBD01204042FBE7500E0020B3
:108D600010B50C001300017C2200024800F0B8FB93
:108D700010BDC046500E002010B5017C014800F027
:108D80009FFB10BD500E002007B500236A460193DB
:108D90001380007C01A901F041F86B466A461B78FC
:108DA00050781B02C01880B20EBD13B500236A466E
:108DB000040001931380087C01A901F02FF801A998
:108DC000200003F053FE200016BD00007FB5037C99
:108DD00004000D001600FF2B02D003689B6A984721
:108DE00000F030FF2074FF2816D000222B7D934224
:108DF00000D12A69638A0021029302230090019323
:108E00000800330000F08CFC23682000DB6A9847E0
:108E1000431E984104B070BD0249034803F05EFF51
:108E20000020F7E7E23B0100401A0020F8B50500FA
:108E30000E001700002B0AD00524BAB2287C31009E
:108E400000F072FE002803D1013C002CF5D1002077
:108E5000F8BD0000F0B5037C85B004000E001700DB
:108E6000FF2B02D003689B6A984700F0EBFE0500D9
:108E70002074FF2815D0300008F058FA638AC1B278
:108E8000029304230022019330003B00009500F080
:108E900047FC23682000DB6A9847431E984105B0D1
:108EA000F0BD0349034803F019FF0020F7E7C0466F
:108EB000E23B0100401A0020F0B5037C85B00400BD
:108EC0000E001700FF2B02D003689B6A984700F042
:108ED000B9FE05002074FF2815D0300008F026FAEE
:108EE000638AC1B2029302230022019330003B0047
:108EF000009500F015FC23682000DB6A9847431EAC
:108F0000984105B0F0BD0349034803F0E7FE002097
:108F1000F7E7C046E23B0100401A00207FB5037C22
:108F200004000D001600FF2B02D003689B6A9847CF
:108F300000F088FE2074FF2816D000222B7D93427B
:108F400000D12A69638A00210293042300900193CF
:108F50000800330000F0E4FB23682000DB6A984738
:108F6000431E984104B070BD0249034803F0B6FEA9
:108F70000020F7E7E23B0100401A00207FB5037CA8
:108F800004000D001600FF2B02D003689B6A98476F
:108F900000F058FE2074FF2816D00023297D1A0007
:108FA000994200D12A69618A0193029100210090BF
:108FB0003300080000F0B4FB23682000DB6A984708
:108FC000431E984104B070BD0249034803F086FE79
:108FD0000020F7E7E23B0100401A0020FA239B0043
:108FE0008360054B002208330360FF230374FE3BBC
:108FF0004260428203757047F83B0100FA239B00F0
:109000008360054B00220833036001234260017432
:10901000428203757047C046F83B010010B5037CDF
:109020000020FF2B02D0180000F008FC10BD00004B
:1090300070B50400007CFF2814D000F0CBFB322573
:109040002000FFF7EBFF002806D0013D002D03D0E4
:10905000642004F0E1FAF3E7217C034800F0EAF928
:10906000FF23237470BDC046500E002070B5037CF2
:1090700004000025FF2B05D003681B699847A84210
:1090800002D00125280070BD2000FFF7C7FF0A2885
:10909000F7D8054BC340DB07F3D5217C034800F02C
:1090A000C9F9FF232374EDE7EF040000500E002000
:1090B00013B56B460268D971073354681900012251
:1090C000A04716BD70B50500002A04D10123002475
:1090D0006B60200070BD92B2007A00F025FD041E86
:1090E000F4D0287A00F062FD0028EFD0F1E700000C
:1090F000044B41810833036000234360013B03813B
:109100007047C0465C3C010010B50400007AFF289F
:1091100004D000F093FA01235B42238110BD10B507
:109120000400FFF7F1FF00F08DFD01002072FF2821
:1091300003D06089002200F001FA10BDF0B50B7A6F
:1091400089B004000D001600FF2B39D0497AFF29A1
:109150000FD002A8FFF752FF02A8FFF787FF0028F1
:1091600007D002A8FFF7DAFD002802D0687AFF28AE
:1091700005D1287A002100F0D3FBFF2820D0C7B208
:10918000390002A8FFF73AFF002E03D002A8FFF72C
:1091900045FF3070039B6F726360049BA360059B67
:1091A0000193E360094B236002AB1B7C237402AB89
:1091B0005B8A638202AB1B7D2375200009B0F0BD82
:1091C000FF212000FFF71AFFF7E7C046003C01002F
:1091D00010B503689B6B984710BD4069704713B585
:1091E0006B460268D9710733546819000122A04701
:1091F00016BD7047F8B5037C04000F00FF2B02D0AA
:1092000003685B6A984700F01DFD00250600FF28F3
:1092100008D001000122380000F090F96561267441
:10922000678201352800F8BDF8B5037C04000F0003
:109230001600FF2B02D003685B6A984700F002FD1E
:1092400005000020FF2D0DD03B7D834200D1386901
:1092500003232A00310000F0AFF900230120257418
:1092600066826361F8BD000010B50400007CFF2831
:1092700007D000F0AFFA217C024800F0DBF8FF23B2
:10928000237410BD500E0020F0B50E008FB0040006
:1092900002A8019203F0C6FB02AA31000B48FFF7B7
:1092A00085FC002810D0236803AA9E6A084B08A9F1
:1092B000089309ABA1CAA1C3126820001A6002ABCF
:1092C0001B7D019A0B75B0470FB0F0BD480E002012
:1092D0007846010070B5037C04000D001600FF2BDA
:1092E00002D100F0AFFC2074227C0020FF2A08D0BD
:1092F0002B7D834200D128690123310000F0CEF993
:10930000012070BD10B5007C00F0D0FB10BD10B581
:109310001400007C92B200F07FFB200010BD000022
:10932000436937B50400002B0CDD6B46DD1D017C65
:1093300001232A00054800F0D3F863692878013B2F
:1093400063613EBD01204042FBE7C046500E002055
:1093500013B504006369217C5A1E6261002B06D09C
:109360006A4601230732044800F0BAF8F2E7080021
:1093700000F09AFA606116BD500E0020436910B5E6
:10938000002B04DD017C034800F09AF810BD012099
:109390004042FBE7500E002007B500236A460193C8
:1093A0001380007C01A900F039FD6B466A461B78EA
:1093B00050781B02C01880B20EBD13B500236A4658
:1093C000040001931380087C01A900F027FD01A986
:1093D000200003F04BFB200016BD000070B5040018
:1093E0000020130062690D00824209DD217C2A0001
:1093F000044800F075F8002802DD63691B1A6361F8
:1094000070BDC046500E0020FA239B008360044BC1
:10941000002208330360FF234260037442617047F7
:10942000783C010010B504007822002107F013FAFF
:10943000200010BD10B50C244C43041920680028EE
:1094400005D007F0C1F9002363602360A36010BD5D
:1094500070B505000024210028000134FFF7EAFF61
:109460000A2CF8D1280070BDF7B50C244C43041920
:10947000A36805000E00002B1AD12768002F05D124
:109480000E4807F097F9A760606020606B469F1D4B
:109490000A4BF0B23A0021683B8000F081FA0028C4
:1094A00006D023683A8863600C237343EB189A60F4
:1094B0000C235E43AD19A868FEBDC046DC05000064
:1094C00070B504000D00FFF7CFFF002805D00C2178
:1094D000694364186368187870BD01204042FBE757
:1094E000F8B506000C0017001D00FFF7BDFF0028AF
:1094F00011D0854200DD05000C235C4334192A009D
:109500006168380007F08BF9280063685B196360B5
:10951000A3685B1BA360F8BD10B5054C2000FFF7E6
:1095200081FF044A0449200004F064FC10BDC046D9
:10953000500E002000000020519400007FB56B46C3
:10954000DD1D9C1D1B4B0600187829702270002819
:1095500001D101F02DF9002001F012F901F086F996
:109560000321282001F034FB3000002101F01EFB14
:1095700028000022012101F0EDF901222000110054
:1095800001F0E8F901F0C6F901F098F9002001F0C6
:10959000F7F801F06BF90E220F2300216A446B44A7
:1095A000117019702820013101F0FCF901F086F9E1
:1095B0007FBDC046411300207FB50E0069468C1C5C
:1095C00023701D4B01901878CD1C2A70002801D102
:1095D00001F0EEF8002001F0D3F801F047F9042182
:1095E000282001F0F5FA002201A8042101F0B2F9C7
:1095F0003000002101F0DAFA28000022012101F0F8
:10960000A9F901222000110001F0A4F901F056F996
:10961000002001F0B5F801F029F90E220F230021F6
:109620006A446B44117019702820013101F0BAF9B5
:1096300001F044F97FBDC046411300201FB56B46C1
:10964000DC1D154B20701878002801D101F0B0F80E
:10965000002001F095F801F009F90121382001F00E
:10966000B7FA01222000110001F074F901F026F987
:10967000002001F085F801F0F9F80E220F230021F7
:109680006A446B44117019703820013101F08AF975
:1096900001F014F91FBDC046411300207FB50E0034
:1096A00069468C1C23701D4B01901878CD1C2A70C4
:1096B000002801D101F07CF8002001F061F801F0F0
:1096C000D5F804212D2001F083FA002201A80421FD
:1096D00001F040F93000002101F068FA2800002272
:1096E000012101F037F901222000110001F032F9C7
:1096F00001F0E4F8002001F043F801F0B7F80E2281
:109700000F2300216A446B44117019702D20013120
:1097100001F048F901F0D2F87FBDC04641130020A6
:10972000F0B585B01E000CAB1C88294B07001878DB
:109730000D000192002801D101F03AF8002001F05B
:109740001FF801F093F806212D2001F041FA3800AE
:109750000022290001F0FEF80022042101A801F0F6
:10976000F9F83000002101F021FA0BAE00220121AE
:109770000AA801F0EFF800220121300001F0EAF818
:109780000121200001F012FA03272C0014343C4080
:109790000135002C02D001F0BDF8F6E701F08EF89B
:1097A0003078043843425841C0B200F0E9FF01F07C
:1097B0005DF80E220F236A446B4401212D201470A2
:1097C0001C7001F0EFF801F079F805B0F0BDC0466B
:1097D000411300201FB56B46DC1D174B2070187815
:1097E000002801D100F0E4FF002000F0C9FF01F0E3
:1097F0003DF801212E2001F0EBF90122200011009B
:1098000001F0A8F801F086F801F084F801F056F8AC
:10981000002000F0B5FF01F029F80E220F230021EF
:109820006A446B44117019702E20013101F0BAF8AE
:1098300001F044F81FBDC046411300201FB56B4620
:10984000DC1D184B20701878002801D100F0B0FF03
:10985000002000F095FF01F009F801212F2001F010
:10986000B7F901222000110001F074F801F052F85C
:1098700001F050F801F022F8002000F081FF0E24E2
:1098800000F0F4FF0F2300226C446B441A70227026
:10989000012122002F2001F085F801F00FF8207837
:1098A00004B010BD411300201FB56B46DC1D2070B5
:1098B00000F076FF002398422DD0184B187800282E
:1098C00001D100F075FF002000F05AFF00F0CEFF3C
:1098D00001212B2001F07CF901222000110001F070
:1098E00039F801F017F801F015F800F0E7FF002053
:1098F00000F046FF0E2400F0B9FF0D2300226B4458
:109900006C441A702280012122002B2001F04AF8B9
:1099100000F0D4FF2388180004B010BD41130020CC
:1099200030B585B06B46DD1D9C1D2870217000F0A0
:1099300037FFFF2300282ED0184B1878002801D1BC
:1099400000F036FF002000F01BFF00F08FFF022127
:109950002B2001F03DF900220121280000F0FAFF40
:1099600001222000110000F0F5FF00F0A7FF002009
:1099700000F006FF0E2400F079FF0D2300226B4457
:109980006C441A702280012122002B2001F00AF879
:1099900000F094FF2378180005B030BD411300207B
:1099A00073B56B46DD1D0E001400287000F0F8FE44
:1099B000002801D1208076BD164B1878002801D1EF
:1099C00000F0F6FE002000F0DBFE00F04FFF022169
:1099D000452001F0FDF800220121280001F0D1F816
:1099E00001220221200001F0CCF800F093FF00F0EA
:1099F00065FF002000F0C4FE00F038FF22003100B7
:109A0000452001F08CF800F059FF2088431E984152
:109A1000C0B2D0E7411300207FB56B46DC1D224B5E
:109A2000207018780E001500002801D100F0C0FE4B
:109A3000002000F0A5FE00F019FF0221462001F0F1
:109A4000C7F800220121200001F09BF8300001221C
:109A5000290001F096F803262C0009343440013522
:109A6000002C02D000F056FFF6E70E250F2600F07E
:109A700025FF6E4420006D4400F082FE00F0F6FEEB
:109A80003200290046202C70347000F0BFFF00F037
:109A900015FF33782000002B04D028780138444289
:109AA0006041C0B204B070BD411300207FB56B4669
:109AB000DC1D1C4B20701878002801D100F078FEC6
:109AC000002000F05DFE00F0D1FE0121392001F000
:109AD0007FF801220E250F2620000024110000F03F
:109AE00039FF6E4400F016FF6D4400F013FF00F0E4
:109AF000E5FE002000F044FE00F0B8FE3200290030
:109B000039202C70347000F081FF00F0D7FE3378DC
:109B10002000A34204D02878013844426041C0B2FA
:109B200004B070BD411300207FB56B46DC1D1E4B99
:109B3000207018780E001500002801D100F038FEC2
:109B4000002000F01DFE00F091FE0221442001F0F3
:109B50003FF800220121200001F013F8300001221B
:109B6000290001F00EF803262C0009343440013599
:109B7000002C02D000F0CEFEF6E700F09FFE0E258E
:109B8000200000F0FDFD00F071FE0D226D446A44DE
:109B90002900442014702C8000F038FF00F08EFE65
:109BA000288804B070BDC04641130020F0B50E25D2
:109BB00085B00F2700246B4601266D446F44D87191
:109BC0002C703C701E4B1878002801D100F0F0FD7D
:109BD000002000F0D5FD00F049FE31002A2000F001
:109BE000F7FF6B4632003100D81D00F0B3FE00F0E5
:109BF00091FE00F08FFE00F061FE002000F0C0FD3D
:109C000000F034FE3B002A0031002A2000F0CAFE9A
:109C100000F054FE2B78002B0FD101346420A4B245
:109C200003F0FAFC2B78002B01D1182CCAD9193C6F
:109C3000601E8441E0B205B0F0BD0024F2E7C046EA
:109C400041130020134B13B51878002801D100F000
:109C5000AFFD002000F094FD00F008FE00213F2041
:109C600000F0B6FF00F02AFE002000F089FD00F0B1
:109C7000FDFD6B469C1DFF2323706B4600220733BE
:109C80001A70012122003F2000F08CFE00F016FE29
:109C9000207816BD41130020F7B51D00234B0700A7
:109CA00018780C001600002801D100F081FD00207A
:109CB00000F066FD00F0DAFD0421682000F088FF66
:109CC0000022A1B2380000F05CFF30000326002122
:109CD00000F06CFF0021280000F068FF099B0122C2
:109CE00099B2089800F04DFF099B0A34E41825004A
:109CF000354003D000F00EFE0134F8E700F0DEFD41
:109D0000280000F03DFD00F0B1FD6B4601219C1DD7
:109D10009D71220007336820197000F043FE00F0A7
:109D2000CDFD207843425841C0B2FEBD4113002012
:109D3000124B07B51878002801D100F039FD00203A
:109D400000F01EFD00F092FD0021692000F040FFB0
:109D500000F0B4FD002000F013FD00F087FD6B461D
:109D6000002203331A700192012101AA692000F038
:109D700019FE00F0A3FD01980EBDC046411300205E
:109D800070B586B0050014000E000B22002102A859
:109D900006F061FD09232A0A6B441D705A702A0CD3
:109DA0002D0E9A70DD700E236B441E80360C5E8083
:109DB0001323220A6B441C705A70220C240E9A70D2
:109DC000DC70154B1878002801D100F0F1FC002060
:109DD00000F0D6FC00F04AFD2120012100F0F8FE41
:109DE0006B460122D81DFF231100037000F0B2FD65
:109DF00000F090FD00F08EFD00F060FD002000F00E
:109E0000BFFC00F033FD02AA0321212000F02DFE4B
:109E100000F054FD06B070BD4113002070B586B04F
:109E20006B46DE1D0C00150030700622002103A8D1
:109E300006F011FD0D23220A6B441C705A70220C8F
:109E4000240E9A70DC7012236B441D802D0C5D80F3
:109E5000134B1878002801D100F0AAFC002000F074
:109E60008FFC00F003FD01213A2000F0B1FE012239
:109E70003000110000F06EFD00F04CFD00F04AFDD6
:109E800000F01CFD002000F07BFC00F0EFFC03AABA
:109E900002213A2000F0E9FD00F010FD06B070BD8F
:109EA00041130020F7B51D001F4B070018780C0068
:109EB0001600002801D100F07BFC002000F060FCBF
:109EC00000F0D4FC0221112000F082FE21000022CB
:109ED000380000F03FFD30000122290000F03AFD7B
:109EE0000326063464192500354003D000F012FD26
:109EF0000134F8E700F0E2FC280000F041FC00F03B
:109F0000B5FC6B469C1D22000733012111202570F2
:109F10001D7000F047FD002801D1FF23237000F0E1
:109F2000CDFC00202056FEBD4113002010B50F24AB
:109F300086B00093234B6C442070187802910192F4
:109F4000002801D100F034FC002000F019FC00F0E2
:109F50008DFC0421142000F03BFE20000022012192
:109F600000F0F8FC0022042102A800F0F3FC00221B
:109F7000042101A800F0EEFC01220421684600F053
:109F8000E9FC00F0C7FC00F0C5FC00F0C3FC00F0E9
:109F900095FC002000F0F4FB162400F067FC17236A
:109FA00000226C446B4422701A700121220014209C
:109FB00000F0F8FC002801D1FF23237000F07EFCA4
:109FC00006B010BD4113002010B50F2486B01E4B03
:109FD0006C442070187802910192002801D100F0A1
:109FE000E7FB002000F0CCFB00F040FC0321152033
:109FF00000F0EEFD20000022012100F0ABFC002269
:10A00000042102A800F0A6FC0122042101A800F00E
:10A01000A1FC00F053FC002000F0B2FB162400F07D
:10A0200025FC172300226C446B4422701A70012116
:10A030002200152000F0B6FC002801D1FF23237078
:10A0400000F03CFC06B010BD411300201E4B73B560
:10A0500004001878002801D100F0AAFB002000F0CD
:10A060008FFB00F003FC0121162000F0B1FD200061
:10A0700007F05CF90122C1B2200000F06BFC200067
:10A0800007F054F90326441D2500354003D000F0A5
:10A0900041FC0134F8E700F011FC280000F070FBEF
:10A0A00000F0E4FB6B469C1D9D71220007330121EB
:10A0B00016201D7000F076FC002801D1FF232370CC
:10A0C00000F0FCFB73BDC04641130020134B13B5D9
:10A0D0001878002801D100F06BFB002000F050FB45
:10A0E00000F0C4FB0021202000F072FD00F0E6FB30
:10A0F000002000F045FB00F0B9FB6B469C1DFF23E0
:10A1000023706B46002207331A70012122002020A1
:10A1100000F048FC00F0D2FB207816BD411300206F
:10A12000184B13B51878002801D100F041FB00202E
:10A1300000F026FB00F09AFB2220012100F048FDF0
:10A140006B460122981DFF231100037000F002FCF2
:10A1500000F0E0FB00F0DEFB00F0B0FB002000F0C0
:10A160000FFB00F083FB6B460022074C07331A708D
:10A1700001212200222000F015FC00F09FFB2000AE
:10A1800016BDC04641130020D00E002070B505005A
:10A19000054C064A20000649FFF7F2FD2800210081
:10A1A00002F07AFC70BDC046D60E0020C80E00201A
:10A1B000CC0E0020204B73B504001878002801D184
:10A1C00000F0F6FA002000F0DBFA00F04FFB01216E
:10A1D000342000F0FDFC200007F0A8F80122C1B2F5
:10A1E000200000F0B7FB200007F0A0F80326441D74
:10A1F0002500354003D000F08DFB0134F8E700F076
:10A200005DFB280000F0BCFA00F030FB6B469E1DA1
:10A210009D7132000733012134201D7000F0C2FB14
:10A22000C4B200F04BFB002C04D03478013C6042F7
:10A230004441E4B2200076BD41130020FF2130B537
:10A240008BB00B00050000910A0004A802F0F2FB9D
:10A25000184B1878002801D100F0AAFA002000F06D
:10A260008FFA00F003FB0021352000F0B1FC00F074
:10A2700025FB002000F084FA00F0F8FA0B230022FE
:10A280006B441A70012103AA352000F08BFB041ED9
:10A290000AD003A9280002F0FFFB04A9280002F05D
:10A2A0000CFC01244440E4B200F008FB20000BB099
:10A2B00030BDC0464113002010B50C00FFF77AFFF7
:10A2C00003000020834202D02000FFF7B7FF10BD3B
:10A2D000F7B51E00224B070018780D001400002867
:10A2E00001D100F065FA002000F04AFA00F0BEFA51
:10A2F0000321192000F06CFC00222900380000F036
:10A3000029FB31002000002200F024FB012208A8D4
:10A3100011002C1DA41900F01DFB0326250035405B
:10A3200003D000F0F7FA0134F8E700F0C7FA28008C
:10A3300000F026FA00F09AFA6B469C1D22000733C3
:10A340000121192025701D7000F02CFB002801D17F
:10A35000FF23237000F0B2FA00202056FEBDC04655
:10A360004113002010B5054A0549064800F010F8D1
:10A370000022054B05491A705A5410BD0104000013
:10A38000003D0100E0120020DA0E0020020400006F
:10A3900030B5094D094CAB685B035B0F9B001C5942
:10A3A0000460AB6801619BB243606343A4008360B7
:10A3B000C460426130BDC04600400041004201001F
:10A3C000F7B580261A4D01916F6803333E439B0811
:10A3D0006E60002B2BD0174E2E802E7DF107FCD502
:10A3E0001E000768991BBF088F4219D9002E17D08D
:10A3F000FF2117788C433C430F4957780C403F02AC
:10A400003C439778013E39040C4F2740D478BFB2C3
:10A410000F43240601993C4310C101910432E0E747
:10A42000074B2B802B7DDB07FCD53300D1E7F7BD35
:10A430000040004144A5FFFFFF00FFFFFFFF00FFBA
:10A4400004A5FFFF044B054A4908D9611A801A7D0B
:10A45000D207FCD57047C0460040004102A5FFFF6F
:10A4600070B504000D001600E36829002000B34217
:10A4700005D2FFF7E7FFE368ED18F61AF4E7FFF7F8
:10A48000E1FF70BD10B510001A0006F0C8F910BD4C
:10A4900070B506000C008D18AC4207D033682178E7
:10A4A0009B683000984720700134F5E770BD704715
:10A4B000704710B50400406800F0D0FC00232376FC
:10A4C00010BD10B5406800F0EEFC10BDF8B50500F9
:10A4D00040680C0000F0E2FC2B68E7B2260A9B689B
:10A4E000012810D139002800FF2798472B68BC436A
:10A4F00004439B683100280098470302200038403D
:10A50000184380B2F8BD310028009847FF262B6819
:10A510000002344004439B68390028009847B44344
:10A520002043EEE710B5040003F036F9200010BD1B
:10A5300010B54B1C0BD0102909D0EFF3108472B664
:10A54000102905DD02234376002C00D162B610BD30
:10A550000123427E1A43427618224A43044989184D
:10A5600016228A569340C2691343C361ECE7C04682
:10A57000604201004B1C17D0102915D0437E9B0769
:10A5800012D4EFF3108272B618234B430749C9184F
:10A590000123897D49B28B40C1699943C16100D1D2
:10A5A0004176002A00D162B67047C0466042010081
:10A5B000437E002B05D09A0704D5837E002B00D064
:10A5C00062B67047DB07FCD5C369024A9BB2D36011
:10A5D000F7E7C04600180040037E002B04D1437605
:10A5E0008376C36101330376704700007FB503694A
:10A5F00002AE04000D00029172608B4203D1828A88
:10A60000B3889A4226D0200006223100103006F08E
:10A6100006F9606800F039FC7379E17A013B581E55
:10A620008341227B00936068002300F0D3FC3379E0
:10A630000021013BDBB2022B01D8074AD15C074B5A
:10A640002A009D4200D91A00606800F0EFFB6068A4
:10A6500000F011FC7FBDC04620420100001BB70086
:10A6600070B518260400FFF7B7FF33000821207AE1
:10A670000D4D4343EB18595603F00EFB33000821F0
:10A68000A07A4343EB18595603F006FB0821607A81
:10A690004643AD19695603F0FFFA044B200006CB80
:10A6A000FFF7A4FF70BDC0466042010038130020D0
:10A6B00007B5437E00910192002B07D09A070AD577
:10A6C000EFF310835A425341837672B60099019A90
:10A6D000FFF78CFF07BDDB07F8D5C369014A9BB2C2
:10A6E0009360F3E700180040F7B500240125194BEB
:10A6F000194A5D711A601C71184B1948083301938F
:10A700000360184B184F4360184B194E03810D23FB
:10A710003A00310045750461047583720A3B047682
:10A72000C472037303F066FB1248134B019A436033
:10A73000124B4575038119233100026004613A0010
:10A7400004758372163B05730476C37203F052FBE3
:10A75000F7BDC0463813002000093D002442010027
:10A76000F8120020181A0020000000200C0B000036
:10A77000B1A4000018130020201A002017160000B2
:10A7800010B5040002F012FF044B187803F06CFAC5
:10A79000002802D0002CF7D0F4E710BD2D000020D7
:10A7A00010B51A2003F060FA431E984110BD000056
:10A7B000F8B5274B1B78002B01D0002847D0182371
:10A7C000244E254F3370254C04333B70013B2370DE
:10A7D00000F011FA224D1A2804D801232B70237897
:10A7E000DB4323703078012103F0C6F9387800216B
:10A7F00003F0C2F92078012103F0BEF901211A20EB
:10A8000003F0BAF901211A2003F002FA307801218D
:10A8100003F0FEF92978207803F0FAF90A2002F013
:10A82000FBFE297801252078694003F0F1F90D48F5
:10A8300002F0F2FE00211A2003F0EAF900211A20AA
:10A8400003F09AF90848FFF70BFF014B1D70F8BDA4
:10A85000411300202F0000202D0000202E0000209A
:10A8600040130020EE0200001813002013B500244E
:10A870006B466A461C7101235371019A0B490C48BF
:10A88000FFF716FF0B4B2100187803F0C1F902F017
:10A890008DFE0400084B187803F0E6F9012804D077
:10A8A00002F084FE001B0428F4D913BD00127A00C4
:10A8B000181300202F0000202D00002010B5044B9D
:10A8C0000121187803F0A4F90248FFF771FE10BDCA
:10A8D0002F0000201813002007B56B46D871D979D6
:10A8E0000248C9B2FFF7EDFD0EBDC04618130020A7
:10A8F00010B50400FF20FFF7EFFF207010BD70B50A
:10A900000C0005000800FFF7F3FF2078401B4342CE
:10A91000584170BD13B56B46DC1D00232000237029
:10A92000FFF7E6FF207816BD70B50500084CFFF76D
:10A93000F1FFEF2808D0013C002C01D0A842F6D14D
:10A94000401B4342584170BD01204042FBE7C046D6
:10A95000E9030000F8B5050008000E0017002C0000
:10A96000FFF7BAFF631B9E4204DD2078FFF7B4FFB8
:10A970000134F7E7012F02D1EE20FFF7ADFFF8BD5C
:10A9800010B50400000AFFF7A7FFE0B2FFF7A4FF2D
:10A9900010BD10B50400FF20FFF79EFF002C00D073
:10A9A000207010BDF0B585B01F0002ABDC1D002388
:10A9B0000500E020019116002370FFF7B5FF002885
:10A9C00002D1002005B0F0BD2000FFF791FF8022EA
:10A9D00023781543AB42F4D12000FFF789FF237899
:10A9E000019A9342EDD13800FFF7D3FF35003A7852
:10A9F000AB1B9A4204DD2800FFF77AFF0135F6E72A
:10AA00002100EE20FFF77BFF0120DBE7F7B56B4667
:10AA1000DC1D00230500E0200E0017002370FFF767
:10AA200083FF002801D10020FEBD2000FFF760FF5A
:10AA3000802223781543AB42F5D1FFF76BFF002846
:10AA40000DD03800FFF7A5FF35003A78AB1B9A42CE
:10AA500005DDFF20FFF740FF28700135F5E72100F5
:10AA6000EE20FFF74CFF0120DEE7F0B587B004AB26
:10AA7000DE1D00230500E020039114003370FFF772
:10AA800053FF002802D1002007B0F0BD3000FFF7CF
:10AA90002FFF802233781543AB42F4D1FFF73AFF02
:10AAA00001900028EFD005234343E3180293029B53
:10AAB0009C421AD0FF20FFF70FFF00272070237859
:10AAC000BB4210DDA37865781B022B43E578FF209D
:10AAD0002D042B4325792D061D43FFF7FDFEED19AF
:10AAE00028700137EBE70534E1E7019B039A9342B5
:10AAF000C9D13100EE20FFF702FF0120C4E770B595
:10AB00000500FF20FFF7E8FE0400FF20FFF7E4FE4A
:10AB10002402204380B2002D00D0288070BDF0B503
:10AB2000002485B002AB0700DD1DE0200191160076
:10AB30002C70FFF7F9FEA04202D1002005B0F0BD55
:10AB40002800FFF7D5FE80222B781743BB42F4D1B3
:10AB5000FFF7E0FE00280ED03000FFF7D0FF33886B
:10AB6000A34208D9019BFF201F19FFF7B5FE01344E
:10AB70003870A4B2F3E72900EE20FFF7C0FE0120F1
:10AB8000DCE770B504000D0008001600FFF7F8FEC2
:10AB90006519AC4204D02078FFF79EFE0134F8E737
:10ABA000012E02D1EE20FFF797FE70BD70B50400B4
:10ABB00002200D00FFF790FE200AFFF78DFEE0B2A5
:10ABC000FFF78AFE012D02D1EE20FFF785FE70BD52
:10ABD00070B50400E0200D00FFF77EFE7F202040CE
:10ABE000FFF77AFE2800FFF777FE002D02D1EE2056
:10ABF000FFF772FE70BD2120704710B501211A20A9
:10AC000002F0BAFF01211A2003F002F801211B20F3
:10AC100002F0B2FF00211B2002F0FAFF10BD00007D
:10AC200010B5024801F077FD10BDC0464413002066
:10AC300010B5024801F06FFD10BDC0468815002018
:10AC400010B5024801F067FD10BDC046CC170020CA
:10AC5000F0B51F4985B01F4800F058F81E491F483D
:10AC600000F054F81E4D1F49280000F04FF81E4E0A
:10AC70001E49300000F04AF81D491E4800F046F811
:10AC80001D4F1E49380000F041F80124032339000C
:10AC90000093019423000022194801F0B5FC002321
:10ACA0003100019300941D331E22164801F0ACFCC4
:10ACB00019230393013B0293163B01930094143331
:10ACC00017222900104801F05BFC05B0F0BDC0461A
:10ACD00000080042101A0020000C0042181A002040
:10ACE000201A002000100042281A00200014004200
:10ACF00000180042301A0020381A0020001C0042C0
:10AD00004413002088150020CC1700200023037175
:10AD1000016070479446F0B59E1E721E96416246D1
:10AD2000056892072F6836063A4332432A600725A2
:10AD300005AC24780068A40129402143426800241E
:10AD4000022B00D05C03114321434160F0BD30B5BC
:10AD5000C0250368AD031C6812052A402243C024A5
:10AD60000904A40221401143196003685A6814437E
:10AD70005C6030BD0123026811680B4313600368F7
:10AD80001A68D207FCD4DA69D207F9D470470223D3
:10AD9000026811680B4313600268D3699B07FCD4F7
:10ADA00070470268137E9B0702D40379002BF9D108
:10ADB000002303717047002203685A8370470368B9
:10ADC000187E4007C00F70470368187EC00970479F
:10ADD000802302685B42117E0B4313767047036841
:10ADE000588B8007C00F704702230268518B0B43BA
:10ADF000538370470368187EC007C00F704703680D
:10AE0000188DC0B2704703681A7ED207FCD589B28C
:10AE100019850123037118007047012203689A7590
:10AE20007047012203681A757047000070B501264B
:10AE300004684B0833403140256809075B070B4322
:10AE40002B43236004685100034802F0E5FF0138FA
:10AE5000C0B2207370BDC046006CDC0201230268E2
:10AE600011680B43136003681A68D207FCD4DA69CF
:10AE7000D207F9D470470223026811680B431360AC
:10AE80000268D3699B07FCD470470368DA699207AC
:10AE9000FCD402211A688A431A6070470368186854
:10AEA0004000C00F70470268936A5B0A5B02194357
:10AEB000916203681A7E5207FCD5986AC0B2704747
:10AEC0000368214A30B593422FD0204A93422FD0B5
:10AED0001F4A93422FD01F4A93422FD01E4A9342BB
:10AEE0002FD01E4A93421FD10E2319220121032580
:10AEF00099401B48C024016099082B40AB40FC35A9
:10AF00009D4089000918A4000859A843C0259D4008
:10AF10002B0003430B518023DB011A43114B5A8052
:10AF20005A7852B2002AFBDB30BD09231422DDE738
:10AF30000A231522DAE70B231622D7E70C23172260
:10AF4000D4E70D231822D1E700080042000C00428C
:10AF5000001000420014004200180042001C004291
:10AF600000E100E0000C0040F8B504000F001600FE
:10AF70001D00FFF7A5FF2000FFF7FCFE1C21BB0012
:10AF80000B4071072268090C0B431360842322686D
:10AF90009375012F1AD11021012E00D008390C4BC6
:10AFA00069431868C00002F037FF07222168024099
:10AFB0008B895203DB04DB0C13438B81226803046F
:10AFC0009089DB0C400B400318439081F8BDC046CC
:10AFD00038000020F7B50600019308AB1F780D007C
:10AFE0001400FFF73BFF3000FFF76AFFC022240583
:10AFF00092031440BA070C2717433C43C02707228B
:10B00000BF022D0433683D4025431D60019B31681C
:10B0100013401A0080239B0213434B60F7BD0020AE
:10B02000704770B50F26CB1D013902003240D5B2F2
:10B030002C0000093034092A00DD07341C70013B64
:10B040008B42F2D170BD000010B50C000B4B18689C
:10B05000FFF7E7FF21000A4B08311868FFF7E1FF0F
:10B060002100084B10311868FFF7DBFF2100064B69
:10B0700018311868FFF7D5FF202010BD0CA0800004
:10B0800040A0800044A0800048A0800008B4024B8B
:10B090009C46103808BC604749B0000070477047B4
:10B0A0003F20704713B56B460268D9710733546867
:10B0B00019000122A04716BD70B50A260B7892B080
:10B0C0006E44023305000B703C220021300005F075
:10B0D000C2FB394801AC069038482421079006206D
:10B0E00020776846364AA1742281364A364BA281BF
:10B0F000FD3AFF3A8018C177684623390630C17798
:10B1000068460730C17702A8C1770720F277032687
:10B1100008316944C87703A9CE7710212B366E44D5
:10B120003170092621851F3169440E700CA9053E36
:10B130000E7033212380022369440B7006360DA95B
:10B140000E7022493536A1863B216E44307010A81E
:10B150006274E27702703D3269446A440B70137086
:10B1600040210022E37023716371A37341336B4468
:10B17000218719705A702B7DC039A370A372637731
:10B180000133DBB2A3776A7D0B200D0068441543C1
:10B19000C5773120684403703A23501C6B44187003
:10B1A000412302320A436B441A70210042220848AC
:10B1B00000F004FD12B070BD100104240206052445
:10B1C0000904000001020000080B00000705000050
:10B1D000A41A002008B4024B9C46103808BC6047F3
:10B1E000B9B00000F8B5027D0B7904000D0000270E
:10B1F0009A420CD10B784E78A12B0AD1212E06D180
:10B200000100072234311C4800F0D8FC0137380017
:10B21000F8BD212BFBD1202E23D101000722343190
:10B22000154800F00DFC9623626BDB009A421FD19B
:10B230003B342378DB071BD4FA2002F08DFD00217C
:10B240000D4800F0D9FD0127232EE0D1EB78AA7834
:10B250001B021343094A00210748136000F0CCFD8C
:10B26000D5E7222EEFD103008A783B331A70DAE754
:10B2700002F07CFDE3E7C046A41A00203000002065
:10B2800008B4024B9C46103808BC6047E5B100008A
:10B2900010B534300822002105F0DDFA10BD0000A1
:10B2A00010B5417D006A013100F002FB034B1B68C1
:10B2B00001335A1E9341181810BDC04634000020B7
:10B2C00010B5417D006A023100F008FB10BD10B5D9
:10B2D000417D006A023100F0CFFA10BD70B50D005B
:10B2E000417D0400130002312A00006A00F0BCFB1B
:10B2F000002801D10123636070BD000010B5054C2A
:10B3000023685A1C04D103685B69984703002060D6
:10B31000180010BD34000020074A0300106810B563
:10B32000411C03D001235B42136010BD597D186A94
:10B33000013100F049FBF8E73400002070B505004A
:10B3400002F034F9F423FF330024984207D93B3547
:10B350002C780A20631E9C41E4B202F05DF92000C3
:10B3600070BD00207047704770470000FA239B00B3
:10B3700010B58360114B0022C38203002833836120
:10B380000F4B04004260C261180050332361083043
:10B39000631D21622060DA770A4A2F3303CA03C390
:10B3A0008323A362813BE3628033236301F022FCA9
:10B3B0002100103101F0EFFB200010BD030200005E
:10B3C0008045010078450100022110B5094B1A683B
:10B3D000437D5B01D318FF339C7A21439972437DEF
:10B3E0000133DBB25B01D3180122FF33997A0A43A0
:10B3F0009A7210BD5C1F002010B502490248FFF789
:10B40000B5FF10BDA41A0020401A0020704710B5E7
:10B41000040002F0C1F9200010BD0000F0B582293F
:10B4200019D1C3B2294D5A01AA189169284C80013B
:10B430000C40C021890521439161264908334018F9
:10B440007021506128685B011A5C8A431100302228
:10B450000A431A54F0BD0029FCD1C026C1B21B4CCE
:10B460004B01E3189A681A4DB6052A4032439A6098
:10B47000194A800182185A600A0007272468083296
:10B480005201115DB9430F000121394311559F69E4
:10B4900010493D4040182E439E6158617020115D57
:10B4A0008143080010210143115599680B48A218E7
:10B4B000084080214903014399609968890B8903F9
:10B4C0009960402311790B431371C3E75C1F00207F
:10B4D000FFFFFF8FD01A0020901C0020FF3F00F0DC
:10B4E000EFF3108303600123436072B67047036873
:10B4F000002B02D162B6BFF36F8F704773B5836DB7
:10B500000400002B1BD10600A83635786846FFF7EB
:10B51000E7FF019BEDB2013B02D33578EDB2FAE7CC
:10B5200068460193FFF7E3FF002D01D1002076BDAF
:10B530002300A4331868A0342368C01AF7E76846CC
:10B54000FFF7CEFF22000025019BF432013B02D31E
:10B550001578EDB2FAE768460193FFF7C8FF002DB2
:10B56000E4D02300F0331868EC34E5E710B5436D00
:10B570004468DBB25A01A2189168094808330840B0
:10B58000802149030143916091685B01890B890324
:10B5900091602268D318402219790A431A7110BDAC
:10B5A000FF3F00F0F7B5436D4268DBB219000400BD
:10B5B0000831106849014118C979C90711D55B01E3
:10B5C000D21893689B049B0C0CD12000FFF7CEFF90
:10B5D00063681A68636DDBB208335B01D3187F229E
:10B5E000DA71F7BDE16D002923D12100A4310B6090
:10B5F00023000125AC33E56568465360FFF770FF13
:10B60000260020002100019BA836013BF430F531D3
:10B610005A1C33D0357002785F1ED2B20A700A7895
:10B62000002A04D120000193FFF7A0FFE8E73B00C8
:10B63000EEE72100F0310B600023E3652300603367
:10B6400053606846FFF74CFF0125260020002100CB
:10B65000019BF436013BA830F5315A1C0ED03570F1
:10B6600002785F1ED2B20A700A78002A04D1200044
:10B670000193FFF77BFFE8E73B00EEE768460193A5
:10B68000FFF735FFA4E737B56B46DC1D00230D003F
:10B69000237001F0AFFA210001F03AFA2B68181874
:10B6A000286020783EBD00000078002810D00121DD
:10B6B000084B1B681A898A431A810822198B0A438E
:10B6C0001A830422198B0A431A830022024B1A6040
:10B6D0007047C0465C1F0020541F002010B50F4A61
:10B6E00093699B0B9B03936113680222FF331A72C9
:10B6F0009879823A02439A711A7A9207FCD57F248C
:10B70000074A2140937A0800A3431900802301438C
:10B710009172917A5B420B43937210BD5C1F0020C3
:10B720000050004110B50C0001F064FA210001F056
:10B7300022FA002804D1034A93699B0B9B0393616F
:10B7400010BDC0465C1F0020F8B50D00832A19D13A
:10B75000CBB23B4C5A01A21891693A48AD0108405E
:10B76000C021890501439161374920686D18702116
:10B77000083355615B011A5C8A43110040220A4379
:10B780001A54F8BD022A55D1304A8B009858002827
:10B7900002D003685B699847F82001F0F9FF0400C4
:10B7A000274E2B4B4660036040220021083005F0F5
:10B7B00052F822000023A032A3646565E364236588
:10B7C000A365E3655360D3641372136013654C3251
:10B7D00013725372FF222B001340590171188868AD
:10B7E000184F08330740C020800538438860306810
:10B7F00007265B01195CAD00B1430E000321314304
:10B8000019542300616D606811404901411860338B
:10B810004B60616D63680A401B6852019B180122EE
:10B82000FF33997A20000A439A72FFF79FFE074B75
:10B830005C51A6E711002800FFF7F0FDA1E7C04624
:10B840005C1F0020FFFFFF8FD01A0020A81A0020E5
:10B85000E845010070B505000124064BA200D2584E
:10B86000002A06D0210028000134FFF76DFF0A2CC2
:10B87000F3D170BD7C1A00200B4BCAB20B48890172
:10B88000C9185301C318596199690832890B890392
:10B890009961036852019A180223D3715179823B4E
:10B8A0000B4353717047C046D01A00205C1F002024
:10B8B000084B8A00D05810B5002803D003689B6855
:10B8C000984710BDC9B2044B4901591888688004D3
:10B8D000800CF6E7A81A00205C1F002010B50C00B1
:10B8E000FFF7E6FF00280CD0064BE4B21B680834D3
:10B8F00064011C19802362795B4213436371022344
:10B90000E37110BD5C1F0020F0B51C002A4B85B010
:10B910001B6807000D000292002B4AD0274B8A00BB
:10B92000D058002808D0036822005B680299984725
:10B930000400200005B0F0BD3800FFF7B9FF8442D5
:10B9400004D929003800FFF7B3FF04000121EBB24E
:10B950001B4E03935B010193F21893689B0B9B03AF
:10B960009360019A336802989B18FF335A7A0A430E
:10B970005A72144BA901C918220004F050FF002C80
:10B98000D7D029003800FFF793FF0028D1D14021FC
:10B99000039B326808335B01D3181879014319718E
:10B9A0000121D971019BD318FF339A7A0A439A7205
:10B9B000BFE701246442BCE7541F0020A81A0020FE
:10B9C0005C1F0020901C002013B56B46DC1D22007C
:10B9D0000123FFF799FF012801D1207816BD01202E
:10B9E0004042FBE770B5CBB2124A13485C018901B3
:10B9F0008918021951609168104D08330D4080215B
:10BA000049032943402591609168890B890391601E
:10BA100001685A018A1816793543157195796D06B2
:10BA2000FCD55B01C918CB79DB07FCD50019806810
:10BA3000C0B270BD901C00205C1F0020FF3F00F0D2
:10BA400070B50D0000211400FFF7CCFFA04200D913
:10BA5000200000230349A34203D0CA5CEA54013307
:10BA6000F9E770BD901C0020F0B51E003A4B85B080
:10BA70001B680F000192002B35D08023DB019E4212
:10BA800031D80025354B8A01D3180293002E2CD0D3
:10BA9000334B1B680393FF233B401C000093083487
:10BAA000039B64011C19A379DB0921D02D4B2E497E
:10BAB000186802F0B1F92D4B1721584302F0ACF988
:10BAC0002B4BE279920713D4DA5D002A01D10138B9
:10BAD000F7D20122DA55009B5A01214B9B189A6933
:10BAE000920B92039A6101256D42280005B0F0BDCA
:10BAF00000221F4B3400DA553F2E09D9009B402409
:10BB00005A01174B9B188022996912060A439A61C1
:10BB100022000199029804F082FE009BA1045A01C0
:10BB20000F4B890C9B18029A2D195A619A69361B82
:10BB3000920B92030A439A61009B039A08335B01BC
:10BB4000D3180222DA715979823A0A435A71019B59
:10BB50001B1901939AE7C046541F0020D01A0020F9
:10BB60005C1F00203800002040420F0070110100CF
:10BB7000C51A002070B50D001C000D4BAE01F61863
:10BB800011003000220004F04AFEEDB209496D01B7
:10BB90004D196E61AB69084A20001340AB61AB6977
:10BBA000A2049B0B920C9B031343AB6170BDC04678
:10BBB000D01A00205C1F0020FF3F00F0F7B5104BAB
:10BBC00001901B780F001500002B0CD10D4B1600B7
:10BBD0001C78002C09D00C4E0C48348820186419AD
:10BBE00004F01DFE34802800FEBD002EFBD03A1963
:10BBF000330000210198FFF7BDFF2418361AF4E73F
:10BC0000501E0020511F0020521F0020511E0020F6
:10BC1000F8B50F0016000024012A26D9100004F000
:10BC2000C9FD0500380005F081FB03230222013025
:10BC3000400028706B7096420DD9397800290AD0DF
:10BC4000531CDBB20137A9549E4203D00232EC549C
:10BC5000D2B2F0E7320029000548FFF7AFFF441EDB
:10BC6000A041C4B2280004F0AFFD2000F8BDC046DA
:10BC7000A41A0020F0B50024012685B0184B0F004F
:10BC800069461E7005000094FFF7FDFC154B01A9E5
:10BC90000B806A3BFF3BCB715A330B72009B8C715C
:10BCA00009334B800E4B4E7108711C703A00092FFE
:10BCB0000FD00D4F09223E700C4E280000943480A6
:10BCC000FFF77CFF69462800FFF7DDFC3288084952
:10BCD0003C702800FFF772FF012005B0F0BDC046A0
:10BCE000501E002009020000511F0020521F00209A
:10BCF000511E002070B5CE7892B005000C00022EC7
:10BD00000BD18B79C9792C4809021943FFF7B2FF8F
:10BD1000411E8841C0B212B070BD00F06BFF21001F
:10BD200000F00AFF002803D0C117081AC00FF2E77D
:10BD3000012E0ED1E279A37912021A431F49112A6A
:10BD400013D8D2B2002A10D02800FFF737FF012005
:10BD5000E1E7032EDFD1A378002B08D1E279A379A4
:10BD600012021A431649032AEBD90A78ECE7022B90
:10BD700008D1E279A379120212491A432800FFF789
:10BD800047FFC8E7012B05D1E279A37912021A43D4
:10BD90000D49F3E7032BBED14122010001A804F0B5
:10BDA0005AFD00F027FF01A900F0D6FEE279A37941
:10BDB00012021A4301A9E1E7A41A00202846010053
:10BDC00018460100044601001C46010010B5074A50
:10BDD000074B002904D00121117000221A8010BDE8
:10BDE00011701A880349FFF7E9FEF8E7511F002098
:10BDF000521F0020511E0020CBB204495B01C9181C
:10BE00008B699B0B9B038B617047C0465C1F0020B6
:10BE100037B5050048780C000B2810D801F0F2FF68
:10BE2000061B0F2B0F404561494C5A5D097801AA4A
:10BE3000002906D1022311802800FFF79BFE012074
:10BE40003EBD00231380284B1B78012B00D11370BB
:10BE500002230021F0E78A780023012A03D101AAF6
:10BE60001380224BF0E7204A1370214A93699B0B01
:10BE70009B039361E3E78C78012C06D100211B4BD7
:10BE800001AA1C7011702300D6E70120002CD7D125
:10BE9000154B174A187093699B0B9B039361CFE76F
:10BEA00089782800FFF71AFCC9E72800FFF722FF6E
:10BEB000C6E701230F4ACCE70B780020DB06BFD191
:10BEC0002800FFF7C7FCA2780A4B0B481A60FFF75F
:10BED0007BFACAE70123094ABBE78A78074B1A6055
:10BEE000C3E70020ACE7C046C41A0020CC1A0020EB
:10BEF0005C1F0020541F0020401A0020581F002003
:10BF00003A4BF7B51E780500002E5FD1384C2368F8
:10BF10009A8B12070DD5082231009A833000FFF763
:10BF20007DFA10222368FF33997A0A439A72314BC3
:10BF30001E6023689A8B520701D504229A83FF332F
:10BF40001A7A920603D52022597A0A435A721A7A2B
:10BF5000D20623D569460800274AC0CAC0C0A268D5
:10BF6000920B9203A2604022587902435A716023D7
:10BF70000A7828001A422AD1FFF74AFF2368FF33C4
:10BF8000002827D08022997952420A439A711A7A5E
:10BF9000520603D54022597A0A435A727F26012558
:10BFA0002368FF331E722F00236808377F01DB19D7
:10BFB000DB79002B07D0114BAA00D05800280DD0F8
:10BFC00003681B6898470135082DECD1F7BDFFF7D2
:10BFD000A9FBD3E720210A4A9171D8E72900094833
:10BFE000FFF7C2F92368DF19FE71ECE7511F00204B
:10BFF0005C1F0020541F0020901C0020A81A002065
:10C00000FF500041401A002010B50248FFF778FFAA
:10C0100010BDC046A41A002080235B0003800023CB
:10C02000436007330372704783000148C0187047AC
:10C030007C1A0020836C402B09D03F22036CC15432
:10C04000036C013313400364836C013383647047D2
:10C05000F7B505006846FFF743FA00264022019B2A
:10C06000013B02D32E6D961BFAE768460193FFF75A
:10C070003EFAAB6D6846002B4FD1FFF731FA29002D
:10C08000019BA831013B5A1C0CD00C785A1EE4B21B
:10C09000002C05D168460193FFF729FA2000FEBD68
:10C0A0001300F0E7684601930024FFF720FA2A0006
:10C0B0002900A0321368A431B4420ED00868984217
:10C0C0000BD92800591CEB1811606033197808301F
:10C0D000C9B2FFF7AFFF0134E9E709689942DDD142
:10C0E000002313600133AB656846FFF7F9F92F00B1
:10C0F0002A000021019BA837013BF532581CC9D00A
:10C10000397010785E1E002805D011702800019348
:10C11000FFF72CFAEBE73300F0E7FFF7E1F929002E
:10C12000019BF431013B5A1C06D00C785A1EE4B234
:10C13000002CAFD01300F6E7684601930024FFF708
:10C14000D6F92A002900EC321368F031B44202D04B
:10C15000086898421DD8096899429FD10023684613
:10C160001360AB65FFF7BCF92F002A000021019B8B
:10C17000F437013BF532581C00D18BE73970107849
:10C180005E1E002811D0117028000193FFF7EEF910
:10C19000EAE72800591CEB181160AC331978083015
:10C1A000C9B2FFF747FF0134CBE73300E3E710B52F
:10C1B0000400FFF74DFF206D10BD10B50400FFF720
:10C1C00047FF236D002B03D0E36CE418207A10BDE9
:10C1D00001204042FBE7F7B517000E000400FFF70F
:10C1E00037FF6846FFF77CF93F2200259446019B04
:10C1F000013B5A1C19D0BD4215D2226D002A12D023
:10C200000121226D4942002A0AD06046E26CA21840
:10C21000117AE26C01320240E264226D013A226539
:10C2200071550135E7E7013BE3E768460193FFF706
:10C230005EF92800FEBD0000014B024A1A607047FB
:10C240005C1F0020005000412023F7B5474A05003D
:10C25000D1690F200B43D361012245490B78134369
:10C260000B70444B19788143197006211C782143C7
:10C27000197041490C7822430A701A7802401A70EA
:10C28000602219780A431A703C4B3D4A5A805F7805
:10C29000FF09FCD13B4801F083F901233A4C3B4EA6
:10C2A0002268300011780B4313708022390052004D
:10C2B00004F0D1FA22689378DB07FCD456621F267B
:10C2C000334B1B68590B980C9B01314030405B0F7E
:10C2D000B14200D105211F2800D10238072B00D11F
:10C2E000043B31408901178D01912A4930400F40AC
:10C2F000019939431185118D0700B1430800384376
:10C300001085118D1803244B7F260B4003430C200E
:10C3100013850823D17881430B430321D37022680E
:10C32000D3788B4301390B43D370226813783340A1
:10C330001370042322681678334313702268C124D3
:10C340001389A40083431548138103591B021B0A58
:10C35000035180230360137811481943012311709E
:10C360002B700021FEF79AFEF7BDC0460004004086
:10C37000584400413C44004159440041000C0040F5
:10C380000640000009C000005C1F0020601F002064
:10C39000246080003FF8FFFFFF8FFFFF00E100E017
:10C3A000401A00200120704710B50368014A1B6A3B
:10C3B000984710BD13040000FC30006A70478723C3
:10C3C0009B00C018C36880204000C01A704703005B
:10C3D000FC331A6A002A03D0DB69C018007D70475D
:10C3E00001204042FBE710B504000069FEF7C2FCE3
:10C3F00022000023FC329361D361136287229200F2
:10C40000A4186360A360E36010BD872310B59B0090
:10C41000C218D368002BFCD10069FEF7C2FC10BD26
:10C42000F02001403039484248417047F0231B0159
:10C430001940802306209B0099420AD00133FF3324
:10C440000130994205D0802302385B00994200D028
:10C45000002070470F2001400020012903D002393D
:10C46000481E8141481C70478B23F0B5182685B0C3
:10C4700002919B000400C05C330008214343324D0D
:10C480001700EB18595601F007FC304B0821E05C0F
:10C4900033004343EB18595601F0FEFB2C4BE25C92
:10C4A0000393022A09D11133E05CFF2805D008214B
:10C4B0004643AE19715601F0EFFB8C26B600A05D25
:10C4C000FF2819D0012101F057FB1822A35D214953
:10C4D0005A43AB56AD18DB0158188D2189006050C6
:10C4E0001D4901225B188E218900635069688A40CA
:10C4F0008F21890062501A600122029B110020697D
:10C50000FEF732FD39002000FFF790FF39000500EB
:10C510002000FFF79FFF390006002000FFF780FF93
:10C5200033000090290020690122FEF7F3FB0B4B3A
:10C530002069E25C039BE15CFEF709FC2069FEF7E1
:10C5400026FC05B0F0BDC046604201002D0200008F
:10C550002F02000018440041144400412E02000044
:10C56000802210B504005200002104F074F9230069
:10C570000022FC335A6020009A60DA6010BD00008F
:10C58000F0B585B01D000AAB1B78040000930BAB1F
:10C590001B78160001930CAB1B780F0002930DABB8
:10C5A0001B78039300234360FA239B008360124BA4
:10C5B000083303601430FFF7D3FF20002130FF3031
:10C5C000FFF7CEFF8B236A469B002761E6540B4B97
:10C5D0001278E5540A4B2000E2546A46094B12795E
:10C5E000E2546A46127A0133E2546A46127B1033EF
:10C5F000E25405B0F0BDC0463C4601002D020000EB
:10C600002E0200002F020000F7B51D0008AB1B78BA
:10C610000400009309AB1B781600019300234360CC
:10C62000FA239B008360114B0F0008330360143022
:10C63000FFF796FF20002130FF30FFF791FF8B239B
:10C640006A469B002761E654094B1278E554094B72
:10C650002000E2546A46084B1279E2548C22313BA6
:10C66000FF3B9200A3541032A354FEBD3C46010090
:10C670002D0200002E0200002F020000F7B5EFF39C
:10C68000108300930123019372B680260200FF25D8
:10C69000019BFC327600013B5C1C0FD0D4685F1E0E
:10C6A000B44209D054680155546801342C40546098
:10C6B000D4680134D460EEE73B00EDE768460193AF
:10C6C000FEF715FFF7BD13B5EFF3108300930123B9
:10C6D000019372B6019B5A1E0192002B15D00300E4
:10C6E000FC33DA68002A0DD09A68845C9A680132BB
:10C6F000D2B29A60DA68013ADA606846FEF7F7FE6D
:10C70000200016BD01246442F7E701246846FEF7C5
:10C71000EEFE6442F4E710B504000069FEF75FFB2B
:10C72000002805D02069FEF76AFB2069FEF75CFB54
:10C730002069FEF744FB00281BD02069FEF75FFB51
:10C74000010020001430FFF799FF8C239B00E35C6D
:10C75000FF2B0ED02300FC331A6A80235B009B1A48
:10C76000092B06DC8D238F229B009200E358A258F0
:10C770001A602069FEF73EFB00280ED087239B003D
:10C78000E318DB68002B14D020002130FF30FFF7C6
:10C790009AFFC1B22069FEF736FB2069FEF714FB51
:10C7A000002805D02069FEF713FB2069FEF703FB84
:10C7B00010BD2069FEF735FBEFE70000F8B5040077
:10C7C00000690D00FEF716FB87239B00E618002882
:10C7D00002D0F368002B34D001278022F368520086
:10C7E000934223D1EFF310833B4210D1174B5B6888
:10C7F000DB05DB0DF1D0103B5BB2002B10DAF13A18
:10C800001340083B9B08124A9B009B181B68206939
:10C81000FEF7F0FA0028E0D02000FFF77CFFDCE70D
:10C820009B08C0330B4A9B009B58F0E72000213047
:10C83000FF302900FFF722FF2069FEF7EEFA012002
:10C84000F8BD29002069FEF7DEFAF8E700ED00E008
:10C850001CED00E000E100E010B504001430FFF72B
:10C8600032FF8C239B00E35CFF2B0ED02300FC33B4
:10C870001A6A80235B009B1A0A2B06DD8E238F2207
:10C880009B009200E358A2581A6010BD10B51C001E
:10C89000431A0298511A001B584301F047FB001934
:10C8A00010BDF0B589B00191037D0400012B00D0CB
:10C8B0008AE0021D029210000122049300235242DA
:10C8C0001C001500049E03920178002900D06EE040
:10C8D0004178002900D06AE0511C65D001335BB279
:10C8E00004998B4201DD049303920134E1B20230DA
:10C8F0004CB20829E8D100263700039BBB4204DC78
:10C90000049B039A9B18BB4253DC0F22029B1D78A9
:10C910002B111540029ADCB2527811110791694629
:10C92000097F05910F2111400691002B08D02100AD
:10C930005731092B00DC2739019800F0A5F936188A
:10C940002C4308D029005731092D00D827390198E8
:10C9500000F09AF93618059B1C430AD01900079B72
:10C960005731092B01DC05993031019800F08CF921
:10C9700036180699069B5731092B01D8190030311A
:10C98000019800F081F93618072F04D03A21019858
:10C9900000F07AF93618029B013702330293082F10
:10C9A000ABD1300009B0F0BD2200330098E72A0077
:10C9B0009BE7039BBB42EED1002BE7D13A210198C4
:10C9C00000F062F93618E1E7030005000026133392
:10C9D0001035029329780A22019800F0C3F92E211C
:10C9E0000700019800F050F9029B3F180135F61935
:10C9F0009D42EFD1E17C0A22019800F0B3F936188C
:10CA0000CFE7000010B50400054B01750833036043
:10CA100010220021043003F01EFF200010BDC0468C
:10CA20007046010010B504000021FFF7EBFF200065
:10CA300010BD0000F7B50F0000211D0008AB1B78EA
:10CA400004000193084B16000833036001750C22A3
:10CA5000043003F000FF6B461B7927746674A574DD
:10CA60002000E374FEBDC0467046010070B50D00A5
:10CA700000210400074B01750833036010220430C5
:10CA800003F0E9FE200029000422103003F0C7FE65
:10CA9000200070BD7046010070B50D00002104003B
:10CAA00001751022043003F0D6FE20002900042274
:10CAB000103003F0B4FE200070BD10B50A000C7DEC
:10CAC000017D00238C4207D1011D101D102203F0AF
:10CAD00097FE43424341DBB2180010BD037D002B9B
:10CAE00002D11031401870470431FBE707B501212E
:10CAF0000548FFF787FF0021044800910B000A005A
:10CB0000FFF798FF07BDC046602000207820002076
:10CB100070B50E0000254468002C0BD0236831004E
:10CB20005B6820009847002802DB2D18E468F3E7D3
:10CB300001256D42280070BD70B50D004468002CC1
:10CB400008D0236829009B6820009847002802D15C
:10CB5000E468F4E7200070BD70B50D004468002C57
:10CB600007D0236829002000DB689847E4682D1867
:10CB7000F5E72C7070BD70B50D004468002C08D02E
:10CB8000236829001B6820009847002802D1E46828
:10CB9000F4E7200070BDF8B542788B790D00017A7A
:10CBA0009B18040000208B4222DC6368834219D169
:10CBB0006560002623786A71EA792B719B182370CF
:10CBC000AB79B34213D9AB68B7006078DF19FFF7D0
:10CBD0002BFA3B68013603606378F6B20133637069
:10CBE000EEE70B00D9680029FBD1DD60E1E7012009
:10CBF000F8BD000070B50126054D064C2B68334288
:10CC000003D12000FFF708FA2E60200070BDC04657
:10CC10009020002094200020F7B506000D000C00A5
:10CC20008B180193019B671B9C4207D033682178C6
:10CC30001B683000984701340028F3D13800FEBD4E
:10CC400070B5040008000D0004F070FB23680200BA
:10CC500029005B682000984770BD10B50B1E02D0FC
:10CC6000FFF7EEFF0300180010BD10B5FFF7F5FF4A
:10CC700010BD10B503688A685B680968984710BDE5
:10CC800010B5FFF7EAFF10BD10B503681B689847A1
:10CC900010BD0B0010B50A6801001268180090471B
:10CCA00010BD000010B50249FFF7CAFF10BDC04615
:10CCB0007C46010070B50400FFF7CFFF050020009F
:10CCC000FFF7F0FF401970BD70B50500FFF7D1FF09
:10CCD00004002800FFF7E6FF201870BD70B50400BF
:10CCE000FFF7BBFF05002000FFF7DCFF401970BD18
:10CCF00070B50500FFF7CDFF04002800FFF7D2FF55
:10CD0000201870BDF0B58BB06B46150000220533BE
:10CD10000600DA770800012D00D80A2509AC2900A1
:10CD200001F000F9CAB2130037330700DBB209295A
:10CD300002D813003033DBB2013C2370002FEED158
:10CD400021003000FFF789FF0BB0F0BD10B5002ABD
:10CD500004D10368C9B21B68984710BDD2B2FFF76F
:10CD6000D1FFFAE710B5FFF7F1FF10BD70B5050070
:10CD7000FFF7ECFF04002800FFF794FF201870BDB8
:10CD800010B5040000F012FCE060236820005B692D
:10CD90009847002808DA00F009FCE368C01AA36885
:10CDA0009842F2D30120404210BD000070B50D0042
:10CDB00009490400160000F06BF82800FFF7E0FFB7
:10CDC000002806DBC1B2B14203D0200000F075F9A3
:10CDD000F3E7200070BDC0461D3801000B680360FA
:10CDE0004B6843608B68836000230B604B608B60F3
:10CDF000704710B504000068002801D003F0E4FC7F
:10CE0000200010BD10B504000068002801D003F018
:10CE1000DBFC00232360A360636010BD70B50400D9
:10CE20000D000068013104F025FA031E01D0012035
:10CE300028C470BD036810B50400002B04D04368FB
:10CE40008B4201D3012010BD2000FFF7E7FF00282F
:10CE5000F9D0A368002BF5D122681370F3E770B501
:10CE60000E00110004001500FFF7E4FF002804D1B4
:10CE70002000FFF7C7FF200070BD2A003100A56029
:10CE8000206803F0CCFC00232268A1685354F2E729
:10CE9000002370B504000D00036043608360994275
:10CEA00007D0080004F042FA290002002000FFF732
:10CEB000D6FF200070BD70B5050008000C0004F01E
:10CEC00035FA210002002800FFF7C9FF70BD0023DA
:10CED00013B5040001AA0360436083601170110060
:10CEE0005370FFF7E8FF200016BD1FB504000023B4
:10CEF000080023606360A36001A900F025FC200006
:10CF000001A9FFF7D8FF200004B010BD10B5002321
:10CF100004008AB023606360A360080001A900F0E8
:10CF20000FFC200001A9FFF7C6FF20000AB010BDCA
:10CF300070B50E00110004001500FFF77BFF0028FC
:10CF400004D12000FFF75EFF200070BDA560310016
:10CF5000206804F0E3F9F7E770B505000C0088429B
:10CF60000CD0006803F030FC23682B60A368AB6032
:10CF700063686B6000232360A360636070BD10B5BD
:10CF80000B000400884205D00968002904D09A6883
:10CF9000FFF765FF200010BDFFF734FFFAE700231D
:10CFA00010B50400036043608360FFF7E8FF2000D2
:10CFB00010BD10B50400FFF7CFFF200010BD10B565
:10CFC0000400002903D0FFF776FF200010BDFFF713
:10CFD00019FFFAE7002370B5040090B003604360C6
:10CFE0008360151C0A2A00D90A25EDB2AE1C081C64
:10CFF00003F012FB76B203AB009332002B0000F07B
:10D000007DFA01002000FFF7DAFF200010B070BDAC
:10D0100070B504000D1E09D0080004F087F929003E
:10D0200002002000FFF784FF200070BDFFF7EAFE3A
:10D03000FAE7002310B50400036043608360FFF744
:10D04000E7FF200010BDF7B504000191160000298C
:10D0500002D100252800FEBD0125002AFAD08368F0
:10D06000D7183900FFF7E6FE051EF2D02368A26844
:10D0700001999818320003F0D2FB00222368A760C0
:10D08000DA55E7E710B58A680968FFF7DCFF10BDDD
:10D0900070B5050008000C0004F048F921000200FA
:10D0A0002800FFF7D0FF70BD002310B5994202D0D1
:10D0B000FFF7EEFF0300180010BD07B56B46D971EE
:10D0C000073301221900FFF7BEFF0EBDF8B50400BB
:10D0D0000F1E02D100263000F8BD080004F026F92A
:10D0E00001260028F7D0A368C51829002000FFF703
:10D0F000A1FE061EEED02368A2683900981804F03D
:10D100000DF9A560E7E710B58A6809680400FFF724
:10D110009AFF002802D12000FFF774FE200010BD06
:10D1200010B50400002904D12000FFF76BFE200099
:10D1300010BDFFF7B9FF0028F6D0F8E710B50400DE
:10D14000FFF7C4FF002802D12000FFF75BFE20009C
:10D1500010BD026810B50B68002A13D0002B0CD14B
:10D1600081681800002907D0107805E08968100050
:10D17000002901D01878404210BD1900100004F0B9
:10D18000C3F8F9E7002BF1D11800F5E7826810B574
:10D1900094468A680023944504D1FFF7DAFF43429E
:10D1A0004341DBB2180010BD836810B5002B07D1D6
:10D1B0000120002903D0087843425841C0B210BD75
:10D1C0000068002901D10078F6E704F09DF8F3E744
:10D1D00083688B4203D903685818002B02D10023BF
:10D1E000014803707047C046A020002082680023D9
:10D1F0008A4203D902689A4200D0535C18007047F3
:10D2000010B5FFF7F3FF10BD70B50D00002A06D072
:10D21000002904D084689C4202D800230B7070BDA2
:10D22000013AE41A944200D9140001682200C91896
:10D23000280004F082F800232B55F0E7836810B52E
:10D24000934207D90468A01804F050F8002801D0D0
:10D25000001B10BD01204042FBE710B50022FFF784
:10D26000EDFF10BD836810B5934208D904680968C2
:10D27000A01804F076F8002801D0001B10BD012092
:10D280004042FBE710B50022FFF7ECFF10BDF7B5F9
:10D2900015008A680F00002A1BD08368002B18D065
:10D2A0009A4216D8AB4200D85D1E066801243000B1
:10D2B000731964420193019B98420CD8396804F0B9
:10D2C00050F8002807D0831BAB4200D81C00013067
:10D2D000F1E7012464422000FEBD0000F8B506001D
:10D2E0000F0014001D009A4201D92C0015000949B5
:10D2F0003000FFF7CDFDBA68A24208D9AA4200D992
:10D300002A003968121B09193000FFF7A8FD300008
:10D31000F8BDC0461D380100F0B5836885B0040033
:10D320000F0016000193002B00D185E08B6802935B
:10D33000002B00D180E09368029A00689B1A00934A
:10D340000BD1396804F00DF8041E75D0B26831684D
:10D3500003F065FAB368E018F3E70B68019D0393E7
:10D36000009B002B2FDA039903F0FBFF002804D069
:10D37000029BC018009BED18F5E7019BAB425BD008
:10D380001A00013A002A57DB39002000FFF77FFF1F
:10D39000051E51DBBB68C21823689918A3689A1A46
:10D3A000009BC81803F044FAA268009B21689B18F0
:10D3B0000022A360CA542368B2685819316803F088
:10D3C0002EFA6A1EDEE7039903F0CBFF002804D093
:10D3D000029BC018009BED18F5E7019BAB422BD0D8
:10D3E0006368AB4222D3A3685A1E002A24DB3900AB
:10D3F0002000FFF74CFF051E1EDBBB68C218236828
:10D400009918A3689A1A009BC81803F011FAA26829
:10D41000009B21689B180022A360CA542368B2684D
:10D420005819316803F0FBF96A1EDEE72900200075
:10D43000FFF7F4FC0028D6D105B0F0BD70B58568C3
:10D4400004008D4213D9002A11D06B1A934200D9DF
:10D4500013002068ED1ACB18C3186A1A4018A5608B
:10D46000190003F0E5F900212268A368D15470BDCA
:10D47000012210B55242FFF7E1FF10BD10B504685C
:10D48000002C07D02078002804D004F019F8207070
:10D490000134F7E710BDF8B507680600002F22D069
:10D4A0008468002C1FD03D00287803F069F900281B
:10D4B00001D00135F8E7013C3C19207803F060F910
:10D4C000002803D0A54201D8013CF6E70134621BD5
:10D4D000B260AF4203D22900380003F0A9F900215D
:10D4E0003268B368D154F8BD0368002010B5834298
:10D4F00002D0180003F00CF910BD000030B5040094
:10D5000087B00D00064901A803F0D0FE22002B00D1
:10D5100001A90A9803F0CAFE0A9807B030BDC046B8
:10D520007F460100FEE70000034B10B51B68002B8F
:10D5300000D0984710BDC046A420002070B50F4908
:10D540000F4CA14204D100F02BF900F001F9FEE7E5
:10D550000C4D00238D42F6D0CA18E818A24205D31C
:10D56000094B8242EFD00949002204E000680433ED
:10D570001060F1E704C38B42FCD3E4E70000002015
:10D58000480200208C4A010048020020BC200020F4
:10D5900010B500F06FF8002801D100F055F810BD6B
:10D5A000014B18607047C046A4200020014B18684A
:10D5B0007047C046A8200020F7B5134801228446D2
:10D5C0001249134C8E68636805689B0E13400192E4
:10D5D00088686268019F920E3A4067463F689342AE
:10D5E0000ED1BD420CD186420AD35B19FA25486898
:10D5F000AD00861B07486B437043000DC018FEBD8D
:10D600003D0013000600E3E7A820002010E000E042
:10D6100000ED00E05555000070B5041E10D0FFF776
:10D62000CBFF050000F025F8FFF7C6FF054B401BB8
:10D630009842F7D9FA23013C9B00ED18002CF3D156
:10D6400070BDC046E703000010B5034A13680133FC
:10D65000136000F093FB10BDA820002010B5002837
:10D6600006D030230321584300F0D6FB0138FDD10A
:10D6700010BD704700207047F0B50C008BB016004D
:10D68000002926D0931E222B2DD80A2A05D1002846
:10D6900003DA0127404201AD0AE00027FBE7310031
:10D6A00000F040FCCBB2092916D830332B7001357D
:10D6B0002A000028F3D101ABAB42F0D02300002FA9
:10D6C00002D02D21631C217001A98A4206D80022B4
:10D6D0001A7020000BB0F0BD5733E7E7013A11781C
:10D6E00019700133F0E70024F3E7F0B50D008BB0BB
:10D6F000170000290ED0931E222B1FD801AC260044
:10D700002300002809D1A64207D02A00B34210D82E
:10D710000023137028000BB0F0BD390000F002FCAC
:10D72000CBB2092903D8303323700134E8E75733EB
:10D73000FAE7013B197811700132E7E70025E9E7C4
:10D7400010B5FFF799FF10BD10B5FFF7CEFF10BD64
:10D7500010B500F0EFF802F0EFFFFDF74EFA0120F0
:10D76000FFF75AFF084C2000FEF76EFD2000FDF782
:10D770009BFFF9F72BFDFAF7DDF8044B002BFAD0ED
:10D7800000E000BFF7E7C046A41A00200000000038
:10D7900010B503F00FF810BD10B503F015F810BD6B
:10D7A0001E22F0B5504851494368514D93431A0029
:10D7B00002231343436008238A691343FE228B61CB
:10D7C0002B68D2039B0213404A4A13434A4A93618F
:10D7D00013000422DC681442FCD00124474A147070
:10D7E0001678264203D0567876B2002EF8DB012454
:10D7F0009460547864B2002CFBDB414C5460547844
:10D8000064B2002CFBDB8224E4015480547864B2BF
:10D81000002CFBDB02249C840E34DE682642FCD004
:10D82000384CDC621024DE682642FCD02C68A40E42
:10D830003F2C00D1203C9E6A334FA4023E4034432B
:10D840009C629C6A314EA40AA40234439C62304C10
:10D85000DC6200249C841034DE682642FCD02D4C0F
:10D860009C841024DE682642FCD002249E8C344323
:10D870009C841024DE682642FCD0002494605478F6
:10D8800064B2002CFBDB244C5460547864B2002C4E
:10D89000FBDB1C6A214E344080261C621C6AB443A8
:10D8A0001C62032393601E4B536053785BB2002BC2
:10D8B000FBDB0023FF240B721A4A4B728B72CB7274
:10D8C000194B1A60194A2B6811689A065B01C90E38
:10D8D0002340520F12020B431343154A1385802332
:10D8E000426813434360F0BD004000410004004023
:10D8F000246080000606000000080040000C004084
:10D9000001040100B905FF7DFF03FFFFFF010000D7
:10D9100080BB0A1C2405000000070300FFFCFFFF7A
:10D9200003060100006CDC0238000020206080004B
:10D9300000400042FA21314B10B51868890000F010
:10D940006BFA2F4B0138984256D82E492E4A486020
:10D95000C020136A00061B021B0A03431362002443
:10D9600007238C600B608021136A09061B021B0AC7
:10D970000B431362FC22254B196A0A431A62FC22EC
:10D98000196A92010A431A62A022196AD2020A4352
:10D990001A62E0B20021013400F0EEF81F2CF8D139
:10D9A0001B4B1C005A7852B2002AFBDB194A5A80E2
:10D9B000194B1A00597EC9090129FBD0E421C9007D
:10D9C00099803F21D970537EDB09012BFBD0C02306
:10D9D00000205B011361907000F02EF863785BB259
:10D9E000002BFBDB0D4B0E4A6380D379DB09012B47
:10D9F000FBD04123537010BDFEE7C0463800002025
:10DA0000FFFFFF0010E000E000ED00E00004004038
:10DA1000000C00401E400000004000422140000079
:10DA200000480042914202D002D98A1AD040704781
:10DA3000521A9040FBE70000164A00B51300517ED1
:10DA4000C9090129FBD00138042816D81969124ADE
:10DA50000A400F211A615A788A4300F0D3F903086B
:10DA6000060B0300110001220A435A7000BD110089
:10DA70000322F9E711000222F6E7F02311691B05E2
:10DA80000B430F21136153788B43190002230B437F
:10DA90005370EBE700400042FFFFFFF010B50400B9
:10DAA0000D2801D80E34E4B20121200000F0F4F872
:10DAB0001823102163432B4CE4186156002901D030
:10DAC00014290DD1284B1800DA79D209012AFBD08C
:10DAD00002241A78A2431A70C379DB09012BFBD008
:10DAE00022480300427ED209012AFBD01F2402698A
:10DAF0002140A2430A4302615A7ED209012AFBD087
:10DB0000022219780A431A705A7ED209012AFBD0E0
:10DB10000222197B0A431A731A7ED207FCD501220E
:10DB20001A765A7ED209012AFBD00222197B0A43B7
:10DB30001A731A7ED207FCD5588B80B25A7ED2094E
:10DB4000012AFBD002211A788A431A705A7ED20920
:10DB5000012AFBD0064B1A68064B1968FFF762FFD3
:10DB600010BDC04660420100004800420040004233
:10DB7000400000203C000020182330B51D000400A8
:10DB800045430820204A55192856013014D003294E
:10DB900012D808006343D156D31800F033F9022895
:10DBA0000E1B5868CB010221184A9B181A184032E4
:10DBB0001170012282405A6030BD5868CB010621A5
:10DBC000124A9B181A1840321170012282405A6082
:10DBD0009A61F1E75868CB0106210C4A9B181A1884
:10DBE00040321170012282405A605A61E4E758685D
:10DBF000CB010221054A9B181A18403211700122EC
:10DC000082409A60D8E7C04660420100004400416B
:10DC10001823F0B508245843114A13181C5701342F
:10DC20001BD0012635005F688356BD400D4ADB01DD
:10DC30009A18906805420BD10C00601E8441D219DD
:10DC40004032107834400336A400B04320431070B3
:10DC5000044A9B18002901D15D61F0BD9D61FCE77C
:10DC60006042010000440041182310B508244343DA
:10DC700007490020CA181457013408D05B560549DB
:10DC8000DB015B18186A5368D8400123184010BDA7
:10DC9000604201000044004118224243F8B52C4E76
:10DCA0000300B218127A52B2140001320ED0481C8E
:10DCB00000240C280AD800F0A5F8072020202020F6
:10DCC0002020200B0B0B0B00012464422000F8BD28
:10DCD000092905D10021D8B2FFF74EFF0024F5E74E
:10DCE0000A2902D1D8B20839F6E700240B29EDD170
:10DCF000D8B20A39FFF740FFE8E718204343F2188B
:10DD00005568F3562C00134ADB016E0817389B1830
:10DD1000C9B204409E19002C0DD00F243036327841
:10DD2000090122401143C9B25B19317040331A789E
:10DD300010431870D2E732000F27303216785B1983
:10DD4000BE433143117040331A7810431870BDE759
:10DD5000604201000044004110B50400FDF703FBE0
:10DD6000014B1C6010BDC046440000200122024B44
:10DD700052421A607047C04644000020164A10B54F
:10DD80001368591C26D0013B1360002B22D172B6B8
:10DD9000124B134A0433934213D9124A0121100043
:10DDA000147D0C42FCD02021148BFF319B085B00BA
:10DDB00021431183D3610C4B13800123027D1A424E
:10DDC000FCD0BFF34F8F094B094ADA60BFF34F8F86
:10DDD000C046FDE710BDC046440000200020000002
:10DDE000030200000040004102A5FFFF00ED00E03B
:10DDF0000400FA050B0010B50100180002F08EFCBB
:10DE000010BD000002B4714649084900095C490090
:10DE10008E4402BC7047C046002243088B4274D334
:10DE200003098B425FD3030A8B4244D3030B8B421B
:10DE300028D3030C8B420DD3FF22090212BA030C24
:10DE40008B4202D31212090265D0030B8B4219D305
:10DE500000E0090AC30B8B4201D3CB03C01A524125
:10DE6000830B8B4201D38B03C01A5241430B8B426D
:10DE700001D34B03C01A5241030B8B4201D30B0356
:10DE8000C01A5241C30A8B4201D3CB02C01A52417D
:10DE9000830A8B4201D38B02C01A5241430A8B4240
:10DEA00001D34B02C01A5241030A8B4201D30B0229
:10DEB000C01A5241CDD2C3098B4201D3CB01C01A43
:10DEC000524183098B4201D38B01C01A524143094D
:10DED0008B4201D34B01C01A524103098B4201D33B
:10DEE0000B01C01A5241C3088B4201D3CB00C01AA8
:10DEF000524183088B4201D38B00C01A5241430820
:10DF00008B4201D34B00C01A5241411A00D2014644
:10DF1000524110467047FFE701B5002000F0F0F8CD
:10DF200002BDC0460029F7D076E7704703460B4391
:10DF30007FD4002243088B4274D303098B425FD302
:10DF4000030A8B4244D3030B8B4228D3030C8B422E
:10DF50000DD3FF22090212BA030C8B4202D3121214
:10DF6000090265D0030B8B4219D300E0090AC30BE9
:10DF70008B4201D3CB03C01A5241830B8B4201D396
:10DF80008B03C01A5241430B8B4201D34B03C01A7F
:10DF90005241030B8B4201D30B03C01A5241C30AF7
:10DFA0008B4201D3CB02C01A5241830A8B4201D368
:10DFB0008B02C01A5241430A8B4201D34B02C01A52
:10DFC0005241030A8B4201D30B02C01A5241CDD2F7
:10DFD000C3098B4201D3CB01C01A524183098B4242
:10DFE00001D38B01C01A524143098B4201D34B012B
:10DFF000C01A524103098B4201D30B01C01A52418E
:10E00000C3088B4201D3CB00C01A524183088B4214
:10E0100001D38B00C01A524143088B4201D34B00FD
:10E02000C01A5241411A00D201465241104670476F
:10E030005DE0CA0F00D04942031000D34042534074
:10E0400000229C4603098B422DD3030A8B4212D334
:10E05000FC22890112BA030A8B420CD38901921166
:10E060008B4208D3890192118B4204D389013AD0A3
:10E07000921100E08909C3098B4201D3CB01C01A78
:10E08000524183098B4201D38B01C01A524143098B
:10E090008B4201D34B01C01A524103098B4201D379
:10E0A0000B01C01A5241C3088B4201D3CB00C01AE6
:10E0B000524183088B4201D38B00C01A5241D9D2FE
:10E0C00043088B4201D34B00C01A5241411A00D27F
:10E0D0000146634652415B10104601D34042002B7B
:10E0E00000D54942704763465B1000D3404201B5FA
:10E0F000002000F005F802BD0029F8D016E77047AF
:10E100007047C0468446101C62468C46191C634604
:10E1100000E0C0461FB501F09FFB002801D400219C
:10E12000C8421FBD10B501F0F7FA4042013010BDE2
:10E1300010B501F091FB002801DB002010BD01208B
:10E1400010BDC04610B501F087FB002801DD00209E
:10E1500010BD012010BDC04610B501F019FB00280C
:10E1600001DC002010BD012010BDC04610B501F03B
:10E170000FFB002801DA002010BD012010BDC046B1
:10E180008446081C6146FFE71FB500F0BBFA002873
:10E1900001D40021C8421FBD10B500F03DFA404235
:10E1A000013010BD10B500F0ADFA002801DB0020F1
:10E1B00010BD012010BDC04610B500F0A3FA002824
:10E1C00001DD002010BD012010BDC04610B500F0DB
:10E1D0004BFA002801DC002010BD012010BDC04614
:10E1E00010B500F041FA002801DA002010BD01202E
:10E1F00010BDC046002B11D1002A0FD1002900D13B
:10E20000002802D00021C943081C07B4024802A11B
:10E210004018029003BDC046E9FEFFFF03B4684604
:10E2200001B5029800F024F8019B9E4602B00CBC98
:10E230007047C04670B500220C4B04000D00FFF77C
:10E2400095FF002804D12000290002F043F970BD99
:10E25000064B00222000290001F0D8FD02F03AF917
:10E2600080231B069C466044F1E7C0460000E04165
:10E27000F0B54F464646D646C0B5040082B00D0004
:10E28000914698468B422FD82CD04146484602F002
:10E2900033FA29000600200002F02EFA331A9C46B9
:10E2A000203B9A4600D576E04B46524693401F00ED
:10E2B0004B46624693401E00AF4228D825D05346B5
:10E2C000A41BBD41002B00DA7BE00022002300925A
:10E2D00001930123524693400193012362469340E8
:10E2E000009318E08242D0D90022002300920193CB
:10E2F0000A9B002B01D01C605D600098019902B060
:10E300001CBC90469946A246F0BDA342D7D9002234
:10E310000023009201936346002BE9D0FB07984647
:10E32000414672080A437B0866460EE0AB4201D1C3
:10E33000A2420CD8A41A9D41012024196D4100214C
:10E34000013E24184D41002E06D0AB42EED9013ECD
:10E3500024196D41002EF8D10098019953460019F7
:10E360006941002B23DB2B005246D3402A00644630
:10E37000E2401C0053461500002B2DDB26005746BB
:10E38000BE40330026006746BE403200801A9941E5
:10E3900000900191ACE7624620239B1A4A46DA407E
:10E3A0006146130042468A4017001F4380E76246D9
:10E3B00020239B1A2A0066469A402300F340134309
:10E3C000D4E76246202300219B1A0022009101928B
:10E3D0000122DA40019280E72023624626009B1A40
:10E3E000DE402F00B0466646B74046463B0033430A
:10E3F000C8E7C046F8B557464E464546DE46440295
:10E40000E0B546008846640A360EC70F002E63D07A
:10E41000FF2E24D08023E400DB041C430023994614
:10E420009B467F3E434642465D02D20F5B006D0A2B
:10E430001B0E9046924665D0FF2B55D080220021BE
:10E44000ED00D2047F3B1543F61A43464A467B4013
:10E450000F2A00D98DE06D48920082589746002C13
:10E4600054D108239946063BFF269B46DAE7002550
:10E47000534602291BD0032900D1BFE0012928D02F
:10E4800030007F30002820DD6A0704D00F222A40A8
:10E49000042A00D004352A0103D530005C4A8030BC
:10E4A0001540FE2803DCAC01640AC2B201E0FF2281
:10E4B00000246402D205600ADB07104318433CBC09
:10E4C00090469946A246AB46F8BD0122101A1B2879
:10E4D0007CDD00220024ECE7002C1DD104239946AA
:10E4E000033B00269B469DE7FF3E002D20D10221E5
:10E4F00043464A467B400A430F2AD8D845489200F3
:10E5000082589746002D19D10121F1E70C23994635
:10E51000093BFF269B4685E7200002F0CFF87626D0
:10E52000431F9C4000237642361A99469B4679E762
:10E530004A4603231A439146032186E7280002F046
:10E54000BDF8431F36189D40763600217DE78024B4
:10E550000023E403FF22ACE700258023DB031C42F9
:10E5600028D01D4226D12B435C02640A4346FF2279
:10E570009FE762016C01A24224D21B210025013ECB
:10E58000012710006D005200002801DB944201D8E1
:10E59000121B3D4301390029F3D11400621E94413E
:10E5A00025436DE7BA46594625005346022900D057
:10E5B00061E77CE78023DB031C436402640A3B00C1
:10E5C000FF2276E7121B1A210125D9E79E362A0081
:10E5D000B5402C00C240651EAC411443620704D014
:10E5E0000F222240042A00D00434620103D4A40183
:10E5F000640A00225DE7012200245AE78024E40334
:10E600002C436402640AFF2253E7C0468846010097
:10E61000FFFFFFF7C846010070B542004E024C00F4
:10E6200045026D0A120EC30F760A240EC90FFF2A87
:10E630000FD0FF2C11D00120A24200D070BDB542F6
:10E64000FCD18B420DD0002AF8D12800451EA841EC
:10E65000F4E70120002DF1D1EBE70120002EEDD1F0
:10E66000E9E70020EAE7C04670B54A004E024502DD
:10E6700044006D0A240EC30F760A120EC90FFF2C38
:10E6800015D0FF2A0ED0002C15D1002A01D1002E62
:10E690001CD0002D14D08B4227D00220013B184003
:10E6A000013870BD002EEED002204042F9E7002D67
:10E6B000FAD1FF2A0ED0002A0ED1002EEDD00BE0A9
:10E6C00001230139994308000130EAE70020002DB9
:10E6D000E7D0E2E7002EE7D18B42DED1944205DDA0
:10E6E0000221581E08400138DBE70024A24204DC66
:10E6F000B542D2D80020B542D3D2581E0123984348
:10E700000130CEE730B5420044024D02C30F48004D
:10E71000640A120E6D0A000EC90FFF2A12D0FF28DC
:10E720000CD0002A12D1002819D1002D17D1002CAD
:10E730002BD00220013B1840013826E0002DF0D0FC
:10E74000022022E0002CFBD1FF281FD000281FD17F
:10E75000002D1DD10220013B1840013815E0002C8E
:10E760000ED08B42E5D10022904204DCAC42E0D8CE
:10E770000020AC4209D2581E01239843013004E026
:10E780000123013999430800013030BD002DD7D154
:10E790008B42CED18242E7DD0221581E084001386B
:10E7A000F3E7C046F0B54E4657464546DE46E0B56F
:10E7B00043025B0A450083B00F1C99462D0EC60F1D
:10E7C000002D57D0FF2D24D08020DB00C00418433B
:10E7D000002381469A469B467F3D7C027A00FB0FD0
:10E7E000640A120E984623D0FF2A4BD0E3008024FF
:10E7F0000020E4047F3A1C43AD186B1C474601938C
:10E80000534677403A000F2B48D87D499B00CB58A0
:10E810009F46002B00D085E008339A46063B9B4676
:10E820007C027A00FB0FFF25640A120E9846DBD1AA
:10E83000002C00D090E0524601231A43924601205A
:10E84000DBE74C4658461700022824D0032800D1A5
:10E85000CFE00022002301284DD15802D205400A02
:10E86000FF071043384303B03CBC90469946A2468C
:10E87000AB46F0BD002B5BD104239A46033B002539
:10E880009B46AAE7FF35002C60D1524602231A436B
:10E8900092460220B1E7FF220023DEE74B461B0C25
:10E8A0009C464B462604360C180461463300220C65
:10E8B0006446000C43434E435043544380191A0CA2
:10E8C0001218964203D9802149028C4664441B04E5
:10E8D0001B0C1004C01883015E1EB341800E184348
:10E8E000130C1B199B0103431C00230179D5012341
:10E8F00062081C401443019A7F32002A4DDD6307F1
:10E9000004D00F232340042B00D00434230103D56B
:10E910003C4B019A1C408032FE2ABCDCA3015B0AFE
:10E92000D2B29AE70C239A46093BFF259B4654E74F
:10E93000180001F0C3FE4A46431F76259A40002383
:10E940006D4291462D1A9A469B4646E7524603234E
:10E950001A439246032050E7200001F0AFFE431F08
:10E960002D1A9C40763D002047E780230027DB03DB
:10E97000FF2272E7424666E74C463200584662E79D
:10E9800080234A46DB031A4222D01C4220D1234373
:10E990005B025B0A4746FF225FE701239A1A1B2AA4
:10E9A00021DC23000199D3409E318C401A002300C2
:10E9B0005C1EA34113435A0704D00F221A40042AB5
:10E9C00000D004335A0111D49B015B0A002244E7B2
:10E9D00080234A46DB0313435B025B0A3700FF22B6
:10E9E0003BE7019587E70022002336E70122002359
:10E9F00033E78023DB0323435B025B0AFF222CE720
:10EA000008470100FFFFFFF741024200C30F490A18
:10EA1000120E00207E2A0DD99D2A0CD880200004D9
:10EA20000143952A0ADC9620821AD1404842002BE5
:10EA300000D108007047034A9818FBE7963A9140C6
:10EA4000F4E7C046FFFFFF7F70B500283DD0C31735
:10EA5000C5185D40C40F280001F030FE9E22121A36
:10EA6000962A07DCD2B2082833DD083885406802D0
:10EA7000400A23E0992A0BDD052329001B1AD940FF
:10EA800003001B339D402B005D1EAB4119430D005D
:10EA9000052801DD431F9D402B000F490B406E07E9
:10EAA00009D00F263540042D05D004335D0102D571
:10EAB0009F220B40121A9B01580AD2B24002D20583
:10EAC000400AE4071043204370BD002400220020C8
:10EAD000F4E76802400AF1E7FFFFFFFBF0B54F469D
:10EAE0004646D6460C000903C0B5490A470F5E00EA
:10EAF00039431F03DB0F9C4665007B0A570F1F43FA
:10EB00006D0DE40F760DA146C000B846D200AB1BD8
:10EB100064457BD0002B5FDD002E00D0A4E03E00DA
:10EB2000164300D112E15E1E002E00D09EE1871A2E
:10EB30004346B84280410125C91A4042091A0B02D6
:10EB400000D431E149024E0A002E00D16EE13000BE
:10EB500001F0B4FD0300083B1F2B00DD61E1202222
:10EB60003900D21A9E40D1409F400E439D4200DDA5
:10EB700051E15D1B6B1C1F2B00DD7CE12021C91ABC
:10EB80003D0030008F408840DD40791E8F413100CC
:10EB900007222843D940002507433A40002A09D0DC
:10EBA0000F233B40042B05D03B1DBB42BF417F429E
:10EBB000C9191F000B0200D426E26A1CC64B55057A
:10EBC0006D0D9A4200D106E1C44AFF080A4053077E
:10EBD00052023B43120B8EE0002B00D0B8E06B1CBE
:10EBE0005B055B0D012B00DC30E1871A4346B84220
:10EBF000B641CB1A76429E1B330200D54CE13B0056
:10EC00003343A1D100220024002570E0002B00DC5A
:10EC1000E5E0002E00D183E0AF4EB54260D0802603
:10EC200036043743B846382B00DC3EE143461343F5
:10EC30001F007A1E97413F188742804140420918C1
:10EC40000B0200D4B0E0A44B01359D4200D1C3E0DB
:10EC5000A24A7B080A4001210F401F435108D307F5
:10EC600007221F433A4099E79B4EB54238D0802691
:10EC700036043743B846382B00DDDCE01F2B00DCC0
:10EC800030E11E004746203EF740BC46202B04D012
:10EC90004026F31A46469E403243170063467A1ECA
:10ECA00097411F43CCE0002B00D104E243461343BD
:10ECB00000D159E14B07C00818438023C9081B0342
:10ECC000194208D04546ED081D4204D14346D008FC
:10ECD000590708432900420FC9007F4D1143C00066
:10ECE0004B07CA087C49C00803438D4268D0120311
:10ECF0006D05120B6D0D002112031800130B0A0D88
:10ED000012051A43764B2D0513402B435B00E40795
:10ED10005B08234319001CBC90469946A246F0BDEF
:10ED20003E00164312D05E1E002E00D000E1871870
:10ED30008742804141444042091801250B0233D5E6
:10ED4000022585E764463300414610001D00C7E7F1
:10ED5000002D00D0DAE00C000443F3D05C1C00D19D
:10ED60009FE15D4CA64200D12FE1DB43382B00DD53
:10ED700066E11F2B00DD83E120240500E41A0F006B
:10ED8000DD40D940A0404346A7405B1A441EA04145
:10ED900098462F433843171ABA429241434652428B
:10EDA000991A64463500CAE607223A40002A00D084
:10EDB000F6E64B07CA084849FF083B438D4296D107
:10EDC0001900114300D19EE1802109030A43120377
:10EDD000120B414D8FE71500002200238BE7002B1B
:10EDE00000D0C7E06B1C5F057F0D012F00DCF1E058
:10EDF000394DAB4200D1B9E085180A0085428941FE
:10EE00004244494251180722CF076D082F43490851
:10EE10003A401D00C2E607223049ED1A31403A401F
:10EE2000BCE63E002838864000279FE6380001F007
:10EE300045FC20308EE6434613431F007A1E97415F
:10EE4000C71BB84280414042091A78E60E003B00D9
:10EE500006431343002D61D1002E00D0F4E0002BB7
:10EE600000D11BE164463900100039E71A4FBB425C
:10EE70007AD03300FFE630001F3DE840202B03D05E
:10EE80004021CB1A9E4037437B1E9F4107220743F8
:10EE90003A400021002589E7171A4346BA42B64195
:10EEA000591A76428E1B64464EE61F2B00DDADE0FC
:10EEB00020264746F61AB740B9461700B246DF404B
:10EEC0004E463E4337005646B240561EB2411743A7
:10EED0004246DA408918AEE6FF070000FFFF7FFFD9
:10EEE000FFFF0F8020264746F61AB740B9461700A5
:10EEF000B246DF404E463E4337005646B240561EAD
:10EF0000B24117434246DA40891A99E77F4CA6423C
:10EF10005BD0802424045B42214327E7002E0CD1E0
:10EF2000002B00D1CBE0644639001000774DD7E6C6
:10EF3000764FBB4218D0330075E6002B14D04B0738
:10EF4000C00818438023C9081B03194207D0FC08D6
:10EF50001C4204D17907D0080843E14621004C4601
:10EF6000420FC9001143C000684DB9E61D000022E0
:10EF70000023C0E6002D5BD10D00054300D1E2E681
:10EF80005D1C00D1B0E0614DAE421FD0DB43382B99
:10EF900071DC1F2B00DD96E020250F00ED1AAF403D
:10EFA000B9460700AA46DF404D463D432F0055466F
:10EFB000A840D940451EA84188440743BF1897423E
:10EFC00092415142414435003AE66446350041469B
:10EFD000100085E60B000343002D00D063E6002BF4
:10EFE000F5D04346134300D17AE687188742804123
:10EFF00007224144404209183A400B0200D4D5E6AA
:10F00000434B01351940C9E5380069E61E00474603
:10F01000203EF740BC46202B04D04026F31A46463B
:10F020009E403243170063467A1E97411F4302E613
:10F03000364DAE42CAD080252D045B422943A6E757
:10F040000843411E8841A6E6002B00D148E6871AF6
:10F050004346B842B641CB1A76429E1B33024BD58B
:10F06000171A4346BA429241591A5242891A072244
:10F0700064463A4092E501430F00791E8F419DE7B7
:10F080001C000F00203CE740202B03D04024E31A53
:10F0900099400843411E884138437CE60022002401
:10F0A00025E6171A4346BA429241591A5242891A22
:10F0B0006446350043E541461000144D10E68022B9
:10F0C0000024120380E61D000F00203DEF40BC46E7
:10F0D000202B03D04025EB1A9940084307006346D4
:10F0E000781E87411F4369E7871897429B41414437
:10F0F0005B42C9183500A3E53B003343CED007225D
:10F1000031003A4052E600231A00F4E5FF07000000
:10F11000FFFF7FFFF0B55746DE464E464546E0B559
:10F12000834607000E03480085B092461C00360B4C
:10F13000400DCD0F002800D19DE0954B984239D06D
:10F140008023F6001B041E43924A7B0F33439946EB
:10F15000944603006344009300230026FF000293BB
:10F1600023031B0B98466300E40F52465B0D01948A
:10F1700000D1B3E086498B4200D19EE04246D100E7
:10F18000802212040A435146490F11438B4681499C
:10F1900052468C4600996344CB1A0021D20000935A
:10F1A0002B0063409A460F2E00D905E17A4BB6003A
:10F1B0009B599F465B463343994600D0B8E00223F3
:10F1C0000826002700900293CAE7CB463A0002992E
:10F1D0000195019B9A46022927D0032900D180E29C
:10F1E000012944D06D49009B8C4663441C00002CCF
:10F1F00038DD530700D013E2D2085B46DB0109D5A6
:10F200005946674B19408B468021C9008C46009BAC
:10F2100063441C00634B9C4207DC5B4664055F074C
:10F220005B0217431B0B620D02E000230027584AC4
:10F2300000211B031C0B0B0D1B05234314055A4A0D
:10F24000380013401C4353466400DB0764081C432A
:10F25000210005B03CBC90469946A246AB46F0BDA5
:10F260000122524201231B1B382B00DCADE100229E
:10F2700000230027DCE75B46334399465ED0002E2F
:10F2800000D18AE1300001F019FA03000B3B1C2B7E
:10F2900000DD7BE11D22D31A5A460100DA4008390D
:10F2A0008E4013005F46334399468F403F4B002604
:10F2B0001B1A00930023029352E7414653460B4327
:10F2C0003B499B468C46009B634400935B46002B66
:10F2D0003BD1022300221E43022161E74346134330
:10F2E0009B4637D04346002B00D162E1404601F0F7
:10F2F000E5F903000B3B1C2B00DD53E10200414606
:10F30000083A914088461D21CB1A5146D9400B003E
:10F3100041460B439B46534693401A00009B2549A8
:10F320009C46604403008C4663440093002137E709
:10F330000323B14600900C26029311E700230093AB
:10F3400001330426002702930AE70323C3461E4322
:10F35000032125E701331E430022012120E700237A
:10F360009A46802300271B03094A61E78023494608
:10F370001B03194200D1E2E05946194200D0DEE0F9
:10F380000B431B0317001B0BA246014A50E7C04664
:10F39000FF07000001FCFFFF48470100FF030000DA
:10F3A000FFFFFFFEFE070000FFFF0F800DFCFFFFC9
:10F3B00001F8FFFFF3030000D94500D9CBE000D1ED
:10F3C000C6E03C0048460027009B013B00935B469B
:10F3D000160E1B021E431302984633041B0C99465B
:10F3E000310C0191FEF79EFD4A4642430B04210C6D
:10F3F000050019438A4207D98919013D8E4203D875
:10F400008A4201D9851E8919881A0199FEF78AFD59
:10F4100009048C464A46210464464243090C030011
:10F4200021438A4204D98919013B8E4200D8F1E078
:10F430002D041D43AB464346891A4246280C12044C
:10F440001D0C5B46140C22001B041B0C5A43039436
:10F450006B434443029568431B19150CEB189C42FF
:10F4600003D980246402A44660441C0C15041B04C8
:10F470002D0C20185D19814277D373D00C1AA24A43
:10F480007D1BAF42BF419446009B7F426344E01B1B
:10F490001C00864200D1DBE00199FEF743FD4A469D
:10F4A00042430B04290C070019438A4207D98919E2
:10F4B000013F8E4203D88A4201D9871E8919881AD2
:10F4C0000199FEF72FFD09044A46894629044D4655
:10F4D0004243090C030029438A4207D98919013B99
:10F4E0008E4203D88A4201D9831E89193F04891AA2
:10F4F0003A00039F1A43380013041B0C58438146FB
:10F500000298150C6F43434345434846000C84461C
:10F51000DB1963449F4203D980204002844665443E
:10F5200048461F0C00041B04000C7D191818A94242
:10F5300000D284E000D17FE001231A4357E6802304
:10F540004A461B0313431B031B0BAA466F4A6FE675
:10F55000BA4200D935E74B46DC0758087B081C4304
:10F56000FF0734E70024AF4289D247444745A4410E
:10F570005B466442A4196418013BA6421ED2A04215
:10F580006DD800D1B6E0241A9B4678E703005A46AE
:10F59000283B9A400027914688E6584601F08EF8AD
:10F5A000203072E603005246283B9A4093460022E0
:10F5B000B4E6504601F082F820309AE6A642E2D145
:10F5C000B845DCD9341A9B4659E71F2B65DC504CF3
:10F5D0000099A4465C46614408008C4011008240BA
:10F5E000D940501E82410C4314435A46DA4013005E
:10F5F000620709D00F222240042A05D02200141DE0
:10F600009442894149425B181A0262D501220023C3
:10F6100000270DE68A4200D80AE7831E891907E70A
:10F620000F231340042B00D1E6E5171D97429241AA
:10F6300053429B44FA08E0E5002800D1D7E5711851
:10F64000531EB14227D3A94215D358D01A0073E7ED
:10F65000002B00DC04E6012300229B44CDE50223BD
:10F660004744474589415B429C46494289190C19E8
:10F67000E344241A03E743465F0047459B41B846ED
:10F680005B429E19023A8919A94200D054E74045CD
:10F6900000D051E7ABE51A00F6E71F215F4649426B
:10F6A0000C1BE740202B07D01A49009B8C46634473
:10F6B00018005B4683401A43501E82413A43072795
:10F6C0000023174009D00F21002311401400042902
:10F6D00095D122005F075B021B0BD2081743002263
:10F6E000A6E5802359461B030B431B0317001B0B86
:10F6F000064A9DE5BD42B2D89B460024BFE6804540
:10F70000B9D31A00C3E7C046FF030000FF0700009B
:10F710001E0400003E040000F0B54F464646D646A3
:10F720008446C0B58046194E18030F034D00000BE8
:10F730005C0082463F0B6D0DC90F9146640DDB0FD7
:10F740000120B5420AD0B44203D0A54201D15745A9
:10F750000CD01CBC90469946A246F0BD66463E437E
:10F76000F7D1AC42F5D154461443F2D10120C8453B
:10F77000EFD1994207D0002DEBD163461F433800EB
:10F78000471EB841E5E70020E3E7C046FF07000059
:10F79000F0B54F464646D6464D00C0B50E03C90FDC
:10F7A0008A462C491F035C008046360B6D0D91463E
:10F7B0003F0B640DDB0F8D421ED08C4216D0002D06
:10F7C0001ED130438446002C01D13A4323D06246F7
:10F7D000002A1AD09A4529D0514602200139084002
:10F7E00001381CBC90469946A246F0BD3900114331
:10F7F000E5D002204042F4E73043FAD1AC420FD0CA
:10F80000002C0FD13A43E7D00CE00122013B934397
:10F8100018000130E5E763460020002BE1D0DBE76C
:10F820003A43E6D19A45D7D1A542D5DCA54205DBBE
:10F83000BE42D1D808D00020BE42D2D250460123C9
:10F84000013898430130CCE7C845C5D80020C845E9
:10F85000F4D3C6E7FF070000F0B54F464646D6464C
:10F860004D00C0B50E03C90F8A462E491F035C0028
:10F870008046360B6D0D91463F0B640DDB0F8D42BC
:10F8800018D08C4211D0002D18D130438446002C62
:10F890001ED13A431CD163460020002B30D0514684
:10F8A00002200139084001382AE039001143EAD02A
:10F8B000022025E03043FBD1AC4226D0002C26D1DB
:10F8C0003A4324D15146022001390840013817E05B
:10F8D0006246002A0FD09A45E1D1A54205DBBE421F
:10F8E000DDD819D00020BE420AD25046012301388B
:10F8F0009843013004E00122013B9343180001309A
:10F900001CBC90469946A246F0BD3A43D0D19A45D8
:10F91000C5D1A542C3DCE0E7C845C0D80020C84532
:10F92000E3D3EDE7FF070000F0B55746DE464E464D
:10F930004546E0B5834606000F03480087B092466F
:10F940001D003F0B400DCC0F002800D16FE0DE4BB7
:10F95000984238D08023FF001B041F43730F3B43A2
:10F960000193DA4B0027994600239B46F600814419
:10F970002B0369001B0B52469846490DED0F0029D9
:10F9800000D185E0D04B994200D173E04346DA00C4
:10F9900080231B0413435246CC48520F8446134322
:10F9A000524600206144D200894421006940009100
:10F9B0008C46012149448A460F2F00D990E0C44962
:10F9C000BF00CF59BF465B463B43019300D06AE17D
:10F9D00002230827002681469B46C9E73200584685
:10F9E000019B61460091022800D175E0032800D1F7
:10F9F000FEE1012800D02CE100230027002600258D
:10FA00003F032A0D3F0BB34812053A4302401B0542
:10FA10001343009A5B00D1075B080B4330001900C9
:10FA200007B03CBC90469946A246AB46F0BD5B464B
:10FA30003B43019300D12FE1002F00D1A5E1380015
:10FA400000F03CFE03000B3B1C2B00DD96E11D2269
:10FA5000D31A5A460100DA405E4608398F40130037
:10FA60008E403B4301939C4B00271B1A9946002371
:10FA70009B467DE7414653460B4393498C46E14400
:10FA8000002B00D01AE102220220174300228CE74B
:10FA9000134300D10DE14346002B00D181E14046E4
:10FAA00000F00CFE02000B3A1C2A00DD72E101009E
:10FAB000434608398B4098461D239A1A5346D34033
:10FAC0001A004346134352468A404946081A82495F
:10FAD00089468144002068E77B4B002700268EE79B
:10FAE000140C1204120C1100370C3604350C794337
:10FAF00028008C462E006043604483465643210014
:10FB0000300C80465846794340440291844506D9DA
:10FB10008846802149028C46E044414602913604E1
:10FB2000010C360C00048B4681191E0C1B041B0CA7
:10FB30000391190079438C46280075436544A84613
:10FB40005843050C45447743A94203D98021490213
:10FB50008C466744290C8C4639000004000C2D04A7
:10FB60002D186144AB4405915946049101990F0445
:10FB70003F0C080C390051434243904602008C462A
:10FB8000090C8B4662437C4344445C44A04503D942
:10FB90008021490288464244210C88466146090476
:10FBA000090C8C4639005943434370437E430F0C84
:10FBB000F6182404BE19644442448C46B34203D967
:10FBC00080235B0298464044029B61469846049B12
:10FBD000370443449B46AB45AD416B420D04059948
:10FBE0002D0C8C467F196744FD18A8465D462D19DB
:10FBF000A542A44193466442A446C344DC448F42D8
:10FC0000BF4198459B4193459241A445A4415B4225
:10FC10007F421F43360C52426442BF192243BF1831
:10FC2000624638184302D20D039913436A020A430D
:10FC3000501E82416146ED0D2A434E023243D901E6
:10FC400000D4B3E00126500832400243DE073243BD
:10FC50005B08224C5444002C62DD510709D00F2070
:10FC60001040042805D0101D9042924152429B182A
:10FC70000200D90104D580241948E400034054440B
:10FC80001848844200DD27E75E075B02D2081F0B9D
:10FC9000630516435B0DB2E6002399460133042742
:10FCA00000269B4664E60323019781460C279B466A
:10FCB0005EE6012201201743002276E6032303209B
:10FCC0001F43434671E6C046FF07000001FCFFFFEB
:10FCD00088470100FFFF0F800DFCFFFFFF030000BE
:10FCE000FFFFFFFEFE0700000023802700933F0375
:10FCF0000026434B83E6019B3200A446584670E63B
:10FD0000AC466EE6802701993F0339422DD03B4235
:10FD10002BD11F433F033F0B00951600384B6EE677
:10FD200001252D1B382D00DD66E61F2D40DC3548F2
:10FD30001C005044160082408440EE40501E824118
:10FD400034431443EB40620709D00F222240042AB7
:10FD500005D02200141D9442804140421B181A0213
:10FD60003ED501230027002649E68027019B3F035B
:10FD70001F433F033F0B0094214B40E603005A46CC
:10FD8000283B9A40002601926DE6584600F096FC0A
:10FD9000203057E603005246283B9A4013000022C9
:10FDA00093E6504600F08AFC20307BE6CA4650E7D6
:10FDB0001F201E004042041BE640202D03D0124CA1
:10FDC0005444A3401A43501E824132430726002761
:10FDD000164009D00F200023104014000428B9D188
:10FDE00022005E075B021F0BD2081643002306E6C3
:10FDF00080273F031F433F033F0B1600004BFEE5E8
:10FE0000FF0700001E0400003E040000F8B557463E
:10FE10004E464546DE460C000903E0B5490A460F4A
:10FE20005F0031431E03DB0F760A9B46530F3343BB
:10FE3000C84E6500C000E40FD2006D0DA246814699
:10FE40007F0D9C469046B74200D1B9E05B46012643
:10FE500073409B46EE1BA34500D183E0002E63DD7B
:10FE6000002F00D0B1E06346134300D123E1731E9D
:10FE7000002B00D0BAE1861A6346B04280410125CA
:10FE8000C91A4042091A0B0200D447E149024B0A41
:10FE900098464346002B00D189E1404600F00EFC15
:10FEA0000300083B1F2B00DD7CE120223000D21A2A
:10FEB0004146D040994002009E400A439D4200DDE9
:10FEC0006AE15D1B6B1C1F2B00DD94E120211000FB
:10FED0003500C91A8E40DA408840DD40711E8E41DF
:10FEE000110007222843002506433240002A09D08A
:10FEF0000F233340042B05D0331DB342B641764265
:10FF000089191E000B0200D43DE26A1C914B550575
:10FF10006D0D9A4200D119E18F4AF6080A40570741
:10FF200052023743120B9BE0002E00D0C5E06E1C3E
:10FF30007605760D012E00DC48E16746861ACB1B5C
:10FF4000B042BF417F42B8461F004346FF1A3B0004
:10FF5000B8461B0200D55FE137439AD10022002446
:10FF6000002579E0002E00DCFAE0002F00D18DE0C2
:10FF7000784B9D4267D0802367461B041F43BC46D5
:10FF8000382E00DC52E1634613435A1E93411E187B
:10FF900086428041404209180B0200D4BEE06D4BFE
:10FFA00001359D4200D1D2E06B4A73080A4001211D
:10FFB0000E401E435108D30707221E43324095E7E7
:10FFC0001E00164300D045E740E7624B9D423AD001
:10FFD000802367461B041F43BC46382E00DDEBE040
:10FFE0001F2E00DC3AE133006746203BDF403B0038
:10FFF000202E05D04027BF1B6646BE4032439046A8
:020000021000EC
:100000004646721E96413343DAE0002B00D114E2DB
:100010006346134300D168E180234E07C008C90836
:100020001B030643194208D06046C008184204D199
:1000300063460100D2085E071643F3009946C900E3
:10004000720F444D11434B46DE08424B4F07374376
:10005000CA089D4200D16EE012036D05120B6D0DB2
:1000600000211203130B0A0D12051A433B4B2D05F9
:1000700013402B435B00E4075B082343380019005F
:100080003CBC90469946A246AB46F8BD6346134336
:1000900011D0731E002B00D007E1861886428041E4
:1000A00061444042091801250B0237D502257BE740
:1000B0003E00614691463500C5E75C46002D00D004
:1000C000E1E00B000343F3D0731C00D1ACE1214B02
:1000D0009F4200D13AE1F343382B00DD6FE11F2B43
:1000E00000DD8CE120250E00ED1AAE40B046060082
:1000F000AA46DE40454635432E005546D940A84025
:100100006346451EA8415B1A9C463043161AB2420C
:10011000924163465242991A3D00B4E607223240AA
:10012000002A00D0E4E60B4BF6084F073743CA0815
:100130009D4200D090E73B00134300D1A6E180230D
:100140001B031A431203120B024D89E7150000220C
:10015000002785E7FF070000FFFF7FFFFFFF0F80FD
:10016000002E00D0C7E06B1C5E05760D012E00DC72
:10017000F0E0C84DAB4200D1B9E085180A008542D5
:1001800089416244494251180722CE076D082E4327
:10019000490832401D00A9E6BF49ED1A1140072267
:1001A0003240A3E6320028388240002686E630003E
:1001B00000F084FA203073E6634613435A1E9341DD
:1001C000C61AB04280414042091A5CE60E006746FA
:1001D00006431743002D5ED1002E00D0F3E0002F20
:1001E00000D11EE15C46614691462CE7A94FBE4214
:1001F0007BD01E00F1E610001F3DE840202B03D00D
:100200004021CB1A9A401643731E9E410722064393
:1002100032400021002583E7161A6346B24280412E
:10022000591A40420B1A98465C4632E61F2E00DDF2
:10023000ABE02027BB1B9A4663465746BB40994616
:1002400013004F46F3401F433B005746BA40571E2A
:10025000BA4113436246F240891898E62027BB1B37
:100260009A4663465746BB40994613004F46F340B3
:100270001F433B005746BA40571EBA4113436246DC
:10028000F240891A9CE7834B9F425FD080252D0462
:100290007342294320E7002E0CD1002F00D1D0E07B
:1002A0005C46614691467B4DCDE67A4FBE421CD0FE
:1002B0001E0065E6002F18D0C0084E0706438020B8
:1002C000C9080003014208D06346DC08044204D197
:1002D0002100DA46D2085E071643F300994601244E
:1002E0005346C900720F11431C406A4DABE61D0016
:1002F00000220027B4E6002D59D10B00034300D1A2
:10030000D6E6731C00D1B2E0624B9F421ED0F3438D
:10031000382B6FDC1F2B00DD97E020250E00ED1A37
:10032000AE40B0460600AA46DE40454635432E00A4
:100330005546A840D940451EA8418C440643B618EE
:1003400096429241514261443D0025E63D0061469E
:10035000914678E60B000343002D00D055E6002BB4
:10036000F5D06346134300D16DE68618864280417E
:1003700061444042091800220B0200D4D0E6464BEB
:1003800001351940B2E5B1465DE633006746203BD2
:10039000DF403B00202E05D04027BF1B6646BE40F5
:1003A000324390464646721E96413343EFE5394B41
:1003B0009F42CBD080252D0473422943A8E70843F0
:1003C000411E8841A2E6002F00D13CE66346861A12
:1003D000CF1AB0429B415B42FB1A98461B024ED596
:1003E000161A6346B2429241591A5242891A5C4621
:1003F00000227BE501430E00711E8E419FE71D0028
:100400000E00203DEE40B046202B04D04025EB1AD4
:1004100099400843814648464346411E8841184357
:1004200074E60022002417E6161A6346B24292418F
:10043000591A5242891A3D0025E561469146154DEB
:1004400001E680220024120379E61D000E00203D03
:10045000EE40B046202B04D04025EB1A99400843CB
:1004600081464E464346711E8E411E4367E78618FD
:1004700096429B4161445B42C9183D008CE547466A
:100480003743CED007224146324049E600273A00A2
:10049000E6E5C046FF070000FFFF7FFF70B50C4E8A
:1004A0000D031C0349005B002D0B490D240B5B0D54
:1004B000B14208D0064900208B4203D114432000EA
:1004C000441EA04170BD05430120002DFAD1F1E783
:1004D000FF07000030B5144D0A034B00120B5B0DF3
:1004E000C90F0024AB4211DD104CA34210DC802464
:1004F000640322430E4CE41A1F2C0CDD0D48C31A72
:10050000DA4013005C42002900D11C00200030BDFD
:10051000094BCC18FAE7094DE040AC4663449A40D9
:1005200013000343EEE7C046FE0300001D04000075
:100530003304000013040000FFFFFF7FEDFBFFFF0B
:1005400070B500282DD0C317C5185D40C40F280012
:1005500000F0B4F8154B1B1A5B055B0D0A2815DD7E
:100560000B38854000222D032D0B002110002D0398
:100570000A0D2D0B12052A430D4D1B052A4013436E
:100580005B00E4075B082343190070BD02002900EB
:10059000153291400A000B21081AC5402D032D0B7E
:1005A000E3E70024002300250022DEE71E0400000C
:1005B000FFFF0F8010B5041E25D000F07FF8144B0C
:1005C0001B1A5B055B0D0A2812DD0B3884400022E4
:1005D0002403240B0021100024030A0D240B120510
:1005E00022430C4C1B05224013435B00590810BDED
:1005F00002002100153291400A000B21081AC44064
:100600002403240BE6E7002300240022E2E7C0468F
:100610001E040000FFFF0F804100090E4B1C70B547
:10062000DBB24602750AC40F012B14DDE0239B00E8
:100630006D07360BCB1800210A0D280012051C4D42
:1006400032435B052A405B0813435B00E4075B0809
:100650002343190070BD002914D1002D1ED028009D
:1006600000F02CF80A281CDC0B232A001B1ADA40A5
:10067000030015339D400F4B12031B1A5B05160B2D
:100680005B0DD8E7002D06D0320B802636036D07B0
:100690001643094BCFE7084B0026CCE70023002682
:1006A000C9E703002A000B3B9A400025E3E7C04658
:1006B000FFFF0F8089030000FF0700001C210123BA
:1006C0001B04984201D3000C10391B0A984201D335
:1006D000000A08391B09984201D30009043902A213
:1006E000105C40187047C04604030202010101017A
:1006F000000000000000000010B5002903D1FFF742
:10070000DDFF203002E0081CFFF7D8FF10BDC04617
:1007100010B50A22002100F0BFFE10BD10B5040084
:1007200004481300002804D00A000220210000E041
:1007300000BF10BD0000000070B500260C4D0D4C30
:10074000641BA410A64209D1002602F0E3F90A4D69
:100750000A4C641BA410A64205D170BDB300EB582F
:1007600098470136EEE7B300EB5898470136F2E7B9
:100770001802002018020020180200204402002065
:1007800010B5040000F008F808230019407818405C
:1007900010BDEC3000687047044B1B681B6A002BCF
:1007A00000D1034BEC3318687047C0464800002066
:1007B000AC00002010B5034B0100186800F09EF853
:1007C00010BDC0464800002010B5034B010018685A
:1007D00000F04AF810BDC0464800002082B0002951
:1007E00000D101A9101E06D0002B06D013780B6093
:1007F0001078431E984102B0704702204042FAE749
:1008000030B50024A24201D1002005E0035D651C43
:100810000C5DA34201D0181B30BD2C00F2E7002371
:1008200010B59A4200D110BDCC5CC4540133F8E736
:1008300010B5884202D98B18984203D3002307E0F1
:100840008B5C8354013AFBD210BDCC5CC4540133A1
:100850009A42FAD1F8E703001218934200D1704788
:1008600019700133F9E7000070B50500002910D0B8
:100870000C1F2368002B00DAE418280001F0B7FCF5
:100880001D4A1368002B05D163601460280001F035
:10089000AFFC70BDA34209D9216860188342F3D12F
:1008A00018685B6841182160EEE713005A68002A57
:1008B00001D0A242F9D919685818A0420BD120687A
:1008C0000918581819608242E0D11068526841181E
:1008D00019605A60DAE7A04202D90C232B60D5E7F1
:1008E00021686018824203D1106852684118216063
:1008F00062605C60CAE7C046AC200020032370B58C
:10090000CD1C9D43083506000C2D1ED20C25A94296
:100910001DD8300001F06BFC254A14682100002925
:1009200019D1244C2368002B03D1300000F0ACFC1B
:1009300020602900300000F0A7FC431C2BD10C23C1
:100940003000336001F054FC03E0002DDFDA0C23AB
:100950003360002070BD0B685B1B19D40B2B03D9CF
:100960000B60CC18256003E04B688C420DD11360FE
:10097000300001F03DFC200007220B30231D904386
:10098000C31AE7D05A42E250E4E763600C00EFE795
:100990000C004968C3E70323C41C9C43A042E1D078
:1009A000211A300000F070FC431CDBD1C7E7C046C1
:1009B000AC200020B0200020F0B58BB014001D1E2C
:1009C000129953DA802424061B191D0014002D23CC
:1009D0000B702023149E03229E43462E07D0330023
:1009E000453B59424B411099013ACB18109309AB42
:1009F000049308AB0393139B00920293109B220075
:100A000001932B0000F0FCFD0700472E02D1119B43
:100A1000DB0724D5109BFB180793462E14D13B7897
:100A2000302B0CD10022002320002900FDF77AFB97
:100A3000002804D10123109A9B1A139A1360139B68
:100A4000079A1B68D318079300220023200029006F
:100A5000FDF768FB302200280DD0079B0993380072
:100A6000099B159ADB1B13600BB0F0BD0023AFE7A9
:100A7000591C09911A70099B07998B42F8D3EEE72C
:100A8000F0B5831C85B0019306000C0002702B2387
:100A9000002901DA2D234C427370092C22DD02ABB0
:100AA000DD1D20000A21FDF727FB6F1E3031397054
:100AB00020000A21FDF73AFA040009280BDC023D68
:100AC0003034019B2C7002AA07321800AA4204D8C5
:100AD000801B05B0F0BD3D00E3E72A7801351A70B0
:100AE0000133F0E73023E418B370301DF470EFE702
:100AF000F0B595B00C000A920B931A9D099001F085
:100B00005FFB036818000C9300F010FC00231293A5
:100B100023680E900D930D99277E2B680722C90537
:100B200045D59B1893431A0008322A601A685B68FF
:100B3000A264E3640122E56CA66C6B005B080F9372
:100B40005242AC4B30000F99FFF7A8FC002830D17F
:100B50000122A84B524230000F99FDF7F3FA00280A
:100B600027D10022002330002900FDF7E1FA0028F8
:100B700003D023002D2243331A709F4D472F00D8F6
:100B80009E4D032300260D9A236101339A43226070
:100B90000B9B13AA009321000A9B099800F0F4F91B
:100BA000431C00D093E00120404215B0F0BD073354
:100BB000B8E732002B0030002900FFF76FFC002857
:100BC00004D08F4D472FDCD88E4DDAE780230D9966
:100BD0006268DB000B43511C43D10732626012AAEA
:100BE0000021059211AA039223222360069101930A
:100BF00008A9636852180292009332002B000497F0
:100C00000998FFF7D9FE20233A0005009A43472AA6
:100C100007D1119BDA1C02DB6268934245DD023F7B
:100C2000FFB21199652F25D8200001393A005030C4
:100C30001191FFF725FF129A060013182361012A6C
:100C400002DC2268D20701D501332361232308AADD
:100C50009B181B78002B9BD023002D2243331A7046
:100C600096E7672F00D176E1472FB8D1002AB6D199
:100C70000122B3E7662F19D1636800290CDD2161D9
:100C8000002B02D12268D20702D501335B18236101
:100C9000119B0026A365D9E7002B03D1012221680F
:100CA000114200D09A1C2261F2E76727119B129A29
:100CB000934205DB22682361D207E9D50133E6E7D9
:100CC0000121002B01DC4918C91A5218EBE72268F0
:100CD000530508D423692A000A9909980B9DA8474F
:100CE000431C29D15FE7652F00D8E0E0A06CE16CE0
:100CF00000220023FDF716FA002834D00123424ACF
:100D00000A9909980B9DA847431C00D14BE7119BFA
:100D1000129A934202DB2368DB070DD50B9D0E9BD5
:100D20000C9A0A990998A8470025431C00D13AE774
:100D3000129B013BAB420ADC23689B0700D508E10C
:100D4000139BE068984200DB2FE718002DE7220094
:100D500001231A320A9909980B9EB047431C00D10F
:100D600021E70135E4E7119B002B2DDC0123264A06
:100D70000A9909980B9EB047431C00D113E7119BB9
:100D8000002B05D1129B002B02D12368DB07D3D5A2
:100D90000B9E0E9B0C9A0A990998B0470026431C9B
:100DA00000D100E7119B5B42B34201DC129B92E74A
:100DB000220001231A320A9909980B9FB847431C55
:100DC00000D1F0E60136EDE7A36D129F9F4200DDF2
:100DD0001F00002F08DD3B002A000A9909980B9E8E
:100DE000B047431C00D1DEE600230D93FB43DB1725
:100DF0000F9318E0FFFFEF7FD4470100D0470100B9
:100E0000DC470100D84701002338010022000123FC
:100E10001A320A9909980B9EB047431C00D1C2E6CA
:100E20000D9B01330D930F9BA66D0D9A3B40F31A5A
:100E30009342EBDC119B129AAD19934210DB2368AD
:100E4000DB070DD4129F119BBE1BFF1AB74200DDBA
:100E50003700002F0DDCFE43F31700250C931CE038
:100E60000E9B0C9A0A9909980B9FB847431CE9D12D
:100E700099E63B002A000A9909980B9DA847431C54
:100E8000E9D190E6220001231A320A9909980B9EB3
:100E9000B047431C00D186E60135119A129B0C998C
:100EA0009B1A3A000A409B1AAB42EBDC44E7129BC8
:100EB000012B02DC01231A4232D001232A000A99B5
:100EC00009980B9FB847431C00D16CE60E9B0C9A07
:100ED0000A9909980B9F0135B847431C00D162E677
:100EE000A06CE16C129B00225F1E0023FDF71AF933
:100EF0003B00002814D000250AE0220001231A320A
:100F00000A9909980B9FB847431C00D14BE601355D
:100F1000129B013BAB42F0DC220033005032DBE697
:100F20002A000A9909980B9DA847431CF4D13AE678
:100F30002200012319320A9909980B9EB047431CDD
:100F400000D130E60135E368139A9B1AAB42EFDC1F
:100F5000F6E60025F7E7002A00D189E60021069190
:100F600012A9059111A90391232108A8091823604A
:100F7000019300922B000497029132000998FFF729
:100F80001BFD050045E6C046F7B5150001938A68CC
:100F90000B6900900C00934200DA130022002B60D2
:100FA00043321278002A01D001332B6023689B065C
:100FB00002D52B6802332B60062723681F4027D0F9
:100FC000230043331B785A1E93412268920630D483
:100FD0002200019943320098089EB047431C25D057
:100FE000062320682A68E16803400025042B03D10A
:100FF0008D1AEB43DB171D40A3682269934201DD84
:101000009B1AED180027BD4220D1002010E00137C7
:10101000E3682A689B1ABB42D2DD22000123193201
:1010200001990098089EB047431CF0D1012040422E
:10103000FEBD3020E1184331087021005A1C4531B3
:101040000978A218433202331170C1E7220001234C
:101050001A3201990098089EB047431CE6D0013728
:10106000D1E70000F0B589B004920A00433205933D
:10107000039002920A7E0C000E9B6E2A00D186E03D
:101080001FD8632A33D008D8002A00D18CE0582A10
:101090004DD0250042352A7030E0642A01D0692AFB
:1010A000F7D1196825680A1D280629D508681A602D
:1010B000002803DA2D23029A404213706B4E0A2750
:1010C0004FE0732A74D008D86F2A1FD0702AE0D15D
:1010D000202209680A43226003E0752A16D0782A84
:1010E000D7D12200782145321170614E22E02500CF
:1010F0001A684235111D196013682B70012365E0D1
:1011000008681A606906D3D500B2D1E71968256866
:10111000081D186008682E0605D5544E08276F2A4A
:101120001BD00A2719E06D06F7D580B2F5E74531E7
:101130004E4E0A7018682268011D00681960150675
:1011400021D5D30702D520231A4322601027002877
:1011500003D1202322689A432260230000224333D4
:101160001A706368A360002B58DB04222168914346
:101170002160002854D1029D002B5AD025003378DD
:1011800042352B7055E05506DBD580B2D9E71A6899
:101190000D68101D4969186013682E0601D5196085
:1011A00002E06D06FBD519800023029D23614FE00C
:1011B0001A68111D1960156800216268280001F085
:1011C0000BF8002801D0401B606063682361002396
:1011D000029A13703CE023692A0004990398059D44
:1011E000A847431C3ED023689B0715D4079BE068A3
:1011F000984239DA180037E02200012319320499A5
:101200000398059EB047431C2CD00135E368079A2C
:101210009B1AAB42F0DCE9E70025F7E70028ADD0E8
:10122000029D3900FCF77EFE735C013D2B700028A7
:10123000F7D1082F09D12368DB0706D56368226937
:10124000934202DC3023013D2B70029B5B1B236128
:10125000059B07AA00932100049B0398FFF794FEC7
:10126000431CB8D10120404209B0F0BDE047010065
:10127000F147010010B5034B0A000100186801F0A6
:10128000ADFA10BD48000020002370B5064C0500E3
:101290000800236001F030FC431C03D12368002BBD
:1012A00000D02B6070BDC046B82000200EB400B541
:1012B0000B499CB01DAB0290069007910491094820
:1012C000094904CB0591006802A9019301F00EFBC6
:1012D0000023029A13701CB008BC03B01847C04624
:1012E000FFFFFF7F480000200802FFFFC9B203781C
:1012F000002B04D08B4200D170470130F7E74B42FE
:10130000594149420840F7E702780B78002A03D098
:10131000013001319A42F7D0D01A704703000A78A1
:1013200001311A700133002AF9D170470023C25CE1
:101330000133002AFBD1581E704730B50500002A42
:1013400000D130BD0C78013A6B1C2C700131002C9F
:1013500005D19A189A42F4D01C700133FAE71D00A7
:10136000EDE710B50378002B0FD10B785A425341AB
:101370005B42184010BD0023CA5C002AFAD0C45C4E
:10138000944201D10133F7E701300378002BF2D109
:101390001800EFE7F0B51F000E0087B0059001912F
:1013A00002920C983478FFF7F4F908220019437878
:1013B000751C134036D12D2C36D1B51C74780126FE
:1013C000002F62D0102F09D1302C07D120222B788A
:1013D0009343582B54D110276C7802352D4B39008C
:1013E000F31818000393FCF79DFD049101210023DD
:1013F000494202008C4618002100303909291AD8C8
:101400000C00A74223DD591C09D06346824206D353
:1014100002D10499A14202DB0123784320182C78E1
:101420000135E9E72E00BCE72B2C01D01E00C7E7F1
:10143000B51C7478FAE721004139192901D8373CE5
:10144000DFE721006139192901D8573CD9E75A1C37
:1014500008D1059A23331360029B0398002B09D10E
:1014600007B0F0BD002E00D04042029A002AF7D00B
:10147000002B01D06B1E0193029B019A1A60EFE7CB
:101480003024002FAAD10827A8E7302C9ED00A27A5
:10149000A4E7C046FFFFFF7F37B51300064A0500EB
:1014A0001068046A002C00D1044C0A000094290042
:1014B000FFF770FF3EBDC04648000020AC00002092
:1014C00010B50400FFF768F90322001943781340B0
:1014D000012B00D12034200010BD0B1E04D0FF2AA8
:1014E00004D98A2303608B3B180070470A700123DC
:1014F000FAE7F0B503690C6989B007000591002689
:10150000A34265DB0B00013C1433A50003935B1978
:1015100004930300143302935D19049B28681B682D
:10152000591C0193FCF778FC0190B04229D0039B31
:1015300002989C460696624608CA9446019A99B259
:1015400051431B0C534389190A0C9B1807931E0C1B
:10155000036889B29AB2069BD2180368521A190C12
:101560006B469B8BCB1A11145B18191492B21B0497
:101570001A43049B069104C06345DCD22B68002B00
:101580002DD00599380001F049F800281FDB00250F
:10159000019B0298013303990193026808C992B232
:1015A00055199AB2AA1A05681B0C2D0CEB1A1514C2
:1015B0005B191D1492B21B04134308C0049B8B4299
:1015C000EBD2029AA300D3181A68002A11D0019E08
:1015D000300009B0F0BD2B68002B04D1013C029B08
:1015E000043DAB42F7D33C61CBE71A68002A04D133
:1015F000013C029A043B9A42F7D33C61E7E70000C2
:10160000F0B516001F00446A9BB00290239D069619
:101610000797002C08D11020FFF7CCF8029B5862E6
:10162000446084600460C460029B5B6A196800299E
:101630000BD05A68012393404A608B60029800F0F7
:1016400010FE0022029B5B6A1A60002F20DA012341
:101650002B607B005B080793079CB24B220017931B
:101660001A409A4217D1B04B229A1360069B002B66
:1016700003D1240301D100F087FDAC4B249A0893D9
:10168000002A02D0AA4B249A136008981BB0F0BD20
:1016900000232B60E0E7069E079F00220023300016
:1016A0003900FCF73FFD051E0BD00123229A136081
:1016B000A04B249A0893002AE7D09F4A24990A60F5
:1016C000E3E718AB019319AB009332003B0002989B
:1016D00001F022F8630003905B0D74D03A03974C3D
:1016E000120B14432100964A300016959E180022D2
:1016F000944BFEF78BFB944A944BFEF715F9944AF2
:10170000944BFDF7EBF9040030000D00FEF718FFD5
:10171000914A924BFEF708F902000B0020002900C5
:10172000FDF7DCF904000D00FEF7D4FE00220700EF
:10173000002320002900FCF7FBFC002809D038001A
:10174000FEF7FEFE2B002200FCF7ECFC4342584162
:101750003F1A01231493162F0DD88149FB00C91895
:1017600008684968069A079BFCF7F6FC002846D0F3
:101770000023013F1493189B9E1B00230A93330000
:10178000013B0B9304D501239B1B0A9300230B936E
:10179000002F36DB0B9B1197DB190B93002304936F
:1017A000209B0124092B00D984E0052B02DD0024B5
:1017B000043B2093209B981E032800D984E0FCF76B
:1017C00021FB7577286A189B199A9E18654BF218A9
:1017D000202A0FDD40239B1A9C40634B0698F31888
:1017E000D8402043FEF7E6FE0123604C013E091974
:1017F00016937CE7202306989B1A9840F2E71490F2
:10180000B9E70A9BDB1B0A937B42049300231193E5
:10181000C6E701230D93219B002B59DD0C930993FF
:10182000029A556A00226A60043210001430696816
:10183000984252D9029800F0DCFC029B28605B6A57
:101840001B680893099B0E2B00D90AE1002C00D1DC
:1018500007E1069B079C12931394002F00DC89E09C
:101860000F213A003E4B0A40D2009B181D685E686B
:1018700002233C110E93E3060BD53D4B0C401A6A34
:101880005B6A12981399FDF745FC032306900791B4
:101890000E9300233AE001230D93219BFB180C9338
:1018A00001330993002BBBDC0123B9E70023B1E727
:1018B0000023F1E700230D942093013B00220C93B9
:1018C000099313332192ABE701230D93023BF5E714
:1018D00001230C9309931A00F4E701316960520067
:1018E000A3E701231C420ED00E9B214A01330E9325
:1018F000109B2800DB009B1831001A685B68FEF71C
:1019000013F805000E00109B641001331093002C97
:10191000E7D1069807992A003300FDF7FBFB0690F4
:10192000079142E00000F07F0F2700000C49010002
:101930000F49010023380100243801000000F03F66
:1019400001FCFFFF0000F83F61436F63A787D23FB0
:10195000B3C8608B288AC63FFB799F501344D33F9E
:10196000984901003204000012040000000010FE3B
:101970007049010002230E93002F16D0129813997C
:101980007C420D332340CE4ADB00D3181A685B68D3
:10199000FDF7CAFF002301261D00069007912411C0
:1019A000002C00D08CE0002BB9D1149B002B00D16F
:1019B00096E0069C079D0022C24B20002900FCF700
:1019C000B7FB002800D18BE0099B002B00D187E0FA
:1019D0000C9B002B41DDBC4B002220002900FDF7B1
:1019E000A3FF0E9B0690079101330E930C9B7E1E66
:1019F0000E981093FEF7A4FD069A079BFDF794FF3F
:101A00000022B24BFDF76AF8B14A0E900F910E9C7E
:101A10000F9D94460F9B634415931D00109B002B54
:101A200061D1069807990022AA4BFEF7EFF9220030
:101A3000159B06900791FCF78FFB002800D0A8E2C9
:101A4000A5480F99844661440B0006980799220027
:101A5000FCF76EFB002800D095E2129B139C0693C6
:101A60000794199B002B00DA5CE10E2F00DD59E191
:101A7000934BFA009B185C681B6804930594219BA8
:101A8000002B00DBD8E0099B002B00DDD4E000D068
:101A90007DE20498059900228E4BFDF745FF069ADA
:101AA000079BFCF763FB099B04931E00002800D0F2
:101AB0004FE2089B089A5D1C3123013713704BE2FB
:101AC00034420AD00E9B854A01330E93EB009B18DB
:101AD0001A685B68FDF728FF3300641001355FE783
:101AE0003E00099B84E7109B0D995A1E744BD2004F
:101AF0009B181A685B68002949D000207849FDF7D7
:101B000009FB2B002200FEF781F9089B0E900F9134
:101B1000159306980799FEF7DDFC0400FEF710FD0B
:101B200002000B0006980799FEF770F9159B3034F8
:101B30005D1C1C700E9A0F9B06900791FCF7F8FA3B
:101B400000286CD1069A079B00205E49FEF75EF9DB
:101B50000E9A0F9BFCF7ECFA002800D0C3E0089B1C
:101B6000109AEB1A9A4200DC77E70E980F99002240
:101B7000554BFDF7D9FE00220E900F91069807995C
:101B8000514BFDF7D1FE159506900791C1E7200056
:101B90002900FDF7C9FE089C109A230094460E9078
:101BA0000F916344159306980799FEF793FC05007F
:101BB000FEF7C6FC0B00020006980799FEF726F90F
:101BC0003035159B2570013406900791A3422AD128
:101BD0000E980F99089A109B9446634400221D00AA
:101BE0003F4BFCF77BFF02000B0006980799FCF7C0
:101BF000B3FA002800D076E00E9A0F9B00203849F7
:101C0000FEF704F902000B0006980799FCF790FA1A
:101C1000002800D121E76B1E1A78302A01D0370046
:101C20003FE01D00F7E7069807990022264BFDF7D5
:101C30007BFE06900791B6E7089E049A059B0698DE
:101C40000799FDF767FAFEF745FC0400FEF778FCFC
:101C5000049A059BFDF768FE02000B0006980799A1
:101C6000FEF7D4F8230030333370099A089B751CB3
:101C7000EB1A9A4248D102000B00FCF72FFF049A9E
:101C8000059B06900791FCF767FA00282AD1049A71
:101C9000059B06980799FCF745FA002801D0E30751
:101CA00020D40399029800F0DCFA00232B70229BC9
:101CB00001371F60249B002B00D1E6E41D60E4E4A3
:101CC000984901000000F03F0000244000001C4043
:101CD0000000C0FC000014400000C07C70490100FE
:101CE0000000E03F3E006B1E1A78392A06D1089AA0
:101CF0009A4207D130231370130001361A7801324B
:101D00001A708CE71D00EEE70022A44BFDF70CFED5
:101D100000220023069007912E00FCF703FA00280A
:101D20008BD0BEE70D9A002A00D1DAE0209A012A72
:101D300000DDBDE0169A002A00D1B5E0984A9B1854
:101D4000049D0A9C0A9A0121D2180A920B9A0298C1
:101D5000D3180B9300F025FB0600002C0EDD0B9B27
:101D6000002B0BDD0B9A2300944200DD13000A9A2E
:101D7000E41AD21A0A920B9AD31A0B93049B002BE3
:101D80001FD00D9B002B00D1AFE0002D11D03100F2
:101D90002A00029800F09EFB039A010006000298B8
:101DA00000F008FB03991090029800F05AFA109B7B
:101DB0000393049B5A1B04D00399029800F08AFBFA
:101DC00003900121029800F0ECFA119B0490002B83
:101DD00000D1E3E11A000100029800F07BFB209B98
:101DE0000490012B00DD82E00025069BAB420ED162
:101DF000079B1B03AB420AD1179B079A134206D0DD
:101E00000A9B013501330A930B9B01330B93119B02
:101E10000120002B6CD10B9B18181F2318407ED07B
:101E200001331B1A042B70DD1C23181A0A9B24187B
:101E30001B180A930B9B1B180B930A9B002B05DDA9
:101E40001A000399029800F097FB03900B9B002B5C
:101E500005DD1A000499029800F08EFB0490149B93
:101E6000002B5ED00499039800F0D8FB002858DAC4
:101E700000230A220399029800F00CFA0D9B013FFF
:101E80000390002B00D190E1002331000A22029838
:101E900000F000FA0C9B0600002B00DD88E0209B80
:101EA000022B00DC84E044E03623189A9B1A47E7B3
:101EB000099B5D1E049BAB4208DB5D1B099B002B4D
:101EC0000CDA0A9B099A9C1A00233BE7049B0495B1
:101ED000EA1A119B00259B181193EFE70A9C099BB6
:101EE00030E7049D0A9C0D9E37E7049A64E70025BD
:101EF000049B049A1B69109303339B00D318586802
:101F000000F006FA2023181A85E7042B95D00A9AC8
:101F10001C33D2180A920B9AE418D3188CE70300EA
:101F2000F5E7099B002B3DDC209B022B3ADD099B4A
:101F30000C930C9B002B0CD104990522029800F005
:101F4000A9F904900100039800F068FB002800DD67
:101F5000AFE5219B089DDF43002309930499029874
:101F600000F07FF9002E00D19BE6099B002B05D0E5
:101F7000B34203D01900029800F073F931000298BF
:101F800000F06FF98DE6109B04931E00E1E700233B
:101F9000FAE7109B370004931E008AE500002440F6
:101FA000330400000D9B002B00D1B2E0099B0C9381
:101FB000002C05DD31002200029800F0DDFA060059
:101FC0003000002D11D07168029800F012F9310034
:101FD000040033690C319A1C92000C30FEF71FFC90
:101FE00001222100029800F0C7FA09960600089B1A
:101FF0000A9304990398FFF77CFA09990D9004005D
:10200000039800F00BFB320010900499029800F046
:102010001FFB01230B93C36830340500002B04D150
:102020000100039800F0FAFA0B902900029800F0E2
:1020300018F90B9B209A13430ED1069A01331342D1
:102040000AD1392C26D0109B002B01DD0D9C313498
:102050000A9B5D1C1C7081E7109B002B07DB1D0099
:10206000209B1D4322D10123069A13421ED10B9BB4
:10207000002BEDDD03990122029800F07DFA04990E
:10208000039000F0CBFA002802DCE1D1E307DFD5B2
:10209000392CDBD10A9B0A9A5D1C392313706B1E05
:1020A0001A78392A67D001321A7057E70A9B5D1CEB
:1020B0000B9B002B04DD392CECD001340A9BC9E7C3
:1020C0000A9B0C9A1C70089BEB1A93423ED000238B
:1020D0000A220399029800F0DDF8099B0390B342AD
:1020E00009D100230A220999029800F0D3F8099037
:1020F00006000A957DE7099900230A22029800F05C
:10210000C9F8002309900A223100029800F0C2F8B1
:10211000EEE7099B0C93089B069304990398FFF73D
:10212000E8F9069B30305D1C18700C9A089B04007F
:10213000EB1A9A4208DD00230A220399029800F064
:10214000A9F806950390E8E7002309930399012273
:10215000029800F011FA0499039000F05FFA002849
:102160009DDC01D1E3079AD46B1E1A78302A00D087
:10217000F4E61D00F8E7089A9A4203D131230137AB
:102180001370EBE61D008AE70B4B249A08930B4B68
:10219000002A01D0FFF777FAFFF777FA209B012B8F
:1021A00000DC21E6119D012035E60C9B002BB2DC02
:1021B000209B022BAFDDBCE6034901000B49010067
:1021C000034B1B68186A002800D10248F0307047A2
:1021D00048000020AC000020C9B28218904201D112
:1021E0000020704703788B42FBD00130F6E7704740
:1021F000704770B5466A04000D00002E07D110200C
:10220000FEF7D8FA6062466086600660C660666A5D
:10221000F368002B13D0636AAA00DB689B18186868
:10222000002818D101210E00AE40721D920020003E
:1022300000F0C6FA00280CD0456086600DE021222F
:102240000421200000F0BCFA636AF060DB68002B18
:10225000E1D1002070BD02681A6000230361C360F1
:10226000F8E770B5446A06000D00002C07D1102075
:10227000FEF7A0FA7062446084600460C460002DC0
:1022800007D0736A6A68DB6892009B181A682A6034
:102290001D6070BDF7B51E0014239C4607000C009E
:1022A00000200D698C4463461B68013099B2634677
:1022B0001B6851431B0C534389190E0C9B1989B29F
:1022C0001E0C1B045B18614608C18C468542EADC83
:1022D000002E1BD0A368AB4212DC63683800591C87
:1022E000FFF787FF2100236901909A1C92000C31AF
:1022F0000C30FEF794FA21003800FFF7B2FF019C82
:102300002B1D9B00E31801355E6025612000FEBD9A
:102310000300020C0020824201D11B0410301A0E6F
:1023200001D108301B021A0F01D104301B019A0F92
:1023300001D102309B00002B03DB01305B0000D495
:10234000202070470722036810B501001A400DD005
:1023500001240020234205D10230034203D0E34090
:1023600020000B6010BD9B080B60FBE79CB21000C7
:10237000002C01D110201B0CDAB2002A01D1083048
:102380001B0A1A0701D104301B099A0701D1023038
:102390009B08DA07E8D45B0801D00130E4E720208D
:1023A000E0E710B50C000121FFF723FF0123446192
:1023B000036110BDF0B50B691400126989B00D00FE
:1023C000934201DA25000C002F6926696968BB1960
:1023D0000293AB68BA19934200DA0131FFF709FFA3
:1023E0000200BB1914329B00D3189C460021130035
:1023F000049063451DD31435BF00EB191434B600A7
:102400000593A319039501940793079B019999429A
:1024100011D3029B002B06DD04235B429C446346E0
:102420001B68002B51D0049B029A18001A6109B056
:10243000F0BD02C3DDE7019B1B6898B200281CD0E9
:1024400015000026039F02CF2C688BB24343090C72
:102450004143A4B21B199B190E0029680695090C6B
:1024600071181E0C89190E0C9BB209040B4308C588
:10247000059BBB42E7D8069B5E60019B1B681D0C59
:102480001ED0100000271368039E3168046889B2CB
:102490006943240C0919C9190F049BB23B4303601B
:1024A00080CE43683F0C6F439BB2FB18090C5B184E
:1024B000059906901F0C0430B142E6D806994B608E
:1024C000019B0432043301939FE7029B013B02937B
:1024D0009FE700000323F7B5134005000E0014002A
:1024E000002B08D02249013B9A00525800233100AA
:1024F000FFF7D0FE0600A310019336D06C6A002CC3
:1025000007D11020FEF756F96862446084600460C9
:10251000C4606F6ABC68002C07D116492800FFF719
:1025200040FF00230400B86003600122019B1342B6
:102530000AD0310022002800FFF73CFF07003100DD
:102540002800FFF78EFE3E00019B5B1001930CD02C
:102550002068002807D1220021002800FFF72AFF69
:102560000023206003600400DFE73000FEBDC046AA
:10257000604A010071020000F0B50D0017002B69E0
:10258000541185B0E3180193013300934968AB6897
:102590000290009A934235DB0298FFF72AFE00234F
:1025A0000200060019001432A3422EDBE343DB17BE
:1025B0001C402B00A40014192A69143392009A18A5
:1025C00094461F22174024D00132D21B03920022CE
:1025D00019682000B9400A4304C404CB0399CA40D7
:1025E0009C45F5D84260002A02D0019B023300933B
:1025F000009B0298013B33612900FFF732FE300057
:1026000005B0F0BD01315B00C3E798001150013304
:10261000CAE704CB04C49C45FBD8E9E70A6903690F
:1026200030B59B1A0DD192001430143184188918DA
:10263000043C043925680A68954204D00123954278
:1026400004D3180030BDA042F2D3FAE75B42F8E7AA
:10265000F0B50D0085B00700110028001400FFF749
:10266000DDFF061E08D101003800FFF7C2FD01237F
:102670004661036105B0F0BD01230193002804DB2E
:1026800023002C001D000023019361683800FFF730
:10269000B0FD2F000022019B2669C3601434B300F3
:1026A000E31802932B6914379B00FB180393030074
:1026B0009446143320CC04CF0192AAB294446A46C3
:1026C000614692882D0C8A1A0199090C691A151411
:1026D00049190D1492B209040A431A60039AAC46D0
:1026E0000433BA42E6D802991A008C4205D3043A60
:1026F0001368002B0ED00661BCE704CC91B2614494
:102700000D14120C5219151489B212040A43AC4666
:1027100004C3E8E7013EEAE7F7B51D000121140014
:10272000089FFFF766FD2B036D0006001B0B6D0D68
:1027300024D10193002C27D068460094FFF702FEB5
:10274000009C00281ED0019B20211A00091A8A40F3
:10275000C340224372610193019CB461631E9C419A
:1027600001343461002D18D0124BED1835232D188B
:102770003D60181A099B18603000FEBD802252038C
:102780001343D6E77461E7E701A8FFF7DBFD0124F7
:10279000019B346173612030E4E7074BC018074B9D
:1027A0003860E3189B00F3185869FFF7B1FD640126
:1027B000201ADFE7CDFBFFFFCEFBFFFFFFFFFF3F50
:1027C0004A4370B511001400FEF798F8051E03D0B7
:1027D00022000021FEF73FF8280070BDF8B5070081
:1027E0000D001600002905D11100FEF787F804003E
:1027F0002000F8BD002A03D1FEF736F83400F7E7D1
:1028000000F072F92C00B042F2D231003800FEF72D
:1028100075F8041EECD029003200FEF700F82900FC
:102820003800FEF721F8E3E7F0B58E6885B00700C1
:102830000C00039201939E423CD890238A89DB00CE
:102840001A4234D00325096923685B1A029363692D
:1028500002985D43EB0F5D19019B6D1001331B184E
:10286000AB4200D91D00530532D529003800FEF7D0
:1028700045F8061E09D10C233B6040230120A289A4
:1028800040421343A38105B0F0BD029A2169FDF7D0
:10289000C6FFA389144A1A4080231343A381029BD5
:1028A0002661F61826606561019EED1AA560019B00
:1028B0009E4200D9019E320003992068FDF7B8FFBF
:1028C000A36800209B1BA36023689E192660DAE79B
:1028D0002A003800FFF782FF061EE0D12169380088
:1028E000FDF7C2FFC7E7C0467FFBFFFFF0B59FB013
:1028F000029005938B890F0016001B0611D50B69FA
:10290000002B0ED14021FDF7F9FF38603861002817
:1029100005D10C23029A013813601FB0F0BD40238B
:102920007B61002306AC6361203363761033A376AA
:1029300035002B78002B01D0252B46D1AB1B0493FF
:102940000CD0320039000298FFF76EFF431C00D113
:10295000AEE06269049B9446634463612B78002B6C
:1029600000D1A5E0012200235242626002A9543244
:1029700052186E1C2360E360A3601370A365317866
:1029800005225448FFF728FC751C00281FD1226837
:10299000D30604D5532302A95B182021197013070D
:1029A00004D5532302A95B182B21197033782A2BE5
:1029B00016D0350000210A20E3682A786E1C303AD0
:1029C000092A4ED9002918D010E00135B1E7414B52
:1029D0002268C01A01238340134323602E00CEE7F0
:1029E000059B191D1B680591002B01DB099304E071
:1029F0005B42E3600223134323602B782E2B0AD122
:102A00006B782A2B35D1059B02351A1D1B68059260
:102A1000002B2BDB0793304E297803223000FFF781
:102A2000DBFB002806D04023801B83402268013551
:102A3000134323602978062228486E1C2176FFF76D
:102A4000CBFB00283CD0264B002B25D10722059B31
:102A500007339343083305936369039A9B186361B3
:102A600066E7434301219B183500A6E701235B423B
:102A7000D0E700230A201A000135636029786E1C14
:102A80003039092903D9002BC5D00792C3E7424347
:102A9000012352183500F1E705AB00933A00114BC2
:102AA00021000298FEF724F80390039B0133D3D151
:102AB000BB890B985B0600D42FE7012040422CE72E
:102AC00005AB00933A00074B21000298FEF7CAFAC3
:102AD000EAE7C0466C4A0100724A0100764A0100EA
:102AE000F10A0100292801000B1F1B68181F002B89
:102AF00001DA0B58C0187047044A1368002B00D144
:102B0000034B1818106018007047C046B42000200E
:102B1000BC200020F8B5C046F8BC08BC9E467047F3
:102B2000F8B5C046F8BC08BC9E46704700000000DF
:102B300000000000AD210000C3210000B72100000B
:102B40009A9999999999B93F7B14AE47E17A843F54
:102B50002D431CEBE2361A3F3A8C30E28E79453E2B
:102B6000BC89D897B2D29C3C33A7A8D523F6493963
:102B70003DA7F444FD0FA5329D978CCF08BA5B2585
:102B8000436FAC642806C80A00000000000024401F
:102B90000000000000005940000000000088C34011
:102BA0000000000084D797410080E03779C341439B
:102BB000176E05B5B5B89346F5F93FE9034F384DA3
:102BC000321D30F94877825A3CBF737FDD4F15754F
:102BD0004745540050555400763100617069006DCE
:102BE000616E6167656D656E74006170706C6963BC
:102BF0006174696F6E2F6A736F6E00746578742FDD
:102C00006576656E742D73747265616D0074657898
:102C1000742F706C61696E3B2063686172736574B8
:102C20003D7574662D38003A4346494C3B00536568
:102C3000727665725472616E73616374696F6E4906
:102C40004400485454502F312E312000323030206F
:102C50004F4B00436F6E74656E742D547970653AF6
:102C60002020003230312043726561746564003287
:102C70003034204E6F20436F6E74656E74003430B4
:102C80003020426164205265717565737400343080
:102C900034204E6F7420466F756E640034313420DA
:102CA000526571756573742D55524920546F6F20AC
:102CB0004C6F6E67003431352052657175657374E1
:102CC00020456E7469747920546F6F204C6172676F
:102CD000650035303020496E7465726E616C20532A
:102CE0006572766572204572726F720064617461FC
:102CF0003A20003A4346494C3B303B2300436F6E39
:102D000074656E742D4C656E6774683A00616C7002
:102D1000616361646973636F7665727931007B22E8
:102D2000416C70616361506F7274223A38307D007B
:102D30004572726F724E756D626572004572726F88
:102D4000724D657373616765003A494D45533B2089
:102D500020537472696E67204572726F7220666FBD
:102D6000726D6174203A200049534C56003A495321
:102D70004C563B230049564533003A575645333BA2
:102D800000312E310049444533003A574445333B26
:102D9000004D6963726F636F6E74726F6C657572EC
:102DA0002041726475696E6F206E616E6F20494FAD
:102DB000542033332043616C696267756964650030
:102DC0004354454D003A4354454D3B00435354450D
:102DD00000434754450046494C300046494C3100B9
:102DE00046494C32003A494D45533B4D6F6465208E
:102DF0006E6F6E207065726D69733B230046494C9F
:102E0000330046494C34004346494C0043474D4F3C
:102E1000003A43524D4F3B0043534D4F003A494D0A
:102E200045533B5B43616C69627265785D20436129
:102E30006C6962726578206D6F646520757064617D
:102E400074653B23003A494D45533B5B43616C69D4
:102E5000627265785D206E6F2076616C69642076A1
:102E6000616C75652063616C6962726578206D6F55
:102E70006465203B23003A494D45533B5B43616CFD
:102E800069627265785D206E6F2076616C6964207E
:102E900076616C7565202063616C6962726578206B
:102EA000736572766F3B23004353504F003A435390
:102EB000504F3B23003A4353504F3B4F4B3B230073
:102EC0003A4353504F3B4E4F3B23004353414F0037
:102ED0003A494D45533B5B43616C69627265785D6D
:102EE000204F70656E20736572766F20616E676C1F
:102EF00065207570646174653B23003A494D455304
:102F00003B5B43616C69627265785D206E6F207611
:102F1000616C69642076616C756520736572766F8B
:102F200020616E676C653B230043534143003A497F
:102F30004D45533B5B43616C69627265785D20432C
:102F40006C6F736520736572766F20616E676C6558
:102F5000207570646174653B23004347414F003A1C
:102F60004352414F3B0043474143003A43524143A0
:102F70003B00435357490041502043616C696272E2
:102F80006578003A494D45533B576966692053536C
:102F900049443A00205265626F6F742E2E2E3B23F7
:102FA0000043475749003A435257493B0073657401
:102FB0007570003C68323E53657475702043616CD7
:102FC00069624C69676874203C2F68323E3C6272CB
:102FD0003E203C68333E3C6120687265663D226855
:102FE000747470733A2F2F7370656374726F2D75DC
:102FF0007665782E746563682F3F703D32393637B9
:10300000223E557365205556455834204D616E61FA
:1030100067657220746F20736574757020746865BD
:10302000206465766963653C2F613E3C2F68333EC2
:1030300000746578742F68746D6C006170697665D2
:103040007273696F6E7300636F6E66696775726520
:1030500064646576696365730056616C75650049E3
:103060006E76616C6964206D6574686F64200044DD
:1030700065766963654E616D650043616C69624C9C
:1030800069676874004465766963655479706500A2
:10309000537769746368004465766963654E756D3E
:1030A00062657200556E69717565494400536572B9
:1030B0007665724E616D65004D616E756661637413
:1030C00075726572004E6963652050656F706C653E
:1030D000004D616E756661637475726572566572D6
:1030E00073696F6E004A756C20313720323032368A
:1030F0000031363A34323A3233004C6F63617469CE
:103100006F6E00636F6D6D616E64626C696E6400FA
:10311000636F6D6D616E64626F6F6C00636F6D6D78
:10312000616E64737472696E67004E6F20636F6DB9
:103130006D616E64626C696E6420617661696C6158
:10314000626C65004E6F20636F6D6D616E64626FBF
:103150006F6C20617661696C61626C6500636F6E93
:103160006E6563746564004E6F20636F6D6D616E94
:1031700064737472696E6720617661696C61626CF8
:103180006500636F6E6E656374696E6700436F6E92
:103190006E65637465640042616420726571756573
:1031A000737400646973636F6E6E65637400647238
:1031B00069766572696E666F002C20566572736958
:1031C0006F6E3A2000647269766572766572736913
:1031D0006F6E0043616C69624C6967687420627548
:1031E000696C64696E20416C70616361206472690E
:1031F00076657200737570706F7274656461637464
:10320000696F6E730066696C3165787400696E74FD
:1032100065726661636576657273696F6E0061637E
:1032200074696F6E006D61787377697463680063A9
:10323000616E6173796E6300416374696F6E0050F3
:103240006172616D657465727300253342003A46A0
:10325000494C313B00496E76616C6964206F722085
:103260006D697373696E6720706172616D657465F5
:10327000720063616E77726974650063616E636585
:103280006C6173796E6300537769746368206E753F
:103290006D626572206F7574206F662072616E6753
:1032A000650064657669636573746174650067655C
:1032B0007473776974636864657363726970746941
:1032C0006F6E004964006765747377697463686E34
:1032D000616D650047657453776974636856616C06
:1032E0007565300047657453776974636856616C1F
:1032F0007565310047657453776974636856616C0E
:103300007565320047657453776974636856616CFC
:103310007565330047657453776974636856616CEB
:1033200075653400676574737769746368004D6F01
:10333000646520646520666F6E6374696F6E6E6588
:103340006D656E740046696C310046696C320046EA
:10335000696C330046696C3400676574737769740F
:10336000636876616C7565006D696E737769746307
:103370006876616C7565006D6178737769746368F0
:1033800076616C7565007365747377697463680042
:1033900073657473776974636876616C75650073BF
:1033A0007769746368737465700053746174650041
:1033B00054727565003A43534D4F3B003A46494CB1
:1033C000303B23003A46494C313B23003A46494CB6
:1033D000323B23003A46494C333B23003A46494CA2
:1033E000343B23007365747377697463686E616D31
:1033F000650056616C7565206F7574206F6620726C
:10340000616E6765007365746173796E63007365DF
:10341000746173796E6376616C75650043616E6E7D
:103420006F74206D6F6469667920746865206E61C1
:103430006D650073746174656368616E6765636F61
:103440006D706C657465004E6F204173796E6320FA
:103450006F7065726174696F6E20666F7220746838
:10346000697320737769746368004E6F20417379C4
:103470006E63206F7065726174696F6E20666F7223
:1034800020737769746368006572726F7220757259
:103490006C002F003D002600436C69656E74547209
:1034A000616E73616374696F6E4944003F00636CC1
:1034B00069656E747472616E73616374696F6E694D
:1034C00064001B001C001C001A001A001B000000F6
:1034D00000000000000000000000000000000000EC
:1034E00000000000000000000000000000000000DC
:1034F00000000000000000000000000000000000CC
:1035000000000000000000000000000000000000BB
:103800001213140F10116E756C6C002F2F272722C6
:10381000225C5C6208660C6E0A720D7409005C75AD
:103820003030303000747275650066616C7365000D
:10383000436C69656E7420636F6E6E656374653A80
:10384000200044656D61727261676520696E6974FC
:1038500069616C69736174696F6E0053746172742D
:10386000696E67204954696D6572204F4B2C206D3D
:10387000696C6C69732829203D200043616E2774B0
:1038800020736574204954696D65722E2053656CF0
:1038900065637420616E6F7468657220667265710D
:1038A0002E206F722074696D6572004C65206D6FFB
:1038B000646520736572766F203A20003A494D4561
:1038C000533B4D6F646520736572766F206E6F6E2B
:1038D0002076616C6964653B2300416E676C6520EE
:1038E000736572766F20706F736974696F6E206F85
:1038F00070656E203A20003A494D45533B616E6732
:103900006C6520736572766F20706F736974696F70
:103910006E206F70656E206E6F742076616C6964C6
:103920003B2300416E676C6520736572766F207073
:103930006F736974696F6E20636C6F7365203A20D2
:10394000003A494D45533B616E676C652073657263
:10395000766F20706F736974696F6E20636C6F731C
:1039600065206E6F742076616C69643B23003A4970
:103970004D45533B4572726575723A206D6F6475A3
:103980006C652057694669204E494E41206162733B
:10399000656E743B23003A494D45533B436F6E6E51
:1039A000656374696F6E20776966692E2E2E3B23DE
:1039B00000417474656D7074696E6720746F206364
:1039C0006F6E6E65637420746F206E6574776F72AE
:1039D0006B2C20535349443A20003A494D45533B00
:1039E00044C3A9636F75766572746520416C70611C
:1039F00063612064C3A96D617272C3A9003A494D25
:103A000045533B44C3A9636F757665727465204165
:103A10006C70616361206E6F6E20646973706F6E8D
:103A200069626C65003A494D45533B44656D61726E
:103A3000726167652041502E2E2E3B23006E696314
:103A40006570656F706C650043414C494252455842
:103A5000003A494D45533B41502065636865633BDF
:103A600023003A494D45533B4150204F4B2049508C
:103A70003A20003A494D45533B4D41433A003A49BB
:103A80004D45533B53657276657220737461727451
:103A900065642E3B230046494E20494E4954494116
:103AA0004C49534154494F4E003A494D45533B57B9
:103AB00069666920636F6E6E656374696F6E2066F8
:103AC00061696C65642120003A494D45533B576953
:103AD0006669204F4B2049503A200005010906A194
:103AE000018502050719E029E715002501750195F3
:103AF0000881029501750881039506750815002552
:103B0000730507190029738100C000000000000040
:103B100000000000117D00005D7B0000FD20000022
:103B20000121000000000000000000002A2B2800F6
:103B30000000000000000000000000000000000085
:103B4000000000002C9EB4A0A1A2A434A6A7A5AE9C
:103B5000362D3738271E1F20212223242526B33354
:103B6000B62EB7B89F8485868788898A8B8C8D8E80
:103B70008F909192939495969798999A9B9C9D2F4C
:103B80003130A3AD350405060708090A0B0C0D0EEC
:103B90000F101112131415161718191A1B1C1DAF2C
:103BA000B1B0B5000000000000000000397E000048
:103BB000617D0000DD7D0000397D00005E00BC00FD
:103BC0007701005EBCE2613FDD83C29C7E20A3FDE5
:103BD0001F41009D23BE46DB65F88C11AF32CA57EA
:103BE000E9744E6F20536F636B6574206176616971
:103BF0006C61626C650000000000000000000000C5
:103C0000318C0000C78C0000FD200000498C0000B2
:103C10001D8D0000358D0000798D00007D8F000026
:103C2000598C0000618D0000319000006D90000003
:103C30004B8C0000CD8D0000B98E00001D8F000060
:103C4000558E0000A58C0000BF8C00002D8E00005A
:103C5000458C0000AB8D0000898D00000000000045
:103C600000000000B1900000C5900000FD200000A1
:103C7000012100001F910000000000000000000072
:103C8000DF9100000F930000FD200000F391000081
:103C9000DB910000219300007D930000F59100006E
:103CA0002992000069920000D592000089920000DC
:103CB0000593000051930000DD930000D1910000B6
:103CC000BB9300009993000000000000000000007A
:103CD00000000000000000000000000000000000E4
:103CE00000000000000000000000000000000000D4
:103CF00000000000000000000000000000000000C4
:103D000000000000000000000000000000000000B3
:104200000800000010000000200000004000000036
:104210008000000000010000000200000004000017
:10422000010203000000000000000000B1A4000033
:1042300025A50000C3A40000CDA4000091A40000A7
:1042400031A5000075A50000B1A60000B1A50000D1
:10425000AFA40000AFA4000061A60000B3A400005A
:10426000010000001700000003000000040000002F
:10427000FF00FFFFFFFFFF0001000000160000002D
:104280000300000004000000FF00FFFFFFFFFF002D
:10429000010000000A000000080000001C000000EF
:1042A000FF00000500050A00010000000B000000EF
:1042B000080000001C000000FF00010501050B00C4
:1042C0000000000007000000080000001C000000C3
:1042D000070001010101FF000000000005000000CF
:1042E000080000001C000000050001000100FF00A4
:1042F0000000000004000000080000001C00000096
:10430000040000000000FF000000000006000000A4
:1043100008000000040000000600FFFFFFFFFF0090
:10432000000000001200000008000000040000006F
:10433000FF00FFFFFFFFFF0000000000140000006F
:10434000080000002C000000FF0002000200040032
:104350000000000015000000080000002C00000014
:10436000FF00030003000500000000001000000033
:10437000020000001C000000FF000002000200001C
:104380000000000013000000020000001C000000FC
:10439000FF0001030103FF00000000001100000006
:1043A0000200000004000000FF00FFFFFFFF01000B
:1043B00000000000020000000100000006000000F4
:1043C0000000FFFFFFFFFF000100000002000000EF
:1043D00001000000040000000A00FFFFFFFF0200D0
:1043E000000000000B000000010000002C00000095
